:020000040800F2
:1000000000040020E10100080D0E0008110E000898
:10001000650E0008110E0008390E0008E301000803
:10002000E3010008E3010008E30100083D2F000898
:10003000E3010008E3010008E3010008E301000810
:10004000E3010008E3010008E3010008E301000800
:10005000E3010008E30100089D310008C9310008F0
:10006000F5310008213200084D320008E301000894
:10007000E3010008E3010008E3010008E3010008D0
:10008000E3010008E3010008E3010008E3010008C0
:10009000E3010008E3010008E301000879320008E9
:1000A000E3010008E3010008E3010008E3010008A0
:1000B000B92F0008E3010008E3010008E30100088C
:1000C000E3010008E3010008E3010008E301000880
:1000D000E3010008E3010008E3010008E301000870
:1000E000E1320008E3010008E3010008E301000831
:1000F000E3010008E3010008E3010008E301000850
:10010000E3010008E3010008E3010008E30100083F
:10011000E3010008E3010008E3010008E30100082F
:10012000E3010008E3010008E3010008E30100081F
:10013000E3010008E3010008E3010008E30100080F
:10014000E3010008E3010008E3010008912600082C
:10015000E3010008E3010008E3010008E3010008EF
:10016000E3010008E3010008E3010008E3010008DF
:10017000E3010008E3010008E3010008E3010008CF
:10018000E3010008E3010008E3010008E3010008BF
:10019000E3010008E3010008E3010008E3010008AF
:1001A000E3010008E3010008E3010008E30100089F
:1001B000E3010008E3010008E3010008E30100088F
:1001C000E3010008E3010008E3010008E30100087F
:1001D000E3010008E3010008E3010008E30100086F
:1001E00002E000F000F8FEE772B6394880F30888B4
:1001F000384880F3098838484EF60851CEF200019D
:10020000086040F20000CCF200004EF63471CEF2ED
:1002100000010860BFF34F8FBFF36F8F40F2000003
:10022000C0F2F0004EF68851CEF200010860BFF334
:100230004F8FBFF36F8F4FF00000E1EE100A4EF6C4
:100240003C71CEF200010860062080F31488BFF3F1
:100250006F8F01F0E5FE02F007FE4FF055301F49A9
:100260001B4A91423CBF41F8040BFAE71C49194A6A
:1002700091423CBF41F8040BFAE71A491A4A1B4B5A
:100280009A423EBF51F8040B42F8040BF8E70020F5
:100290001749184A91423CBF41F8040BFAE701F0B4
:1002A000C3FE02F03DFE144C144DAC4203DA54F888
:1002B000041B8847F9E700F03FF8114C114DAC42A0
:1002C00003DA54F8041B8847F9E701F0ABBE0000DD
:1002D000000400200024002000000008000000208E
:1002E00000040020F8360008002400202824002004
:1002F0002824002018300020E0010008E001000858
:10030000E0010008E00100082DE9F04F2DED108A12
:10031000C1F80CD0C3689D46BDEC108ABDE8F08FD3
:10032000002383F311882846A047002001F0FCFA3F
:1003300001F0ACFA00DFFEE71A4B6FF07A0270B5FD
:1003400000241A700F225C709C70DC701C715C7150
:100350009C71DC711C725C729A72DC7201F032FE6C
:10036000064601F057FE054650B90F4B9E4217D086
:1003700001339E4241F2883412BF05460024012514
:10038000002001F029FE0DB100F0B4F800F012FDDC
:1003900000F0F4FB204600F00BF900F0ABF8F9E7B1
:1003A0000446EDE728240020010007B008B500F05E
:1003B00087FBA0F120035842584108BD07B5054B03
:1003C00002211B88ADF8043001A800F0C7FB03B080
:1003D0005DF804FBC4330008064991F8243033B1BA
:1003E00000230822086A81F8243000F0E9BB0120CC
:1003F000704700BF482400202DE9F84F234C94F8A3
:1004000024300546884617468BBB2E46DFF87C9085
:10041000002F38D094F824A0BAF1000F05D1202283
:10042000FF214846266200F0B3FCCAF10805BD4230
:1004300028BF3D465FFA85FBAD0041462A4604EBE6
:100440008A0000F07BFC94F82430A7EB0B079B4458
:100450005FFA8BFBBBF1080F2E44A844FFB284F86F
:1004600024B0D5D1FFF7B8FF0028D1D108E0266A23
:1004700006EB8306B042C9D0FFF7AEFF0028C4D117
:100480000020BDE8F88F0120BDE8F88F4824002047
:1004900010B5202383F311881248C3680BB101F013
:1004A000C9FA0023104A0F484FF47A7101F086FA16
:1004B000002383F311880D4C236813B12368013B9B
:1004C0002360636813B16368013B6360084B1B786A
:1004D00033B9636823B9022000F026FC322363603D
:1004E00010BD00BF342400209104000878250020AE
:1004F0007024002010B5254B254953F8042F0132F4
:1005000000D110BD8B42F8D1224C234B22689A4275
:100510003AD9224B9B6803F1006303F580339A427A
:1005200032D2002000F044FB1D4B0220187000F076
:10053000F1FB1C4B1A6C00221A64196E1A66196EB4
:10054000596C5A64596E5A665A6E5A6942F0800262
:100550005A615A6922F080025A615A691A6942F056
:1005600000521A611A6922F000521A611B6972B6B0
:100570000D4A0E4B13601B682268202181F31188FD
:100580009D4683F30888104710BD00BFFCFF00089C
:100590001C00010804000108FFFF000828240020B7
:1005A000702400200038024008ED00E0000001083F
:1005B0002DE9F04F99B0B34C01902022FF2110A8F3
:1005C000A66800F0E5FBB04A1378A346A3B9AF488C
:1005D0000121C3601170202383F31188C3680BB11C
:1005E00001F028FA0023AA4AA8484FF47A7101F0D2
:1005F000E5F9002383F31188019B13B1A54B019A00
:100600001A60A54AA349019F0292002313704B6010
:1006100099461C461D469846012000F07BFB002FA2
:1006200000F012829B4B1B68002B40F00D8219B02A
:10063000BDE8F08F0220FFF7B9FE002840F0FB81F3
:10064000019BB9F1000F08BF1F46944B1B88ADF802
:100650002C3002210BA800F081FADDE74FF47A700C
:1006600000F02EFA031E0393EADB0220FFF79EFE42
:1006700082460028E4D0039B581E042800F2DD8146
:10068000DFE800F0030E1114170018A8052340F846
:10069000343D042100F062FA54464FF0000856E061
:1006A00004217848F6E704217D48F3E704217D48DA
:1006B000F0E71C24204600F07DFA04340B9004215E
:1006C0000BA800F04BFA2C2CF4D1E5E7002DB7D0A5
:1006D000002CB5D00220FFF769FE0546002800F087
:1006E000AF8101206C4C00F063FA0220207000F012
:1006F00011FB4FF000095FFA89FA504600F068FAE2
:10070000074658B1504600F073FA09F10109002874
:10071000F1D12C46A9460027634B97E7012302201D
:10072000237000F0EDFA3E46DBF808309E4206D218
:10073000304600F03FFA0130EBD10436F4E7029B7B
:1007400000261E70534BA9465E602C46374600F0CB
:1007500027FB15B1002C18BF0027FFF72FFE5BE722
:10076000002D3FF46DAF002C3FF46AAF029B0220D6
:10077000187000F0CFFA322000F0A2F9B0F1000AB0
:10078000C0F25E811AF0030540F05A81DBF80820C0
:1007900006EB0A03934200F25381BAF5807F00F220
:1007A0004F8155450DDA4FF47A7000F089F90490C5
:1007B000049B002BC0F244813C4A049BAB5401359E
:1007C000EFE7C820FFF7F2FD0546002800F038816A
:1007D0001F2E11D8C6F12004544528BF544610AB33
:1007E00026F0030022463149184400F0A7FA2246B9
:1007F000FF212E4800F0CCFA4FEAAA0A5FFA8AF2EB
:100800002A493046FFF7F8FD0446002800F01A8117
:1008100006EB8A0605469AE70220FFF7C7FD002887
:100820003FF40EAFFFF7D8FD00283FF409AF4FF0BB
:10083000000A5346DBF8082092451CD2BAF11F0F7C
:1008400012D8109A01320FD02AF0030218A90A44D4
:1008500052F8202C0B92184604220BA900F016FB2C
:100860000AF1040A0346E5E75046039300F0A2F9B3
:10087000039B0B90EFE718A8042140F84C3D00F0D3
:100880006DF964E72824002074250020342400201A
:10089000910400087825002070240020C633000849
:1008A0002C24002030240020C833000874240020A9
:1008B00018A8002340F8343D642100F02BF90028EB
:1008C0007FF4BEAE0220FFF771FD00283FF4B8AE02
:1008D0000B9800F09FF918AB43F8480D0421184617
:1008E000CDE718A8002340F8343D642100F012F948
:1008F00000287FF4A5AE0220FFF758FD00283FF442
:100900009FAE0B9800F094F918AB43F8440DE5E75F
:100910000220FFF74BFD00283FF492AE00F08EF965
:1009200018AB43F8400DD9E70220FFF73FFD002840
:100930003FF486AE0BA9142000F086F9824618A871
:10094000042140F83CAD00F009F951460BA896E7A8
:10095000322000F0B5F8B0F1000AFFF671AE1AF0DF
:10096000030F7FF46DAEDBF808200AEB0803934217
:100970003FF666AE0220FFF719FD00283FF460AE97
:100980002AF0030AC244D0453FF4E1AE404600F0ED
:1009900011F904210A900AA800F0E0F808F104080F
:1009A000F1E74FF47A70FFF701FD00283FF448AEFD
:1009B000FFF712FD00283FF4AFAE109B01330CD0BF
:1009C000082210A90020FFF717FD00283FF4A4AE6D
:1009D0002022FF2110A800F0DBF9FFF7EFFC3748D9
:1009E00000F0A8FF23E6002D3FF42AAE002C3FF4D0
:1009F00027AE18A8002340F8343D642100F08AF89F
:100A0000824600287FF41CAE0220FFF7CFFC0028AE
:100A10003FF416AE0390FFF7D1FC41F2883000F0AE
:100A200089FF0B9800F0F0F900F0BAF9039B5746E4
:100A30001C461D46F0E5054689E64FF00008FFE537
:100A40002546FDE52C4667E6002000F039F80490C5
:100A5000049B002BFFF6E3AD012000F051F9049B4D
:100A6000213B122B3FF6D8AD01A252F823F000BF74
:100A7000350600085D060008CD06000819060008C6
:100A80001906000819060008610700085109000846
:100A900019080008B1080008E30800081109000857
:100AA000190600082909000819060008A30900080A
:100AB0004F07000819060008E7090008A086010092
:100AC00037B5114B1A780132D2B20024012A0146FF
:100AD0008DF8074011D80D4803681D6A4FF47A73EA
:100AE0004B4301220DF10701A847012805D1084B0E
:100AF0009DF807001C7003B030BD4FF4FA7000F091
:100B000019FF4FF0FF30F6E70024002048260020B0
:100B10008425002038B50E4B1A780132D2B2012A52
:100B200005460ED80B4803681C6A4FF47A734B4392
:100B300004222946A047042803D1074B002018703F
:100B400038BD4FF4FA7000F0F5FE4FF0FF3038BDBD
:100B500000240020482600208425002030B4054CC5
:100B60002368DD69044B0A46AC460146204630BC8A
:100B7000604700BF48260020A086010070B501F044
:100B800025F9094C094E20700025306823788342EE
:100B900008D901F015F9336805440133B5F5803FF4
:100BA0003360F2D370BD00BF852500208025002072
:100BB00001F0BAB900F1006000F5803000687047BC
:100BC00000F10060920000F5803001F045B90000AE
:100BD000054B1A68054B1B789B1A834202D91044B7
:100BE00001F0EEB800207047802500208525002008
:100BF00038B5074D04462868204401F0E9F828B9C3
:100C000028682044BDE8384001F0FAB838BD00BF7C
:100C10008025002010F0030308D1B0F5007F05D82F
:100C200000F10050A0F508400068704700207047B0
:100C3000014BC058704700BF107AFF1F014B186866
:100C4000704700BF002004E070B52A4B1C68C4F355
:100C50000B03240C63B140F21342934231D040F2B3
:100C6000194293422FD040F2214293422DD10323C7
:100C7000214A0C2505FB03235D6893F9082042F205
:100C800001039C4224D0B4F5805F23D041F20103DC
:100C90009C4221D041F203039C421FD041F2070342
:100CA0009C4208BF3122441E0C44013D0B46A34226
:100CB0001ED215F9016F581C96B1034600F8016C5D
:100CC000F5E70123D4E70223D2E73F220B4DD6E715
:100CD0003322E3E74122E1E75A22E4E75922E2E73F
:100CE0002C2584421D7001D9981C5A70401A70BD81
:100CF0001846FBE7002004E0D8330008CC33000896
:100D0000022802BF024B4FF080729A61704700BF09
:100D100000000240022802BF024B4FF480729A6129
:100D2000704700BF00000240022801BF024A536919
:100D300083F48073536170470000024010B50023B4
:100D4000934203D0CC5CC4540133F9E710BD0000DA
:100D500030B5441E14F9010F0B4660B193F90050F1
:100D6000854201F1010106D11AB993F90020801AD8
:100D700030BD013AEEE7002AF7D1104630BD000041
:100D800002460346981A13F9011B0029FAD170474D
:100D900002440346934202D003F8011BFAE770476E
:100DA000024B1A78024B1A70704700BF842500204E
:100DB0000024002038B5104D104C284600F002F9F0
:100DC0002146284600F02AF924680D48626DD2F8C1
:100DD000043843F00203C2F8043800F0ABFD0949BF
:100DE000204600F027FA626DD2F8043823F002039F
:100DF000C2F8043838BD00BF48260020A4340008DB
:100E000040420F00CC34000870470000FEE70000AD
:100E100000B59BB0EFF3098168226846FFF78EFFAB
:100E2000EFF30583034B9A6B9A6A9A6A9A6A9A6AF5
:100E30009B6AFEE700ED00E000B59BB0EFF309818F
:100E400068226846FFF77AFFEFF30583044B9A6B3D
:100E50009A6A9A6A9A6A9A6A9A6A9B6AFEE700BFD5
:100E600000ED00E000B59BB0EFF309816822684611
:100E7000FFF764FFEFF30583034B5A6B9A6A9A6A94
:100E80009A6A9A6A9B6AFEE700ED00E030B5084D69
:100E90000A4491420BD011F8013B09245840013C0F
:100EA000F7D040F300032B4083EA5000F7E730BD52
:100EB0002083B8ED002304491A465A50C818083355
:100EC000802B4260F9D17047882500200268436872
:100ED0001143016003B118477047000013B5446B1C
:100EE000D4F894341A681178042915D1217C022988
:100EF00012D11979128901238B4013420CD101A917
:100F000004F14C0001F02AFED4F89444019B2179AD
:100F10000246206800F0DAF902B010BD143001F08A
:100F2000ADBD00004FF0FF33143001F0A7BD00004D
:100F30004C3001F07FBE00004FF0FF334C3001F029
:100F400079BE0000143001F07BBD00004FF0FF318E
:100F5000143001F075BD00004C3001F04BBE0000B4
:100F60004FF0FF324C3001F045BE0000D0F8942421
:100F700038B5136819780429054601D0012038BD19
:100F8000017C0229FAD112795C8901209040044049
:100F9000F4D105F1140001F00DFD02460028EDD05A
:100FA000D5F894544FF480732868697900F07CF97F
:100FB000204638BD406BFFF7D9BF000000207047C6
:100FC000704700007FB5124B0360002343608360CD
:100FD000C360012502260F4B05740446029001935D
:100FE00000F18402294600964FF48073143001F01A
:100FF000BDFC094B0193029400964FF4807304F5F5
:101000002372294604F14C0001F084FD04B070BD48
:1010100028340008B50F0008DD0E00080B682022F8
:1010200082F311880A7903EB820290614A790932CE
:1010300043F822008A7912B103EB820398610223FC
:101040000374C0F89414002383F3118870470000E0
:1010500038B5037F044613B190F85430ABB9201D66
:1010600001250221FFF732FF04F1140025776FF00C
:10107000010100F087FC84F8545004F14C006FF03B
:101080000101BDE8384000F07DBC38BD10B501213C
:1010900004460430FFF71AFF0023237784F8543006
:1010A00010BD000038B504460025143001F076FC70
:1010B00004F14C00257701F045FD201D84F85450C3
:1010C0000121FFF703FF2046BDE83840FFF74EBF80
:1010D00090F8443003F06003202B19D190F845209C
:1010E000212A0AD0222A4FF000030ED0202A0FD145
:1010F000084A82630722C26304E0064B8363072326
:10110000C36300230364012070478363C363F9E76B
:101110000020704701240020D0F8943437B51A68B5
:101120001178042904461AD1017C022917D11979B2
:10113000128901238B40134211D100F14C0528463E
:1011400001F0C0FD58B101A9284601F007FDD4F80F
:101150009444019B21790246206800F0B7F803B05F
:1011600030BD000000EB8103F7B59C6905460E46D3
:10117000F4B1202383F3118805EB8607201D082195
:10118000FFF7A4FEFB685B691B684C3413B1204673
:1011900001F0F2FC01A9204601F0E0FC024648B152
:1011A000019B3146284600F091F8002383F3118813
:1011B00003B0F0BDFB685A691268002AF5D01B8A9B
:1011C000013B1340F1D105F14402EAE7093138B59A
:1011D00050F82140DCB1202383F31188D4F8942403
:1011E0001368527903EB8203DB689B695D6845B144
:1011F00004216018FFF76AFE294604F1140001F08B
:10120000E3FB2046FFF7B2FE002383F3118838BDCD
:101210007047000000F08EBF01230370002343607D
:10122000C36183620362C3624362036303814381D8
:101230007047000038B50446202383F31188002549
:101240004160C56005614561856100F083FF02234F
:10125000237085F3118838BD70B500EB8103054616
:101260005069DA600E46144618B110220021FFF7CB
:101270008FFDA06918B110220021FFF789FD3146CA
:101280002846BDE8704001F02FB80000028902F046
:1012900001020281428902F00102428100220261C0
:1012A0004261826101F0B4B8F0B400EB8104478977
:1012B000E4680125A4698D403D43458123600023F6
:1012C000A2606360F0BC01F0CFB80000F0B400EBA6
:1012D00081040789E468012564698D403D430581E7
:1012E00023600023A2606360F0BC01F049B90000F4
:1012F00070B50223002504460370A0F84C5080F816
:101300004E5080F84F5005814581C56005614561AB
:10131000856180F8345000F083FF63681B6823B157
:1013200029462046BDE87040184770BD43680278E2
:101330001B6880F85020052202700BB10421184769
:1013400070470000436890F850201B6802700BB192
:10135000052118477047000090F8343070B50446F6
:1013600013B1002380F8343004F14402204601F028
:1013700071F863689B6863BB94F8445015F060068D
:1013800015D194F8453005F07F0545EA032540F274
:1013900002339D4200F00E815BD8022D00F0DC800C
:1013A0003FD8002D00F08780012D00F0CF80002174
:1013B000204601F0A7FA0021204601F099FA63685F
:1013C0001B6813B1062120469847062384F8343061
:1013D00070BD204698470028CED094F84B2094F852
:1013E0004A3043EA0223E26B934238BFE36394F945
:1013F0004430E56B002B4FF0200380F2FD80002D80
:1014000000F0EC80092284F8342083F31188002155
:10141000E36BA26B2046FFF759FF002383F311888B
:1014200070BDB5F5817F00F0B180B5F5407F49D042
:10143000B5F5807FBBD194F84630012BB7D1B4F815
:101440004C3023F00203A4F84C30A663E663266414
:10145000C3E740F201639D421ED8B5F5C06F3BD291
:10146000B5F5A06FA3D1B4F84430B3F5A06F0ED199
:1014700094F8463084F84E30204600F029FF636827
:101480001B6813B1012120469847032323700023D2
:10149000A363E3632364A0E7B5F5106F32D040F691
:1014A00002439D4252D0B5F5006F80D104F14F0345
:1014B000A363012324E004F14C03A3630223E36349
:1014C00025648AE794F84630012B7FF470AFB4F8B6
:1014D0004C3043F00203B6E794F84920616894F871
:1014E00048304D6894F8471043EA0223204694F8A8
:1014F0004620A84700283FF45AAF4368A363036817
:10150000E363A4E72378042B10D1202383F311880D
:101510002046FFF7BBFE86F31188636884F84F60AE
:101520001B68032121700BB12046984794F8463080
:10153000002BACD084F84F300423237063681B6801
:10154000002BA4D0022120469847A0E7374BA36385
:101550000223E36300239DE794F8481011F0800F05
:10156000204601F00F010ED000F066FF012806D0E2
:1015700002287FF41CAF2E4BA363E06367E72D4B7B
:10158000A363E56363E700F049FFEFE794F84630B3
:10159000002B7FF40CAF94F8483013F00F013FF4A8
:1015A00076AF1A06204602D501F0C0F96FE701F0C8
:1015B000B3F96CE794F84630002B7FF4F8AE94F85A
:1015C000483013F00F013FF462AF1B06204602D5EE
:1015D00001F098F95BE701F08BF958E7142284F8E1
:1015E000342083F311882B462A4629462046FFF7EC
:1015F0005BFE85F3118870BD5DB1152284F834203F
:1016000083F311880021E36BA26B2046FFF74CFEA9
:1016100003E70B2284F8342083F311882B462A46F3
:1016200029462046FFF752FEE3E700BF5834000882
:10163000503400085434000838B590F8343004466B
:10164000152B29D8DFE803F03E28282828283E2833
:10165000280B293928282828282828283E3E90F8B1
:101660004B1090F84A20C36B42EA01229A4214D9E7
:10167000C268128AB3FBF2F502FB15356DB920235F
:1016800083F311882B462A462946FFF71FFE85F370
:1016900011880A2384F8343038BD142384F8343098
:1016A000202383F3118800231A4619462046FFF7AA
:1016B000FBFD002383F3118838BD036C03B1984709
:1016C0000023E7E7002101F01DF90021204601F089
:1016D0000FF963681B6813B106212046984706235B
:1016E000D8E7000090F83420152A38B5044622D8EF
:1016F0000123934040F6416213421DD113F480153B
:101700000FD19B0217D50B2380F83430202383F3AD
:1017100011882B462A462946FFF7D8FD85F3118804
:1017200038BDC3689B695B682BB9036C03B19847EC
:10173000002384F8343038BD002101F0E3F80021A3
:10174000204601F0D5F863681B6813B106212046D6
:1017500098470623EDE70000024B00221B605B6008
:101760009A60704708260020002303748268054BA6
:101770001B6899689142FBD25A680360426010600E
:10178000586070470826002008B5202383F311888D
:10179000037C032B05D0042B0DD02BB983F31188C8
:1017A00008BD436900221A604FF0FF334361FFF721
:1017B000DBFF0023F2E790E80C001A600268536038
:1017C000F2E70000002303748268054B1B689968E8
:1017D0009142FBD85A6803604260106058607047BD
:1017E00008260020054B19690874186802681A60F9
:1017F0005360186101230374FEF786BD082600209C
:1018000030B54B1C87B005460A4C10D023690A4AF4
:1018100001A800F0D3F82846FFF7E4FF049B13B1BA
:1018200001A800F007F92369586907B030BDFFF738
:10183000D9FFF8E7082600208917000838B50C4DB5
:1018400041612B6981689A689142044603D8BDE8DA
:101850003840FFF789BF1846FFF786FF01232C6148
:10186000014623742046BDE83840FEF74DBD00BF59
:1018700008260020044B1A681B6990689B689842F0
:1018800094BF0020012070470826002010B5084CA6
:10189000236820691A6822605460012223611A7447
:1018A000FFF790FF01462069BDE81040FEF72CBD10
:1018B00008260020826002220274002242747047CF
:1018C0008368A3F17C0243F80C2C026943F83C2C9A
:1018D000426943F8382C074A43F81C2CC26843F885
:1018E000102C022203F8082C002203F8072CA3F185
:1018F000180070472103000810B5202383F31188D6
:10190000FFF7DEFF00210446FFF798FF002383F373
:101910001188204610BD0000024B1B6958610F2042
:10192000FFF760BF08260020202383F31188FFF70C
:10193000F3BF000008B50146202383F31188082077
:10194000FFF75EFF002383F3118808BD49B1064B02
:1019500042681B6918605A60136043600420FFF7F7
:101960004FBF4FF0FF3070470826002003689842B1
:1019700006D01A680260506059611846FFF7F4BE3D
:101980007047000038B504460D462068844200D1F7
:1019900038BD036823605C604561FFF7E5FEF4E74E
:1019A000054B03F114025A619A614FF0FF32DA617C
:1019B00000221A62704700BF08260020F8B50361B4
:1019C0004FF08043C2605C6A194B1A46022952F8F4
:1019D000145F38BF0221954206461F460AD158615E
:1019E00098611C620560456081600819BDE8F84097
:1019F00001F08AB9186AAB68241A0C1902D3E41AE8
:101A00002D6804E09C4202D2204401F08BF9AB68BF
:101A10009C42F4D86B68736035601E606E60B46081
:101A2000A9684FF0FF33091BA960FB61F8BD00BF37
:101A30000826002010B41B4C234653F8141F814283
:101A400010D0416802680A60026851609A424FF003
:101A50000001C16003D0936881680B4493605DF816
:101A6000044B70470A68626100209A425360C86064
:101A700003D15DF8044B01F04FB9936888680344C3
:101A800093604FF08042206A526A121A9342E6D95C
:101A9000991A012998BF931C18445DF8044B01F072
:101AA00041B900BF0826002000207047FEE7000073
:101AB000704700004FF0FF3070470000022906D049
:101AC000032906D00129064818BF002070470548A1
:101AD0007047032A9ABF044800EBC20000207047F9
:101AE00028350008DC3400080824002070B59AB0BE
:101AF00001AD064608462946144600F095F82846EA
:101B0000FFF73EF9C0B2431C5B0086E81800237063
:101B100003236370002302341946DAB2904204F1C1
:101B2000020401D81AB070BDEA5C04F8022C04F873
:101B3000011C0133F1E7000008B5202383F311886D
:101B40000348FFF7E9FA002383F3118808BD00BFBB
:101B50004826002010B50446052916D8DFE801F014
:101B600016150316161D202383F311880E4A012132
:101B7000FFF772FB20460D4A0221FFF76DFB0C4870
:101B8000FFF790FA002383F3118810BD202383F31D
:101B900011880748FFF75CFAF4E7202383F31188E4
:101BA0000348FFF773FAEDE75C340008803400085F
:101BB0004826002038B50C4D0C4C0D492A4604F13E
:101BC0000800FFF793FF05F1CA0204F1100009496C
:101BD000FFF78CFF05F5CA7204F118000649BDE84D
:101BE0003840FFF783BF00BF102B002008240020DF
:101BF000AC340008B6340008C134000870B504469F
:101C000008460D46FFF7BCF8C6B2204601340378FB
:101C10000BB9184670BD32462946FFF799F80028DF
:101C2000F3D1012070BD00002DE9F04704460D46B8
:101C3000FFF7A6F82C49C6B22046FFF7DFFF08B130
:101C40000636F6B229492046FFF7D8FF08B110360C
:101C5000F6B2632E0BD8DFF89080DFF89090244F17
:101C6000DFF898A0267846B92E70BDE8F0872146A7
:101C70002846BDE8F04701F09DBB252E2FD1072255
:101C800041462046FFF764F870B91A4B2A4603F123
:101C90000C0153F8040B42F8040B8B42F9D11B786A
:101CA000137007340D35DDE7082249462046FFF75B
:101CB0004FF8A0B9104BAA1C13F8011F090953458E
:101CC000C95D02F8021C197801F00F0102F102024D
:101CD000C95D02F8031CEFD118350834C2E72E7035
:101CE00001340135BEE700BF48350008C1340008A3
:101CF0005E350008503500080F7AFF1F1B7AFF1F62
:101D0000BFF34F8F024AD368DB03FCD4704700BF98
:101D1000003C024008B5094B1B7873B9FFF7F0FF90
:101D2000074B1A69002ABFBF064A5A6002F188327F
:101D30005A601A6822F480621A6008BD6E2D002075
:101D4000003C02402301674508B50B4B1B7893B953
:101D5000FFF7D6FF094B1A6942F000421A611A6870
:101D600042F480521A601A6822F480521A601A688B
:101D700042F480621A6008BD6E2D0020003C0240D3
:101D80000B2870B513D80B4A0B4C137863B90B4E64
:101D90004FF0006144F8231056F8235001330C2B08
:101DA0002944F7D10123137054F8200070BD00209E
:101DB00070BD00BFA02D0020702D002070350008E0
:101DC000014B53F820007047703500080C20704715
:101DD0000B2810B5044601D9002010BDFFF7D0FF35
:101DE000064B53F824301844C21A0BB9012010BD19
:101DF00012680132F0D1043BF6E700BF70350008ED
:101E00000B2810B5044621D8FFF77AFFFFF782FFB1
:101E10000F4AF323D360C300DBB243F4007343F0F3
:101E200002031361136943F480331361FFF768FF02
:101E3000FFF7A6FF074B53F8241000F0DDF8FFF77B
:101E400083FF2046BDE81040FFF7C2BF002010BD51
:101E5000003C0240703500082DE9F84312F0010300
:101E6000154640D18218B2F1016F3CD22C4B1B6851
:101E700013F0010337D02B4CFFF74CFFF323E36043
:101E8000FFF73EFF40F20127032D01D9830713D04E
:101E9000244C0F46401A40F20118EB1B0B44012B57
:101EA00000EB0706236924D823F001032361FFF721
:101EB0004BFF0120BDE8F883236923F440732361BD
:101EC00023693B43236151F8046B0660BFF34F8FD6
:101ED000FFF716FF03689E4208D0236923F0010331
:101EE0002361FFF731FF0020BDE8F883043D043093
:101EF000CAE723F440732361236943EA080323619B
:101F0000B94637F8023B3380BFF34F8FFFF7F8FE37
:101F10003688B9F80030B6B2B342BED0DDE700BFB4
:101F200000380240003C0240084908B50B7828B14F
:101F300053B9FFF7EFFE01230B7008BD23B1BDE8D5
:101F400008400870FFF700BF08BD00BF6E2D0020DD
:101F500010B50244064B0439D2B2904200D110BDF4
:101F6000441C00B253F8200041F8040FE0B2F4E73B
:101F700050280040104B30B51C6F240407D41C6F50
:101F800044F400741C671C6F44F400441C670B4C41
:101F9000236843F4807323600244094B0439D2B2AE
:101FA000904200D130BD441C00B251F8045F43F8A8
:101FB0002050E0B2F4E700BF00380240007000405B
:101FC0005028004007B5012201A90020FFF7C0FFFB
:101FD000019803B05DF804FB13B50446FFF7F2FF68
:101FE000A04206D002A9012241F8044D0020FFF7CB
:101FF000C1FF02B010BD000070470000034B1B681A
:102000009B0042BF024B01221A7070477438024095
:10201000A12D0020014B1878704700BFA12D002092
:1020200070470000FEE70000084A094B09498B424F
:1020300004D3094A0021934205D3704752F8040F94
:1020400043F8040BF3E743F8041BF4E71C370008DC
:10205000183000201830002018300020836D30B573
:1020600000229D68446D11464FF0FF3004EB42138F
:1020700001329542C3F80019C3F81019C3F80809D2
:10208000C3F8001BC3F8101BC3F8080BEED24FF0C7
:102090000113C4F81C3830BD890141F020010161F1
:1020A00003699B06FCD4122000F0C4BE204B03EB56
:1020B00080022DE9F047D2F80CE05D6DDEF81420C7
:1020C000461CD2F800C005EB063605EB40185168F7
:1020D00061450BD3D5F83428012303FA00F022EA36
:1020E0000000C5F834081846BDE8F087BEF8104077
:1020F000ACEB0103A34228BF2346D8F81849A4B289
:10210000B3EB840F10D894681F46A4F1040959F862
:1021100004AFC6F800A0042F01D9043FF7E71C4420
:102120000B4494605360D2E70020BDE8F08700BF05
:10213000A42D002010B5054C2046FFF76DF84FF098
:10214000A0436365024BA36510BD00BFA42D002012
:10215000C43500080378012B70B5054650D12A4BD1
:10216000446D98421BD1294B5A6B42F080025A634E
:102170005A6D42F080025A655A6D5A6942F08002E7
:102180005A615A6922F080025A610E2143205B692C
:1021900000F0D6FB1E4BE3601E4BC4F80038002352
:1021A000C4F8003EC02323606E6D4FF40413A36394
:1021B0003369002BFCDA012333610C2000F03AFE76
:1021C0003369DB07FCD4122000F034FE3369002BA6
:1021D000FCDA0026A6602846FFF740FF6B68C4F8CB
:1021E0001068DB68C4F81468C4F81C684BB90A4B63
:1021F000A3614FF0FF336361A36843F00103A36061
:1022000070BD064BF4E700BFA42D0020003802404B
:102210004014004003002002003C30C0083C30C0A5
:10222000F8B5446D054600212046FFF735FFA96D3E
:1022300000234FF001128F68C4F834384FF0006665
:10224000C4F81C284FF0FF3004EB431201339F42C7
:10225000C2F80069C2F8006BC2F80809C2F8080B9E
:10226000F2D20B686A6DEB65636210231361166925
:1022700016F01006FBD1122000F0DCFDD4F8003877
:1022800023F4FE63C4F80038A36943F4402343F009
:102290001003A3610923C4F81038C4F814380A4B9A
:1022A000EB604FF0C043C4F8103B084BC4F8003B50
:1022B000C4F81069C4F80039EB6D03F1100243F45F
:1022C0008013EA65A362F8BDA035000840800010C5
:1022D000426D90F84E10D2F8003823F4FE6343EAC2
:1022E0000113C2F8003870472DE9F0410EB200EB3F
:1022F00086080D46D8F80C100F6807F00303022B70
:1023000050D0032B50D03D4A3D4F012B18BF1746EC
:10231000446D4FEA451E04EB0E030022C3F8102B58
:102320008A6905F1100C002A40D04A8A05F1580349
:102330005B013A43E2500123D4F81C2803FA0CF362
:102340001343A6444A69C4F81C380023CEF8103958
:1023500005F13F03002A39D00A8A898B92080129A6
:1023600088BF4A43C16D04EB8303561841EA024219
:10237000C66529465A602046FFF78EFED8F80C3015
:102380001B8A43EA85531F4305F148035B01E7506D
:102390000123D4F81C2803FA05F51543C4F81C588A
:1023A000BDE8F081174FB3E7174FB1E704EB4613D1
:1023B000D3F8002B22F40042C3F8002BD4F81C28D9
:1023C000012303FA0CF322EA0303BAE704EB8303C5
:1023D0000E4A5A6004EB461629462046FFF75CFE7B
:1023E000D6F8003923F40043C6F80039D4F81C3875
:1023F000012202FA05F523EA0505CFE70080001067
:10240000008004100080081000800C1000040002FE
:10241000826D1268C265FFF721BE00005831436D1E
:1024200049015B5813F4004004D013F4001F14BF9B
:1024300001200220704700004831436D49015B587C
:1024400013F4004004D013F4001F14BF0120022035
:102450007047000000EB8101CB68196A0B681360BC
:102460004B6853607047000000EB810330B5DD68B6
:10247000AA691368D36019B9402B84BF4023136045
:102480006B8A1468426D1C44013CB4FBF3F4634353
:10249000033323F0030302EB411043EAC44343F048
:1024A000C043C0F8103B2B6803F00303012B09B2B3
:1024B0000ED1D2F8083802EB411013F4807FD0F827
:1024C000003B14BF43F0805343F00053C0F8003B7F
:1024D00002EB4112D2F8003B43F00443C2F8003B48
:1024E00030BD00002DE9F041244D6E6D06EB401328
:1024F0000446D3F8087BC3F8087B38070AD5D6F81A
:102500001438190706D505EB84032146DB682846F5
:102510005B689847FA072FD5D6F81438DB072BD518
:1025200005EB8403D968CCB98B69488A5E68B6FB31
:10253000F0F200FB12628AB91868DA6890420DD294
:10254000121A83E81400202383F311880B482146D4
:10255000FFF78AFF84F31188BDE8F081012303FAB5
:1025600004F26B8923EA02036B81CB6823B1214615
:102570000248BDE8F0411847BDE8F081A42D0020D5
:1025800000EB810370B5DD68436D6C692668E66019
:102590004A0156BB1A444FF40020C2F810092A68B9
:1025A00002F00302012A0AB20ED1D3F8080803EBA5
:1025B000421410F4807FD4F8000914BF40F080501A
:1025C00040F00050C4F8000903EB4212D2F80009B1
:1025D00040F00440C2F80009D3F83408012202FA9E
:1025E00001F10143C3F8341870BD19B9402E84BFFE
:1025F0004020206020682E8A841940F00050013C61
:102600001A44B4FBF6F440EAC440C6E7F8B5044601
:102610001E48456D05EB4413D3F80869C3F80869F3
:10262000F10717D5D5F81038DA0713D500EB840376
:10263000D9684B691F68DA68974218D2D21B002705
:102640001A605F60202383F311882146FFF798FF0B
:1026500087F31188330617D5D5F834280123A34012
:10266000134211D02046BDE8F840FFF71FBD0123FB
:1026700003FA04F2038923EA020303818B68002B27
:10268000E8D021469847E5E7F8BD00BFA42D00201B
:1026900096482DE9F84F456D6E69AB691E4016F4FA
:1026A000805F6E61044605D0FEF722FEBDE8F84F5C
:1026B00000F054BC002E12DAD5F8003E8B489B0780
:1026C0001EBFD5F8003E23F00303C5F8003ED5F841
:1026D000043823F00103C5F80438FEF733FE37054C
:1026E00002D58248FEF722FEB0040CD5D5F8083892
:1026F00013F0060FEB6823F470530CBF43F4105330
:1027000043F4A053EB60310704D56368DB680BB179
:1027100076489847F2025AD4B3020CD5D4F85480C4
:10272000DFF8C8A100274FF00109A36D9B68F9B23B
:102730008B4280F08780F70619D5616D0A6AC2F373
:102740000A1702F00F0302F4F012B2F5802F00F026
:10275000A180B2F5402F0AD104EB830301F580512B
:10276000DB68186A00231A469F4240F087803003D6
:10277000D5F8184813D5E10302D50020FFF7B2FEC3
:10278000A20302D50120FFF7ADFE630302D50220AC
:10279000FFF7A8FE270302D50320FFF7A3FE75036A
:1027A00084D5E00702D50020FFF730FFA10702D54E
:1027B0000120FFF72BFF620702D50220FFF726FF5B
:1027C00023077FF573AF0320FFF720FF6EE7D4F8F0
:1027D0005480DFF818A100274FF00109A36D9B6812
:1027E0005FFA87FB5B4597D308EB4B13D3F80029BF
:1027F00002F44022B2F5802F22D1D3F80029002A1A
:102800001EDAD3F8002942F09042C3F80029D3F829
:102810000029002AFBDB5946606DFFF73DFC228949
:1028200009FA0BF322EA0303238104EB8B03DB6831
:102830009B6813B15946504698475846FFF736FCF7
:102840000137CBE708EB4112D2F8003B03F44023F9
:10285000B3F5802F10D1D2F8003B002B0CDA62893F
:1028600009FA01F322EA0303638104EB8103DB68C5
:10287000DB680BB150469847013756E79C0708BF05
:102880000A68072B98BF027003F101039CBF120A6C
:10289000013069E7023304EB830201F5805152688D
:1028A00090690268D0F808C04068A2EB000E0022D0
:1028B000104697420AD104EB830463689B699A68C7
:1028C0003A449A605A6817445F6050E712F0030F69
:1028D00008BF0868964588BF8CF8000002F1010225
:1028E00084BF000A0CF1010CE3E700BFA42D002017
:1028F000436D03EB4111D1F8003B43F40013C1F8E1
:10290000003B7047436D03EB4111D1F8003943F4AC
:102910000013C1F800397047436D03EB4111D1F842
:10292000003B23F40013C1F8003B7047436D03EBF9
:102930004111D1F8003923F40013C1F80039704770
:1029400000F1604300F01F02400903F561430901F3
:102950008000C9B200F1604083F8001300F56140C7
:1029600001239340C0F880310360704730B5039C69
:102970000172043304FB0325C361049B036300213C
:10298000059B00604060C160426102618561046234
:1029900042628162C162436330BD00000022416A2D
:1029A00041610161C2608262C2626FF00101FEF7A3
:1029B000E9BF000003694269934203D1C2680AB1CA
:1029C00000207047181D704703691960C268013202
:1029D000C260C269134482690361934224BF436A9F
:1029E00003610021FEF7C2BF38B504460D46E36817
:1029F0003BB16269131D1268A3621344E3620020B5
:102A000038BD237A33B929462046FEF79FFF0028B8
:102A1000EDDA38BD6FF00100FBE70000C368C26962
:102A2000013BC3604369134482694361934224BFFD
:102A3000436A436100238362036B03B11847704705
:102A400070B52023044683F31188866A3EB9FFF7E8
:102A5000CBFF054618B186F31188284670BDA36ADE
:102A6000E26A13F8015BA362934202D32046FFF7A8
:102A7000D5FF002383F31188EFE700002DE9F84F1D
:102A800004460E4690469946202787F31188002574
:102A9000AA46D4F828B0BBF1000F09D14946204618
:102AA000FFF7A2FF20B18BF311882846BDE8F88F0D
:102AB000A16AE36AA8EB050B5B1A9B4528BF9B46FE
:102AC000BBF1400F1BD9334601F1400251F8040B12
:102AD00043F8040B9142F9D1A36A40334036A36214
:102AE0004035A26AE36A9A4202D32046FFF796FF76
:102AF0008AF311884545D8D287F31188C9E7304653
:102B00005A46FEF71BF9A36A5B445E44A3625D4428
:102B1000E7E7000010B5029C0172043303FB0421B7
:102B2000C36100238362C362039B0363049B006051
:102B30004060C46042610261816104624262436339
:102B400010BD0000026AC260426A42610261002256
:102B50008262C2626FF00101FEF714BF436902692D
:102B60009A4203D1C2680AB100207047184650F853
:102B7000043B0B6070470000C368C2690133C36047
:102B80004369134482694361934224BF436A4361AA
:102B90000021FEF7EBBE000038B504460D46E368A1
:102BA0003BB123691A1DA262E2691344E36200206B
:102BB00038BD237A33B929462046FEF7C7FE0028E0
:102BC000EDDA38BD6FF00100FBE700000369196022
:102BD000C268013AC260C2691344826903619342C8
:102BE00024BF436A036100238362036B03B1184768
:102BF0007047000070B5202304460E4683F3118809
:102C0000856A35B91146FFF7C7FF10B185F3118802
:102C100070BDA36A1E70A36AE26A01339342A36285
:102C200004D3E16920460439FFF7D0FF002080F388
:102C3000118870BD2DE9F84F04460D4691469A461D
:102C40004FF0200888F311880026B346A76A4FB9D1
:102C500051462046FFF7A0FF20B187F31188304688
:102C6000BDE8F88FA06AE76AA9EB06033F1A9F4206
:102C700028BF1F46402F1BD905F1400355F8042BF0
:102C800040F8042B9D42F9D1A36A4033A362403639
:102C9000A26AE36A9A4204D3E16920460439FFF745
:102CA00095FF8BF311884E45D9D288F31188CDE773
:102CB00029463A46FEF742F8A36A3B443D44A362E4
:102CC0003E44E5E7026943699A4203D1C3681BB9F0
:102CD000184670470023FBE7836A002BF8D0043BBB
:102CE0009B1AF5D01360C368013BC360C3691A44E3
:102CF000836902619A4224BF436A036100238362AD
:102D00000123E5E700F06CB94FF0804300225863DF
:102D10001A610222DA6070474FF080430022DA60C5
:102D2000704700004FF0804358637047FEE7000093
:102D300010B5174CFEF710FDFEF732FE8022154944
:102D40002046FEF7B7FD012344F8180C0374124B1C
:102D5000124AD96821F4E0610904090C0A431049B8
:102D6000DA60CA6842F08072CA600E490A6842F0AE
:102D700001020A601022DA77202283F82220002341
:102D800083F3118862B60848BDE81040FEF7B4BD71
:102D900030260020D035000800ED00E00003FA05E1
:102DA000F0ED00E0001000E0D83500082DE9F84F04
:102DB0001F4C4FF00008656904F11407C1464FF03D
:102DC0008043266A5B6AAA689E1B96421DD34FF019
:102DD000200AAA68236AD5F80CB0134423622B6832
:102DE000BB425F60A6EB02066361C5F80C8001D1AF
:102DF000FFF792FF89F311882869D8478AF3118871
:102E00006569AB689E42E4D2D9E76269BA420CD0E8
:102E1000916823628E1B9660A86802282CBF181840
:102E2000981CBDE8F84FFFF77DBFBDE8F88F00BFE5
:102E300008260020034B59685A68521A9042FBD862
:102E4000704700BF001000E04B6843608B688360F0
:102E5000CB68C3600B6943614B6903628B69436252
:102E60000B6803607047000008B5224B22481A69BE
:102E700040F2FF110A431A611A6922F4FF7222F02C
:102E800001021A611A691A6B0A431A631A6D0A431E
:102E90001A651A4A1B6D1146FFF7D6FF184802F152
:102EA0001C01FFF7D1FF174802F13801FFF7CCFFF3
:102EB000154802F15401FFF7C7FF144802F17001F1
:102EC000FFF7C2FF124802F18C01FFF7BDFF114866
:102ED00002F1A801FFF7B8FF0F4802F1C401FFF7A4
:102EE000B3FF0E4802F1E001FFF7AEFFBDE8084076
:102EF00000F0E0B80038024000000240F835000859
:102F00000004024000080240000C02400010024091
:102F10000014024000180240001C02400020024041
:102F200008B500F037FAFFF703FFFFF767F8BDE8D1
:102F30000840FEF73FBE000070470000064A536895
:102F400023F001035360EFF30983683383F30988A7
:102F5000002383F31188704730EF00E010B5202381
:102F600083F31188104B5B6813F4006318D0F1EE03
:102F7000103AEFF309844FF0807344F84C3C0B4B4C
:102F8000DB6844F8083CA4F1680383F30988FEF782
:102F900071FC18B1064B44F8503C10BD054BFAE7E4
:102FA00083F3118810BD00BF00ED00E030EF00E0BA
:102FB00031030008340300084FF0804310B51A694C
:102FC000920708D500241C61202383F31188FFF7A2
:102FD000EDFE84F31188BDE81040FFF7BFBF00008D
:102FE000104B1A6C42F001021A641A6E42F0010290
:102FF0001A660D4A1B6E936843F0010393604FF00D
:10300000804353229A624FF0FF32DA6200229A61C3
:103010005A63DA605A6001225A6108211A601C2042
:10302000FFF78EBC00380240002004E01F4B1A69F5
:103030006FEAC2526FEAD2521A611A69C2F30802E9
:103040001A614FF0FF301A695A69586100215A69B4
:1030500059615A691A6A62F080521A621A6A02F059
:1030600080521A621A6A5A6A58625A6A59625A6ACD
:103070001A6C42F080521A641A6E42F080521A663C
:103080001A6E0B4A106840F480701060186F00F4DC
:103090004070B0F5007F1EBF4FF48030186719678D
:1030A000536823F40073536000F054B900380240B1
:1030B00000700040304B4FF080521A642F4A4FF49A
:1030C000404111601A6842F001021A601A689207C2
:1030D000FCD59A6822F003029A60274B19469A6839
:1030E00012F00C02FBD1186800F0F90018609A6029
:1030F0001A6842F480321A600B689B03FCD54B6F50
:1031000043F001034B671C4B5A6F9007FCD51C4AD8
:103110005A601A6842F080721A60184A536859045B
:10312000FCD5154B1A689201FCD5164A9A60164BCD
:103130001A68164B9A42164B1BD1164A1168164A4A
:10314000914216D140F205121A600B4B9A6842F078
:1031500002029A609A6802F00C02082AFAD15A6CAC
:1031600042F480425A645A6E42F480425A665B6E60
:10317000704740F20572E7E70038024000700040F7
:103180000854400700948838002004E011640020AF
:10319000003C024000ED00E041C20F41084A08B582
:1031A000536911680B4003F00103536123B1054AD1
:1031B00013680BB150689847BDE80840FFF7CEBED2
:1031C000003C014088250020084A08B55369116871
:1031D0000B4003F00203536123B1054A93680BB11E
:1031E000D0689847BDE80840FFF7B8BE003C0140F2
:1031F00088250020084A08B5536911680B4003F080
:103200000403536123B1054A13690BB15069984710
:10321000BDE80840FFF7A2BE003C01408825002021
:10322000084A08B5536911680B4003F0080353615D
:1032300023B1054A93690BB1D0699847BDE80840AE
:10324000FFF78CBE003C014088250020084A08B5E5
:10325000536911680B4003F01003536123B1054A11
:10326000136A0BB1506A9847BDE80840FFF776BE75
:10327000003C014088250020174B10B55C691A6896
:10328000144004F478725A61A30604D5134A936A71
:103290000BB1D06A9847600604D5104A136B0BB186
:1032A000506B9847210604D50C4A936B0BB1D06B39
:1032B0009847E20504D5094A136C0BB1506C984746
:1032C000A30504D5054A936C0BB1D06C9847BDE8B3
:1032D0001040FFF743BE00BF003C0140882500209E
:1032E0001A4B10B55C691A68144004F47C425A61A8
:1032F000620504D5164A136D0BB1506D984723052E
:1033000004D5134A936D0BB1D06D9847E00404D5F2
:103310000F4A136E0BB1506E9847A10404D50C4AA6
:10332000936E0BB1D06E9847620404D5084A136FB0
:103330000BB1506F9847230404D5054A936F0BB126
:10334000D06F9847BDE81040FFF708BE003C014031
:1033500088250020062108B50846FFF7F1FA062166
:103360000720FFF7EDFA06210820FFF7E9FA06210A
:103370000920FFF7E5FA06210A20FFF7E1FA062106
:103380001720FFF7DDFA06212820BDE80840FFF7E7
:10339000D7BA000008B5FFF749FEFDF78BFDFDF732
:1033A00039FFFDF70DFEFFF7C7FDBDE80840FFF749
:1033B000A9BC0000034611F8012B03F8012B002AD9
:1033C000F9D17047121012131211000053544D33EB
:1033D00032463F3F3F00000000000000CC330008B1
:1033E0003F00000013040000083400083F00000004
:1033F00019040000123400083F00000021040000FE
:103400001C3400083F00000053544D333246343022
:10341000780053544D3332463432780053544D3390
:10342000324634343658580000000000390F000886
:10343000250F0008610F00084D0F0008590F000804
:10344000450F0008310F00081D0F0008BD0F0008D0
:103450000000000001000000000000000200000069
:103460000000000065110008CD1100084000400078
:10347000E02A0020F02A00200200000000000000E6
:10348000030000000000000011120008000000000E
:1034900010000000002B00200000000001000000D0
:1034A00000000000A42D002001010200417264759B
:1034B00050696C6F740025424F415244252D424C97
:1034C000002553455249414C25000000551B00087A
:1034D000BD1A0008D1100008391B00084300000085
:1034E000E434000809024300020100C0320904006C
:1034F0000001020201000524001001052401000161
:10350000042402020524060001070582030800FFC7
:1035100009040100020A0000000705010240000042
:10352000070581024000000012000000303500084D
:10353000120110010200004009124157000201026D
:10354000030100000403090425424F4152442500B1
:103550004F6D6E696275734E616E6F563600303115
:10356000323334353637383941424344454600001A
:10357000004000000040000000400000004000004B
:103580000000010000000200000002000000020034
:103590000000020000000200000002000000020023
:1035A000000000005913000839160008E51600084D
:1035B00040004000042E0020042E002001000000E6
:1035C000142E0020800000004001000003000000D5
:1035D0006D61696E00000000F0350008202E0020AB
:1035E00018300020010000002D2D00080000000010
:1035F00069646C6500000000000181420000000069
:10360000AAAAAAAA00010040FFFE000000000000D4
:1036100000A00A004000000100000000AAAAAAAA17
:1036200040000001FFFF000000000000000000005B
:103630000000000000000000AAAAAAAA00000000E2
:10364000FFFF00000000000000000000000000007C
:1036500000000000AAAAAAAA00000000FFFF0000C4
:10366000000000000000000000000000000000005A
:10367000AAAAAAAA00000000FFFF000000000000A4
:10368000000000000000000000000000AAAAAAAA92
:1036900000000000FFFF000000000000000000002C
:1036A0000000000000000000AAAAAAAA0000000072
:1036B000FFFF00000000000000000000000000000C
:1036C000000000000A0000000000000003000000ED
:1036D00000000000000000000000000000000000EA
:1036E00000000000000000000000000000000000DA
:1036F0000000000000000000FF009600000000082D
:103700000400000044350008000000000000000034
:1037100000000000000000000000000000000000A9
:10372000FFFFFFFFFFFFFFFFFFFFFFFFFFFFFFFFA9
:10373000FFFFFFFFFFFFFFFFFFFFFFFFFFFFFFFF99
:10374000FFFFFFFFFFFFFFFFFFFFFFFFFFFFFFFF89
:020000040801F1
:1000000000060020B5120108D92E0A08352E0A086C
:10001000A12E0A08352E0A086D2E0A08B71201080B
:10002000B7120108B7120108B71201085D470C08A2
:10003000B7120108B7120108B7120108B712010878
:10004000B7120108B7120108B7120108B712010868
:10005000B7120108B712010879590C08A1590C0808
:10006000C9590C08F1590C08195A0C087D020C08E2
:10007000A5020C08D1020C08FD020C0829030C088B
:1000800051030C087D030C0801020C08B71201088B
:10009000B7120108B7120108B7120108415A0C083B
:1000A000655B0C08695B0C087D5B0C08815B0C08C8
:1000B000855B0C08995B0C08AD5B0C08D50B0C0834
:1000C000E90B0C080D0C0C08210C0C08B7120108E8
:1000D000B7120108155B0C08B7120108295B0C0860
:1000E000A55A0C08B7120108B7120108B712010887
:1000F000B7120108B7120108B7120108A9030C08CA
:10010000B7120108B7120108C15B0C08B712010849
:100110003D5B0C08B7120108B7120108B7120108BD
:10012000D5030C08FD030C0829040C0855040C0821
:1001300081040C08B7120108B7120108B7120108B0
:10014000B7120108B7120108B7120108894E0C084E
:10015000A9040C08D5040C0801050C08515B0C0817
:10016000B7120108B7120108B7120108B712010847
:10017000B7120108B7120108B7120108B712010837
:10018000B7120108B7120108B7120108B712010827
:10019000B7120108B7120108B7120108B712010817
:1001A000B7120108B7120108B7120108B712010807
:1001B000B7120108B7120108B7120108B7120108F7
:1001C000B7120108B7120108B7120108B7120108E7
:1001D000B7120108B7120108B7120108B7120108D7
:1001E000693501087D660108D9A00108710402087B
:1001F0009D4D020855D40208C55204082112060874
:10020000291806084162060821B40608E5BB06085D
:100210001DBF06088D240708C5450708451A0808AC
:10022000098D0808A5270A0839220B08F57C0B0858
:1002300059A30B08CDAD0B0851DD0B0831E40B08B9
:1002400081F0004102E000BF83F0004330B54FEA87
:1002500041044FEA430594EA050F08BF90EA020FF4
:100260001FBF54EA000C55EA020C7FEA645C7FEA87
:10027000655C00F0E2804FEA5454D4EB5555B8BFAA
:100280006D420CDD2C4480EA020281EA030382EA1B
:10029000000083EA010180EA020281EA0303362DAD
:1002A00088BF30BD11F0004F4FEA01314FF4801C80
:1002B0004CEA113102D0404261EB410113F0004F92
:1002C0004FEA03334CEA133302D0524263EB430349
:1002D00094EA050F00F0A780A4F10104D5F1200EE7
:1002E0000DDB02FA0EFC22FA05F2801841F1000142
:1002F00003FA0EF2801843FA05F359410EE0A5F116
:1003000020050EF1200E012A03FA0EFC28BF4CF046
:10031000020C43FA05F3C01851EBE37101F00045FC
:1003200007D54FF0000EDCF1000C7EEB00006EEB09
:100330000101B1F5801F1BD3B1F5001F0CD3490893
:100340005FEA30004FEA3C0C04F101044FEA4452EA
:1003500012F5800F80F09A80BCF1004F08BF5FEA71
:10036000500C50F1000041EB045141EA050130BD51
:100370005FEA4C0C404141EB0101013C28BFB1F563
:10038000801FE9D291F0000F04BF01460020B1FAAE
:1003900081F308BF2033A3F10B03B3F120020CDA81
:1003A0000C3208DD02F1140CC2F10C0201FA0CF05F
:1003B00021FA02F10CE002F11402D8BFC2F1200CC4
:1003C00001FA02F120FA0CFCDCBF41EA0C0190407A
:1003D000E41AA2BF01EB0451294330BD6FEA0404C3
:1003E0001F3C1CDA0C340EDC04F11404C4F12002AE
:1003F00020FA04F001FA02F340EA030021FA04F3C0
:1004000045EA030130BDC4F10C04C4F1200220FA16
:1004100002F001FA04F340EA0300294630BD21FA54
:1004200004F0294630BD94F0000F83F4801306BF1A
:1004300081F480110134013D4EE77FEA645C18BF0E
:100440007FEA655C29D094EA050F08BF90EA020FA5
:1004500005D054EA000C04BF1946104630BD91EA9D
:10046000030F1EBF0021002030BD5FEA545C05D1A0
:100470004000494128BF41F0004130BD14F58004DF
:100480003CBF01F5801130BD01F0004545F0FE4153
:1004900041F470014FF0000030BD7FEA645C1ABF88
:1004A000194610467FEA655C1CBF0B46024650EABF
:1004B000013406BF52EA033591EA030F41F40021EB
:1004C00030BD00BF90F0000F04BF0021704730B571
:1004D0004FF4806404F132044FF000054FF0000146
:1004E00050E700BF90F0000F04BF0021704730B507
:1004F0004FF4806404F1320410F0004548BF4042DC
:100500004FF000013EE700BF42004FEAE2014FEA30
:1005100031014FEA02701FBF12F07F4393F07F4F0B
:1005200081F06051704732F07F4208BF704793F00E
:100530007F4F04BF41F40021704730B54FF4607421
:1005400001F0004521F000411CE700BF50EA010224
:1005500008BF704730B54FF000050AE050EA0102CD
:1005600008BF704730B511F0004502D5404261EB3D
:1005700041014FF4806404F132045FEA915C3FF47E
:10058000D8AE4FF003025FEADC0C18BF03325FEA1B
:10059000DC0C18BF033202EBDC02C2F1200300FACC
:1005A00003FC20FA02F001FA03FE40EA0E0021FAF1
:1005B00002F11444BDE600BF70B54FF0FF0C4CF4DF
:1005C000E06C1CEA11541DBF1CEA135594EA0C0F91
:1005D00095EA0C0F00F0DEF82C4481EA030621EACC
:1005E0004C5123EA4C5350EA013518BF52EA033507
:1005F00041F4801143F4801338D0A0FB02CE4FF0B9
:100600000005E1FB02E506F00042E0FB03E54FF0E8
:100610000006E1FB03569CF0000F18BF4EF0010EE0
:10062000A4F1FF04B6F5007F64F5407404D25FEADC
:100630004E0E6D4146EB060642EAC62141EA55518F
:100640004FEAC52040EA5E504FEACE2EB4F1FD0CD1
:1006500088BFBCF5E06F1ED8BEF1004F08BF5FEA4F
:10066000500E50F1000041EB045170BD06F0004601
:1006700046EA010140EA020081EA0301B4EB5C04AE
:10068000C2BFD4EB0C0541EA045170BD41F48011A6
:100690004FF0000E013C00F3AB8014F1360FDEBFCB
:1006A000002001F0004170BDC4F10004203C35DAA7
:1006B0000C341BDC04F11404C4F1200500FA05F32A
:1006C00020FA04F001FA05F240EA020001F00042CB
:1006D00021F0004110EBD37021FA04F642EB060141
:1006E0005EEA430E08BF20EAD37070BDC4F10C046B
:1006F000C4F1200500FA04F320FA05F001FA04F22F
:1007000040EA020001F0004110EBD37041F100011A
:100710005EEA430E08BF20EAD37070BDC4F1200525
:1007200000FA05F24EEA020E20FA04F301FA05F28D
:1007300043EA020321FA04F001F0004121FA04F235
:1007400020EA020000EBD3705EEA430E08BF20EA05
:10075000D37070BD94F0000F0FD101F0004640003F
:1007600041EB010111F4801F08BF013CF7D041EAC1
:10077000060195F0000F18BF704703F000465200C5
:1007800043EB030313F4801F08BF013DF7D043EA96
:100790000603704794EA0C0F0CEA135518BF95EA4C
:1007A0000C0F0CD050EA410618BF52EA4306D1D1D3
:1007B00081EA030101F000414FF0000070BD50EAF2
:1007C000410606BF1046194652EA430619D094EA7C
:1007D0000C0F02D150EA013613D195EA0C0F05D166
:1007E00052EA03361CBF104619460AD181EA0301BA
:1007F00001F0004141F0FE4141F470014FF0000072
:1008000070BD41F0FE4141F4780170BD70B54FF00C
:10081000FF0C4CF4E06C1CEA11541DBF1CEA13558C
:1008200094EA0C0F95EA0C0F00F0A7F8A4EB05046E
:1008300081EA030E52EA03354FEA013100F0888065
:100840004FEA03334FF0805545EA131343EA12632E
:100850004FEA022245EA111545EA10654FEA0026E3
:100860000EF000419D4208BF964244F1FD0404F59C
:10087000407402D25B084FEA3202B61A65EB0305F8
:100880005B084FEA32024FF480104FF4002CB6EBB5
:10089000020E75EB030E22BFB61A754640EA0C0035
:1008A0005B084FEA3202B6EB020E75EB030E22BF75
:1008B000B61A754640EA5C005B084FEA3202B6EBB6
:1008C000020E75EB030E22BFB61A754640EA9C0075
:1008D0005B084FEA3202B6EB020E75EB030E22BF45
:1008E000B61A754640EADC0055EA060E18D04FEA03
:1008F000051545EA16754FEA06164FEAC30343EAA3
:1009000052734FEAC2025FEA1C1CC0D111F4801F6F
:100910000BD141EA00014FF000004FF0004CB6E768
:1009200011F4801F04BF01430020B4F1FD0C88BF07
:10093000BCF5E06F3FF6AFAEB5EB030C04BFB6EB12
:10094000020C5FEA500C50F1000041EB045170BD05
:100950000EF0004E4EEA113114EB5C04C2BFD4EB32
:100960000C0541EA045170BD41F480114FF0000EB6
:10097000013C90E645EA060E8DE60CEA135594EA32
:100980000C0F08BF95EA0C0F3FF43BAF94EA0C0F35
:100990000AD150EA01347FF434AF95EA0C0F7FF4AA
:1009A00025AF104619462CE795EA0C0F06D152EAFE
:1009B00003353FF4FDAE1046194622E750EA4106E2
:1009C00018BF52EA43067FF4C5AE50EA41047FF4F3
:1009D0000DAF52EA43057FF4EBAE12E74FF0FF3C58
:1009E00006E000BF4FF0010C02E000BF4FF0010C29
:1009F0004DF804CD4FEA410C7FEA6C5C4FEA430CA2
:100A000018BF7FEA6C5C1BD001B050EA410C0CBFF0
:100A100052EA430C91EA030F02BF90EA020F002052
:100A2000704710F1000F91EA030F58BF994208BFB9
:100A300090422CBFD8176FEAE37040F00100704776
:100A40004FEA410C7FEA6C5C02D150EA013C07D1CD
:100A50004FEA430C7FEA6C5CD6D152EA033CD3D018
:100A60005DF8040B704700BF8446104662468C4612
:100A70001946634600E000BF01B5FFF7B7FF002845
:100A800048BF10F1000F01BD4DF808EDFFF7F4FF6E
:100A90000CBF012000205DF808FB00BF4DF808EDF9
:100AA000FFF7EAFF34BF012000205DF808FB00BF1C
:100AB0004DF808EDFFF7E0FF94BF012000205DF83E
:100AC00008FB00BF4DF808EDFFF7CEFF94BF0120F3
:100AD00000205DF808FB00BF4DF808EDFFF7C4FFEC
:100AE00034BF012000205DF808FB00BF4FEA410C35
:100AF0007FEA6C5C02D150EA013C0AD14FEA430C18
:100B00007FEA6C5C02D152EA033C02D14FF0000054
:100B100070474FF0010070474FEA410212F5001292
:100B200015D211D56FF47873B3EB625212D94FEA34
:100B3000C12343F0004343EA505311F0004F23FA1E
:100B400002F018BF404270474FF00000704750EA73
:100B5000013005D111F0004008BF6FF00040704730
:100B60004FF00000704700BF4A0011D212F500128A
:100B700011D20DD56FF47873B3EB62520ED44FEAF5
:100B8000C12343F0004343EA505323FA02F0704775
:100B90004FF00000704750EA013002D14FF0FF30B3
:100BA00070474FF0000070474FEA4102B2F1E04356
:100BB00024BFB3F5001CDCF1FE5C0DD901F0004C44
:100BC0004FEAC0024CEA5070B2F1004F40EB830094
:100BD00008BF20F00100704711F0804F21D113F1C0
:100BE0003872BCBF01F00040704741F480114FEAF9
:100BF0005252C2F11802C2F1200C10FA0CF320FA82
:100C000002F018BF40F001004FEAC1234FEAD3239E
:100C100003FA0CFC40EA0C0023FA02F34FEA430308
:100C2000CCE77FEA625307D150EA01331EBF4FF091
:100C3000FE4040F44000704701F0004040F0FE40AC
:100C400040F40000704700BF80F0004002E000BFA9
:100C500081F0004142001FBF5FEA410392EA030FA7
:100C60007FEA226C7FEA236C6AD04FEA1262D2EBF1
:100C70001363C1BFD218414048404140B8BF5B42F6
:100C8000192B88BF704710F0004F40F4000020F08F
:100C90007F4018BF404211F0004F41F4000121F0A5
:100CA0007F4118BF494292EA030F3FD0A2F10102EF
:100CB00041FA03FC10EB0C00C3F1200301FA03F12D
:100CC00000F0004302D5494260EB4000B0F5000F50
:100CD00013D3B0F1807F06D340084FEA310102F10F
:100CE0000102FE2A51D2B1F1004F40EBC25008BFC1
:100CF00020F0010040EA03007047490040EB00008B
:100D0000013A28BFB0F5000FEDD2B0FA80FCACF18B
:100D1000080CB2EB0C0200FA0CF0AABF00EBC250B8
:100D200052421843BCBFD0401843704792F0000FA6
:100D300081F4000106BF80F400000132013BB5E7F9
:100D40004FEA41037FEA226C18BF7FEA236C21D06F
:100D500092EA030F04D092F0000F08BF08467047D4
:100D600090EA010F1CBF0020704712F07F4F04D1A2
:100D7000400028BF40F00040704712F100723CBFB5
:100D800000F50000704700F0004343F0FE4040F4DF
:100D9000000070477FEA226216BF08467FEA23639D
:100DA0000146420206BF5FEA412390EA010F40F488
:100DB000800070474FF0000304E000BF10F00043D4
:100DC00048BF40425FEA000C08BF704743F09643BB
:100DD00001464FF000001CE050EA010208BF7047D6
:100DE0004FF000030AE000BF50EA010208BF70475D
:100DF00011F0004302D5404261EB41015FEA010C72
:100E000002BF84460146002043F0B64308BFA3F169
:100E10008053A3F50003BCFA8CF2083AA3EBC2534B
:100E200010DB01FA02FC634400FA02FCC2F120026A
:100E3000BCF1004F20FA02F243EB020008BF20F0A1
:100E40000100704702F1200201FA02FCC2F1200207
:100E500050EA4C0021FA02F243EB020008BF20EAFC
:100E6000DC7070477BB972B90029BEBF00204FF01B
:100E7000004106E008BF00281CBF6FF000414FF0A2
:100E8000FF3000F015BAADF1080C6DE904CE002971
:100E900009DB002B1ADB00F0A3F8DDF804E0DDE944
:100EA000022304B07047404261EB4101002B1BDB81
:100EB00000F096F8DDF804E0DDE9022304B04042DA
:100EC00061EB4101524263EB43037047524263EBD3
:100ED000430300F085F8DDF804E0DDE9022304B007
:100EE000404261EB41017047524263EB430300F023
:100EF00077F8DDF804E0DDE9022304B0524263EB49
:100F00004303704753B94AB9002908BF00281CBFE2
:100F10004FF0FF314FF0FF3000F0CAB9ADF1080CCF
:100F20006DE904CE00F05CF8DDF804E0DDE90223B1
:100F300004B0704730B1012390FAA0F0B0FA80F00D
:100F40001844704708460029FBD02123F4E700BF6E
:100F5000430803F05533C01A830803F0333300F01D
:100F60003330184400EB101000F00F3000EB00207D
:100F700000EB0040000E704707EE900AF5EEC07AD5
:100F8000F1EE10FA01D400F00BB8F1EE677A08B573
:100F900017EE900A00F004F8404261EB410108BDF1
:100FA000D0B5FFF7B1FA0C4B002206460F46FFF70B
:100FB00003FBFFF7D9FD0446FFF784FA074B002235
:100FC000FFF7FAFA02460B4630463946FFF73CF97E
:100FD000FFF7CAFD2146D0BD0000F03D0000F04102
:100FE0002DE9F047089D04468E46002B4DD18A42DC
:100FF000944669D9B2FA82F252B101FA02F3C2F10F
:10100000200120FA01F10CFA02FC41EA030E94409F
:101010004FEA1C48210CBEFBF8F61FFA8CF708FBC0
:1010200016E341EA034306FB07F199420AD91CEB98
:10103000030306F1FF3080F01F81994240F21C81CA
:10104000023E63445B1AA4B2B3FBF8F008FB103312
:1010500044EA034400FB07F7A7420AD91CEB040447
:1010600000F1FF3380F00A81A74240F20781644417
:10107000023840EA0640E41B00261DB1D44000239C
:10108000C5E900433146BDE8F0878B4209D9002D00
:1010900000F0EF800026C5E9000130463146BDE88A
:1010A000F087B3FA83F6002E4AD18B4202D38242F4
:1010B00000F2F980841A61EB030301209E46002DA3
:1010C000E0D0C5E9004EDDE702B9FFDEB2FA82F2F8
:1010D000002A40F09280A1EB0C014FEA1C471FFA56
:1010E0008CFE0126200CB1FBF7F307FB131140EA3D
:1010F00001410EFB03F0884208D91CEB010103F10A
:10110000FF3802D2884200F2CB804346091AA4B2CB
:10111000B1FBF7F007FB101144EA01440EFB00FE9F
:10112000A64508D91CEB040400F1FF3102D2A64504
:1011300000F2BB800846A4EB0E0440EA03409CE7A3
:10114000C6F12007B34022FA07FC4CEA030C20FA50
:1011500007F401FA06F31C43F9404FEA1C4900FA70
:1011600006F3B1FBF9F8200C1FFA8CFE09FB1811ED
:1011700040EA014108FB0EF0884202FA06F20BD960
:101180001CEB010108F1FF3A80F08880884240F2B0
:101190008580A8F102086144091AA4B2B1FBF9F0F4
:1011A00009FB101144EA014100FB0EFE8E4508D9EF
:1011B0001CEB010100F1FF346CD28E456AD9023874
:1011C000614440EA0840A0FB0294A1EB0E01A14259
:1011D000C846A64656D353D05DB1B3EB080261EBC7
:1011E0000E0101FA07F722FA06F3F1401F43C5E9A1
:1011F000007100263146BDE8F087C2F12003D840D7
:101200000CFA02FC21FA03F3914001434FEA1C4718
:101210001FFA8CFEB3FBF7F007FB10360B0C43EA0A
:10122000064300FB0EF69E4204FA02F408D91CEBBA
:10123000030300F1FF382FD29E422DD902386344B8
:101240009B1B89B2B3FBF7F607FB163341EA034158
:1012500006FB0EF38B4208D91CEB010106F1FF38A7
:1012600016D28B4214D9023E6144C91A46EA00469E
:1012700038E72E46284605E70646E3E61846F8E630
:101280004B45A9D2B9EB020864EB0C0E0138A3E779
:101290004646EAE7204694E74046D1E7D0467BE75A
:1012A000023B614432E7304609E76444023842E7D2
:1012B000704700BF02E000F000F8FEE772B6374862
:1012C00080F30888364880F3098836483649086034
:1012D00040F20000CCF200004EF63471CEF2000174
:1012E0000860BFF34F8FBFF36F8F40F20000C0F272
:1012F000F0004EF68851CEF200010860BFF34F8F28
:10130000BFF36F8F4FF00000E1EE100A4EF63C7114
:10131000CEF200010860062080F31488BFF36F8FBF
:10132000B3F07AFAB4F0C4F94FF055301F491B4AB4
:1013300091423CBF41F8040BFAE71D49184A91421B
:101340003CBF41F8040BFAE71A491B4A1B4B9A426F
:101350003EBF51F8040B42F8040BF8E7002018498F
:10136000184A91423CBF41F8040BFAE7B3F058FA2F
:10137000B4F0F2F9144C154DAC4203DA54F8041BE6
:101380008847F9E702F0E0F8114C124DAC4203DA5D
:1013900054F8041B8847F9E7B3F040BA0006002070
:1013A000002200200000010808ED00E000000020FD
:1013B00000060020D80D0F0800220020742C002009
:1013C000782C002030460120E0010108400201088D
:1013D00040020108400201082DE9F04F2DED108A6E
:1013E000C1F80CD0C3689D46BDEC108ABDE8F08FF3
:1013F000002383F311882846A0470020B2F090F91B
:10140000FEE7B1F0EDFF00DFFEE7000001F0FF01B5
:10141000102A2BDB10F0070F08D010F8013B013A1F
:101420008B422DD010F0070F42B3F6D1F0B441EA51
:10143000012141EA014122F007047FF00007002367
:10144000F0E80256083C85EA010586EA010685FABD
:1014500047F5A3FA87F586FA47F6A5FA87F68EB917
:10146000EED1F0BC01F0FF0102F0070232B110F83A
:10147000013B013A83EA010313B1F8D10020704720
:1014800001387047002D06BF35460338073815F080
:10149000010F07D1013015F4807F02BF013015F430
:1014A000C03F0130F0BC0138704700BF10F8012B7D
:1014B00011F8013B012A28BF9A42F7D0D01A704791
:1014C000034613F8012B002AFBD1181A0138704784
:1014D00038B50022002304460D46FFF7DFFA28B98D
:1014E00020462946BDE8384000F00AB8204605F1FC
:1014F000004100F005F8404261EB410138BD00BFFA
:10150000D0B50C4B002206460F46FFF755F8FFF703
:101510002BFB0446FEF7D6FF074B0022FFF74CF8E3
:1015200002460B4630463946FEF78EFEFFF71CFB9F
:101530002146D0BD0000F03D0000F04103680022CC
:101540001B6818477FB503914021054680F006FAD5
:10155000039A18B90124204604B070BD134E0392BB
:1015600096F9E632002BF5D061F0C6F9437A039A7A
:1015700053B961F0C1F9847A039A2CB90C4B40211C
:10158000284680F0F3F9E6E7D6F8DC3CB6F9E81235
:10159000B3F906309942DDDD064B00934021064B3E
:1015A000284680F0E3F90024D5E700BF804C0020F6
:1015B000B0CD0C08CFCD0C08BDCD0C08F0B50D4654
:1015C0009DB02021044680F0C9F9002800F09D80DC
:1015D0004F4E96F9E632ABB1D6F8DC2CB6F9E832CC
:1015E000B2F90A1003F10A02914203DD40F28D3292
:1015F000934207DC474B2A462021204680F0B6F96B
:10160000002080E096F9D532022B05D1424B2A46C4
:101610002021204680F0AAF9B6F8A832A3F57A7303
:101620009BB241F6583293420DD83C4F96EDC57AA5
:10163000D7F81C3DD3ED097AB4EEE77AF1EE10FA53
:1016400003DD374BD7E7374BD5E796EDC67AD3EDB9
:101650000B7AB4EEE77AF1EE10FAF2DCB6F9E23288
:10166000002B01DC304BC6E796F874230D2A06D810
:101670000123934013F4215F01D02C4BBBE72C488E
:1016800010F0CCF9012806D1D7F8280D87F0BCF965
:1016900098B101281AD00021602204A80391B7F064
:1016A00071F82449D7F8240D642303AA86F0CEFDEF
:1016B00000BB03AB0093204B02E0204B0093204B78
:1016C0002A462021204680F051F999E796F8F03C0F
:1016D00073B11C48192150F01BFA48B11948D6F8CB
:1016E000C062192150F03AFA8642D4DD164BE5E784
:1016F000164BE3E71649D7F81C0D642303AA83F0C1
:1017000065FC0028D5D01DB0F0BD0120FBE700BF6F
:10171000804C0020D8CD0C08EBCD0C08806C00204C
:1017200023CE0C0813CE0C083DCE0C0852CE0C086C
:1017300058820020CCCE0C08D0CE0C0897CE0C08D6
:1017400072CE0C08C0390020B6CE0C08A7CE0C080B
:10175000E2CE0C0807B5044888F0AEFC00F00100AA
:1017600003B05DF804FB00BF807900202DE9F04351
:10177000DFF844910446D9F8EC000368A5B01B6972
:101780000D469847804615F067FC00210746602209
:101790000CA80B91B6F0F6FF64230BAA414638461D
:1017A00014F04EFF064648B93A4A0BAB294620468C
:1017B00080F0FEFA304625B0BDE8F083A9F56B60F5
:1017C0006EF0A2FBB8F1000F03D194F91E30012B8B
:1017D0000AD1314812F02CFC80B9304A2946204603
:1017E00080F0E6FA0026E5E710F0060FE2D0A9F552
:1017F000405012F01DFC08B9294AEFE703A938460A
:1018000014F050FD28B19DF80D305B0601D5254A36
:10181000E4E7DFF8A880D8EDC17AF5EEC07AF1EE02
:1018200010FA4FF00003C5DD089309930A930DF1F8
:10183000200907AB019305AA06AB04A9CDF80090D7
:10184000384615F011F9484630F010FDD8EDC17A50
:10185000B4EEE70AF1EE10FA01DB134ABEE79DEDA4
:10186000057AF4EEC77AF1EE10FA01D80F4AB5E71F
:101870009DED047AF4EEC77AF1EE10FA01D80C4A25
:10188000ACE79DED067AF4EEC77AF1EE10FA91D846
:10189000084AA3E7E8CE0C08802C0020F1CE0C0803
:1018A00008CF0C082ECF0C083CCF0C0851CF0C08E9
:1018B00067CF0C087DCF0C08805C0020804C002096
:1018C00008B5064B93F805319B0704D5044A80F010
:1018D0006FFA002008BD0120FCE700BF805C0020FB
:1018E00094CF0C0870B50C4C0546D4F8EC00036896
:1018F0005B690E46984710B10124204670BDA4F5DF
:10190000405012F0A7FB04460028F5D1034A3146A7
:10191000284680F04DFAF0E7805C0020A4CF0C0848
:101920002DE9F046464ED6F8103193F8CB509BB0D7
:1019300081468A4665B9434B1B68986A03685B6BAE
:101940009847044640B9404A5146484680F030FA2C
:1019500028461BB0BDE8F08660F0CEFF202162F083
:1019600041F858B160F0C8FF1F2162F03BF888B31E
:10197000364A5146484680F01BFA002496F8E23079
:1019800003F01403142B05D1314A5146484680F028
:101990000FFA00245146484681F0D8F800218842C9
:1019A0004FF0600202A808BF0C460191B6F0EAFEB3
:1019B000D6F81001036801AA1B6864219847054600
:1019C00080B9244A01AB5146484680F0F1F92C46D3
:1019D0002546BDE760F090FFA52162F003F80028DE
:1019E000C6D1CBE7002CF3D0D9F808303BB9D9F8F1
:1019F000003051465B6B484698470446E8E751463D
:101A00004846FFF7DBFD514607464846FFF758FFBB
:101A10003840C4B251464846FFF794FD5146044051
:101A20004846FFF75FFF51460440484680F0E8F91A
:101A300051460440484681F0A1F80440C8E700BF81
:101A4000805C0020E0840020B8CF0C08CFCF0C08C9
:101A5000E9CF0C0801D00C0808B5FFF761FF054A73
:101A600092F8E01060F3041182F8E010024A9071DD
:101A700008BD00BF805C0020BD860020F7B505468C
:101A80000F467FF0A7FF044678B1022128467FF079
:101A900065FF064648B1154888F00EFBC205C0F345
:101AA0000723C0F3002403D53446204603B0F0BD1D
:101AB0009B07F9D50D4888F00DFB0D4B03F6CC4381
:101AC000D3ED007AF8EEE77A30EE670ADFED097AB7
:101AD000B0EEC00AB4EEE70AF1EE10FAE4DD064B10
:101AE0003A46022128467FF041FFDEE78079002058
:101AF000806C00200000C8420CD00C08F8B50446E9
:101B00000F4680F01DFA1021054620467FF026FF83
:101B100058B12046FFF71EFE064630B9044B3A4640
:101B2000102120467FF022FF35462846F8BD00BF31
:101B300020D00C0870B505460E467FF0B3FE044673
:101B400078B1802128467FF009FF50B1074B93F808
:101B5000AD3643B1064B3246802128467FF006FF62
:101B60000024204670BD0446FBE700BF805C0020D7
:101B700034D00C0838B50D4D0446D5F8280D86F044
:101B800043FF012810D0D5F8280D86F03DFF02282C
:101B900004D02046BDE838407FF086BE04480FF0F0
:101BA0003DFF0128F5D138BD0020FCE7806C002006
:101BB00058820020F0B5134C04F5005385B0D3F8DB
:101BC000D42C0092D3F8D82C0192D3F8DC2C0292BA
:101BD000D3F8E03C03936A4606460F4680F068FF60
:101BE0003946054630467FF01BFF04F54054284037
:101BF00094F8E03060F3C303C3F3C00084F8E0302E
:101C000005B0F0BD802C00202DE9F843064627489A
:101C1000DFF8A890DFF8A8800F466EF075F904464B
:101C2000D9F8EC0003681B699847054630B914F0F1
:101C3000060F03D1D9F82031022B09D1394630469D
:101C40007FF0DAFF054618B9002488F807400AE05B
:101C500039463046FFF78AFD04460028F4D02DB9F6
:101C6000012388F807302046BDE8F8830821304674
:101C70007FF074FE0028F3D00D4823F0ABFB002862
:101C8000EED00C4B93F81424B02101FB023203F583
:101C90000053B2F81E22B3F9D6329A42E0DD064B69
:101CA0003A46082130467FF061FECDE7D04D002056
:101CB000A02D0020802C002048D00C08805C002043
:101CC000BD8600202DE9F3410E46054615F0C4F906
:101CD000804614F0A9FA044640B9514A0121284629
:101CE00080F066F8204602B0BDE8F0814D4FD7F88D
:101CF000EC00036831469B699847044658B9D7F809
:101D0000EC0003681B6C9847474A034601212846AC
:101D100080F04EF8E6E7AB68002BE3D010212846B0
:101D20007FF01CFE20B3D8ED937A98ED920A20EE56
:101D3000270AB4F0C9FADFED3D7AA7F5805320EE0B
:101D4000270AB3F9A832DFED3A7A20EE270A07EE28
:101D5000903AF8EEE77AB4EEE70AF1EE10FA07DD12
:101D6000344B0122102128467FF000FE0024B9E701
:101D7000402128467FF0F2FD38B3012E1ED0232EDD
:101D80001CD0042E1AD02C4CD4F8DC3CB3F908300B
:101D900000EE103AA4F50050B8EEC00A00F0BCFB0B
:101DA000B5EEC00AF1EE10FA1DDD244B00930122BE
:101DB000234B402128467FF0D9FDD7E7D7F8EC0028
:101DC0000368DB6B98470028DDD01E4B1B68D86A80
:101DD0000368DB6998470128014619D11A4A284649
:101DE0007FF0E6FFC2E7D7F8EC0003685B6998472D
:101DF00030B1D4F8DC3CB3F90830002BE5DDD4E792
:101E0000D7F8EC0003681B6898470B28DDD1F0E792
:101E10003146284602B0BDE8F04180F059BB00BF12
:101E200058D00C08805C002069D00C08E02E654278
:101E30000000C8427DD00C08804C0020CFCD0C089B
:101E400085D00C08E084002091D00C0870B50546C0
:101E50000E46FFF78BFC084B0446D87131462846E6
:101E6000FFF740FD31460028284608BF002480F0D7
:101E700007FD204070BD00BFBD8600202DE9F04168
:101E80004E4F3B78002B40F096804D4CD4F81051CB
:101E900095F8CB5001263E701DB13B702846BDE839
:101EA000F08180F019FF054630B9464A3870137842
:101EB00043F001031370F1E756F046F8314655F050
:101EC0007DF9A4F5405006F047FD3F4B1E710B26EF
:101ED0004AF0F0FE013E4AF0BBFE16F0FF06F7D1D5
:101EE0003A4800F083FF15F0B7F8D0F80022C4F8A4
:101EF000382190F87C32DA074DD414F017FC56F0F4
:101F000023F83C2155F05CFF0023C4F8F830002191
:101F10002E482F4E00F0F0FF2C4812F089F80146B1
:101F20002C488CF03BF82C4B1B68D86A03680121C5
:101F30001B689847D4F8100103689B6A98470121F1
:101F4000D4F8100189F072F855F0FEFF8046D4F8FD
:101F5000EC0003681B68984796F8682201464046E3
:101F600055F004FBA6F5005006F0E8FC53F0E6F946
:101F700052F022FD00233B7090F0E4FFB4F8E23011
:101F800006F5005623F4087343F02003C6F8340D19
:101F9000A4F8E23082E79B07B9D431460B4804F03D
:101FA0005FFD0E4888F096F8DFED0D7A20EE270AE7
:101FB00084ED3E0AABE7002570E700BF782C0020D7
:101FC000805C0020DC860020BD860020802C002064
:101FD000804C00205C570020E084002080790020A5
:101FE0000AD7233C2DE9F043374DD5F8103193F84B
:101FF000CB3087B0002B64D062B1012901D02329F6
:1020000008D195F9E030002B04DB0024204607B00E
:10201000BDE8F08380F00CFF04460028F5D015F0F1
:102020001BF807461BF0F0FF8046384613F006FE0B
:10203000D8B198F92430022B17D100264FF00009AF
:10204000F1B203AA38460191CDF80C90CDF810906A
:10205000CDF8149014F090F9019918B103AA4046F4
:102060001BF082FC0136032EEAD11848012106F04C
:10207000DFFE1648012106F00FFE0021D5F8100101
:1020800088F0D4FF124832F015FE55F05DFF0021B4
:1020900055F094F80F4B1B68D86A036800211B6841
:1020A000984795F8E230D5F8EC100B486FF34513DC
:1020B00085F8E2300B1A594259413C308FF054F9FF
:1020C000A4E70124A2E700BF805C0020802C002050
:1020D000447C0020E0840020E07D002010B5064C08
:1020E000D4F8EC0003685B6A984718B1D4F8103153
:1020F00093F8CB0010BD00BF805C002030B52DED03
:10210000028B89B00C46B0EE408AFFF7E7FF054628
:10211000002838D0B4EE488AF1EE10FA7CBFDFED2B
:102120001C8ADFED1C7A226863689FED1A0A68BF7B
:10213000DFED198A029278BF68EE288A02A878BF7C
:1021400068EEA78AD4ED027A0393F1EE677ACDEDBB
:10215000047A2FF08DFCB4EE488A00220123F1EEC0
:1021600010FACDE900238DED050ACDED060A9FEDAD
:102170000A0A0A488DED071AF0EE680A68BF13468E
:1021800005A90DF029FD284609B0BDEC028B30BD34
:10219000E02E65420000C84200000000FC800020E4
:1021A00007B50191FFF79AFF30B10199044803B0D8
:1021B0005DF804EB00F0F6BA03B05DF804FB00BF75
:1021C000802C002001486EF02BB800BFD04D0020BD
:1021D00008B500F5405090F8E030C3F340128A4251
:1021E0000BD061F3451380F8E03031B155F0ACFE0F
:1021F000BDE808400F2155F0E3BD08BD70B500F5FE
:1022000040560546D6F820318B420C4612D00129A3
:1022100011D0022916D059B955F096FE1B2155F060
:10222000CFFD0D4A05F53A500621383057F088FFAA
:10223000C6F8204170BD55F087FE1A2155F0C0FD4B
:10224000064AEFE7012100F057FE55F07DFE1D2103
:1022500055F0B6FD024AE5E7FCD00C0811D10C0898
:102260000CD10C0810B500F540520C4692F805311F
:1022700003F00101A14209D064F3000382F80531A3
:10228000DB0704D405F038FF024B9C7210BD06F04A
:1022900019F9F9E7BD86002000F5405090F80531A6
:1022A00061F3410380F80531014B1973704700BF9A
:1022B000BD86002010B5044660F01EFB202161F0B1
:1022C00091FB04F54053003893F8E22018BF012039
:1022D00060F3820283F8E22010BD000010B50446CE
:1022E00053F02CF804F54052436FD2F8102104F556
:1022F0008044D360D4F81C2D9366D4F8242DC2F802
:10230000FC32D4F81C0D03685B6D9847D4F81C0DA3
:102310000368BDE810409B6D1847000070B52DEDB7
:10232000028B00F540550446D5F8103193F8CB30B8
:10233000002B71D095F9E030002B6DDB00F5804665
:1023400096F8E83E002B67D1D5F8EC0003685B698E
:102350009847002860D1324BD3F8EC0003681B6823
:1023600098470B2858D0D6F8243D9FED2E7AD3ED10
:10237000DB7AF0EEE77AF4EEC77AF1EE10FA4BD59D
:10238000D5F81001443057F011FA0346DFED260A64
:1023900093ED000A9F20B7EE001A2CF035F9B5EE48
:1023A000C00AF1EE10FA37DD04F59A4087F09EFE80
:1023B000DFED1E7AB0EEC00AB4EEE70AF1EE10FAD5
:1023C0002AD504F58054D6F81C0DD4F8A83407EEAD
:1023D000903A0368D3F89830B8EEE78A984738EE19
:1023E000400ADFED137AB0EEC00AB4EEE70AF1EE70
:1023F00010FA11D5D4F8AC3440F2E63203F2F313FC
:10240000934209D8BDEC028BD5F810019FED090A63
:10241000BDE870408AF08CB8BDEC028B70BD00BF87
:10242000805C0020000000340000000000007042CA
:102430000000FA430AD7233C08B500F54050D0F815
:10244000100103681B699847F6EE007A20EE270A10
:10245000B5EEC00AF1EE10FA48BF9FED010A08BDC3
:102460000000000038B52DED028B00F580450446D4
:10247000D5F81C3DDFED110A93ED370A04F5405401
:102480007120B7EE001A2CF0BFF8D4F81001D5F87F
:10249000245D03681B69B0EE408A984738EE400A15
:1024A000BDEC028BDFED067A05F50575284620EEBA
:1024B000270ABDE8384078F00DBB00BF00000000DF
:1024C00000007A4400F5A853D3ED005AD2ED007A0B
:1024D000D3ED036A91ED006A26EEE77A67EEA57AFE
:1024E000A6EE257AE6EE267A81ED007AC2ED007A34
:1024F0007047000000F50050B0F98C3B33B9B0F9DB
:10250000E2020028B8BF404280B2704783EAE3701D
:10251000A0EBE370F8E7000070B52DED028B00F53D
:10252000405382B093F8051111F00106044605D01E
:102530009FED2E0A02B0BDEC028B70BD8DED010A3D
:1025400060F0DAF9037F002BF2D0DFED298ADFEDAE
:10255000270A9DED010AB0EE681A4E202CF054F8BF
:1025600004F500554FF4C8723146B5F9EA02B0EEF1
:10257000408A2CF087F8A5F8EA02204611F006FB05
:10258000B5F9EA3207EE900AB8EEE77A07EE903A2C
:10259000F8EEE77A77EE676AB4EEE68AF1EE10FAC3
:1025A0000DD52046FFF7A6FF07EE900A38EE668AA3
:1025B000B8EEE70A20EE088A88EE260ABAE777EE38
:1025C000877AB4EEE78AF1EE10FAB1DDB5F9E232BE
:1025D00000EE103A38EE678AB8EEC00A78EEE77A75
:1025E00020EE088A88EE270AA4E700BF000000005A
:1025F00000007A44002070470020704770470000B8
:1026000000F50B503830704700487047F8000D084F
:1026100000F54050D0F8EC0003681B681847000034
:10262000034808603221117008221A60704700BF09
:10263000B8D40C0800F54050D0F8EC000368DB6C0F
:102640001847000000F54050D0F8EC0003689B6C80
:102650001847000000F5405300F59F40D3F8EC30D8
:1026600008301B1A584258417047000010B500F559
:1026700040500C46D0F8EC000368DB6D984707EE3D
:10268000900A9FED057AF8EE677A012067EE877A67
:10269000C4ED007A10BD00BF0AD7233C10B500F589
:1026A00040500C46D0F8EC0003689B6D984707EE4D
:1026B000900A9FED057AF8EEE77A012067EE877AB7
:1026C000C4ED007A10BD00BF0AD7233C10B500F559
:1026D00040500C46D0F8EC0003681B6E9847DFEDC5
:1026E000047A20EE270A012084ED000A10BD00BF05
:1026F0000AD7233C66F030BF6AF078BB62F0A8BB13
:1027000052F066BD29F0BABE54F0D6BE18F0F4BA45
:1027100062F01EBF5FF04ABD5DF054BE10F0CEBE49
:1027200011F028BB06F0B8BD12F040BB05F038BD73
:1027300005F084BA05F0AAB968F08EBC10F00CB8A8
:10274000FFF7ECBD10F0FEBF11F06CBA03F03EB91C
:1027500010F082BF10F0FABE60F01CB84BF004BD60
:1027600024F0E6B806F064B902F0F8BC62F000BFED
:1027700011F076BA06F048BD04F05EB906F0A0BECE
:1027800005F016BA06F004BA10F024BEFFF7A6BD95
:102790002AF092B905F014BF0AF072BA0AF05CB9D7
:1027A0000AF0F0B81FB500F540530446D3F8EC002A
:1027B000039103685B6A984760B1DFED070A0399EC
:1027C000002304F5A8400093B0EE600A1A467C305E
:1027D0000DF058F804B010BD0000000010B52DED4C
:1027E000028B00F540530446D3F8EC0003685B6AA3
:1027F000B0EE408A984720B90024BDEC028B2046F9
:1028000010BD9FED080A04F5A84028EE000A7C30B0
:102810000CF002FB04460028EED003480121FFF72C
:10282000D7FCEAE70000C842802C00200A4A92F94F
:10283000E020002A0B4605DA00228A604A600A601E
:102840000120704700F58040D0F81C2D783207CA6F
:1028500083E80700F4E700BF805C002070B5204BE0
:10286000036000F500531F4AC3F8B82E00F540532B
:102870000446586F08B11AF0FFFD1B4B236004F5A6
:10288000805393F8342F42B9D3F8305F2DB12846E6
:1028900028F0FCFB28461AF0EBFD04F58D501C30A7
:1028A0007EF0A6FA04F58650043062F005FD04F6C9
:1028B000F44504F69446B54204D0183D284628F065
:1028C0003BF8F8E7094BC4F8C83804F6C41056F0D2
:1028D00049FC04F5136056F045FC204670BD00BF6E
:1028E000B0D80C0898E20D083CC30D08E08D0D0827
:1028F00038B54B4B044640F8043B66F04DFF04F1FD
:10290000100017F095FE04F1680052F0EFF904F59D
:10291000907022F06FFC04F58C6016F029FC04F234
:1029200084501AF0ABFD04F6C80029F04BFC04F506
:10293000476066F00FFD04F554604FF00FF804F5A2
:102940007F6054F09BFB04F5855008306CF0BEFDB1
:1029500004F58650043062F097FC04F5885019F0B5
:10296000AFFB04F58D501C307EF02EFA04F58E502E
:10297000183052F07DFD04F591500C3068F0B6F837
:1029800004F580530025274A83F8505204F59253EA
:10299000103304F59350136049F0C8FF04F59550C7
:1029A0002946103012F03AFE04F5C85078F0D0FAFB
:1029B00004F5EE5004307BF039FA04F5F6501C3083
:1029C0007DF05CFB04F5FA507DF092FF04F5FC50BD
:1029D000183012F025FC04F50350383078F0F4FF7D
:1029E00004F5055010306DF033F904F5085010303F
:1029F0007EF086FD04F5005304F50A5083F8685212
:102A0000094D7EF09FFE2B6813B1084890F068FADC
:102A1000204607494DF068FE2C60204638BD00BFB7
:102A20003CC30D089C900020A487002020D10C08F6
:102A300044C20D0810B511F01DF85FF05DFF03688A
:102A4000BDE810405B681847FFF7F4BF10B50446B7
:102A500006F03AF9204611F013FB204603F03CFE45
:102A60002046BDE8104003F09DBF0000FFF7EEBF19
:102A700070B500F544553C350446284617F0B2FCC5
:102A80001BF0C2FA90F9213093B390F840337BB336
:102A900004F5405304F28456D3F81001443056F044
:102AA00085FE0346DFED130A93ED000A9F20B7EE83
:102AB000001A2BF0A9FD94F9B835012B284608BF60
:102AC00086ED0E0A002117F021FADFED0B7A04F2F1
:102AD000DC7494ED287A20EE270ADFED087AA7EE61
:102AE000270A304684ED280ABDE870401BF09CB9E7
:102AF00070BD00BF00000000CDCCCC3D6666663FD7
:102B0000FFF7B6BF10B50121044611F0F5FA60B128
:102B1000114BD3F8EC0003689B6A984728B920460C
:102B200002F02AFA204602F037FA4FF4001120464C
:102B300011F0E2FA18B12BF039F829F01FFA4FF42E
:102B40008021204611F0D8FA28B12BF02FF8BDE8EB
:102B5000104029F021B910BD805C0020FFF7D2BFE2
:102B600070B500F580450446D5F81C0D9FED5A0A56
:102B700086B06C302EF07CFF04F5955003A9103020
:102B80008DED030ACDED040A8DED051A12F0F2FB6E
:102B90000221204611F0B0FA70B10121204611F057
:102BA000ABFA48B94D4BD3F8EC0003689B6A9847E1
:102BB00010B9204602F0E0F90121204611F09CFAFC
:102BC00048B9464BD3F8EC0003689B6A984710B9A4
:102BD000204602F0E1F90121204611F08DFA10B9EA
:102BE000204602F031FA4FF40031204611F084FA09
:102BF00030B104F54053D3F8100103685B6C98477B
:102C00004021204611F078FA60B104F57F60019010
:102C100053F0F2FD04F58053019893F9C4300BB1E1
:102C200053F02CFF4FF48061204611F065FA18B183
:102C300004F57F6053F07AFE2021204611F05CFA03
:102C400058B104F54056D6F8EC0003681B69984764
:102C500018B3D5F8240D84F035FA8021204611F000
:102C60004BFA38B32AF0A2FF29F0BAF81021204617
:102C700011F042FA18B1D5F81C0D80F069FF4FF43D
:102C80000041204611F038FA18B304F59B403C305F
:102C900006B0BDE8704062F09DBD20460DF0ACFC72
:102CA0000028D6D1D6F8EC0003685B699847002865
:102CB000CFD0D2E74FF48021204611F01DFA002832
:102CC000D0D14FF40021204611F016FA0028C9D1C6
:102CD000CCE706B070BD00BFE02E6542805C0020EE
:102CE000FFF73EBF10B50121044611F005FA10B1FF
:102CF000204602F0A9F98021204611F0FDF958B1D3
:102D00004FF48021204611F0F7F928B92AF04EFF40
:102D1000BDE8104029F040B810BD0000FFF7E2BF49
:102D200010B5044605F020FD204605F06BFB20465B
:102D300005F060FD204612F0A9F82046BDE81040DD
:102D400003F0A6BCFFF7ECBF70B54FF6FF71044669
:102D500011F0D2F904F5405528B1D5F8E02007214B
:102D6000204602F0A1F9D5F8103193F8CB308BB999
:102D70002046FFF79FFAD5F8100104F500530268CA
:102D800093F87413166A93F8FE22B047D5F8100131
:102D900089F09AFB61F010FC61F00CF9204612F00A
:102DA00073F895F8E0300F4A04F58044DB43D4F81B
:102DB0001C5DC3F3C01353712B681E6F52F0BEFA33
:102DC00051F026FF2846B047D4F8244D52F0B6FA09
:102DD00004F5057451F01CFF2046BDE8704077F003
:102DE000DFBC00BFBD860020FFF7AEBF70B500F5A9
:102DF000A85300F540551B68C5F8243100F58056EE
:102E000006F20C5304461B68C5F82831D6F8B00406
:102E100000F58C4050302BF0CBFBD5F82431C5F8B1
:102E20003031D5F82831C5F82C01C5F834314FF6CA
:102E3000FF71204611F060F938B1D6F8B024204671
:102E40000921BDE8704002F007B970BD30B500F54A
:102E50004053D3F82041002C4CD093F8E120D10707
:102E600048D56FF3000283F8E12000F50052012CF1
:102E7000D2F8D41CD2F8D85CB1F908400BBFD3ED1E
:102E80004A5AD3ED4D5AD3ED497AD3ED4C7A07EE39
:102E9000104AB5F9084006EE904A0CBFF8EEE66A13
:102EA000F8EEE66AB8EEC77A25EEE66A00F5A853B2
:102EB000A7EE276A67EEA67AD3ED006AE7EE257AD9
:102EC00093ED037A27EE877AA6EE267ABDEEC77ACF
:102ED00017EE104A0C8193ED007AD2F8D82C67EEE9
:102EE000877A93ED037AE6EE477AFDEEE77A17EEFE
:102EF000903A138130BD000038B505462DED028BA8
:102F000000F5405471B1284610F03CFCD4F82C3147
:102F10001B1A03F2F31340F2E63293420CD8BDECD5
:102F2000028B38BDD4F82031022BF8D110F00EFC02
:102F3000B0F57A7FE7D2F2E7C4F82C0100F58C40B7
:102F40005030642390FBF3F308EE103ADFED097A7A
:102F5000B8EEC88A28EE278AB0EE480AB2F0CAFF57
:102F600084ED4C0AB0EE480AB3F04AF984ED4D0AFC
:102F7000D5E700BF35FA8E3C00F5955001211030A1
:102F800013F0CEBFFFF7F8BF10B5044610F004FEF3
:102F90001021204611F0B0F870B1204601F048FF32
:102FA0004FF40011204611F0A7F828B92AF0FEFDD1
:102FB000BDE8104028F0E2BF10BD0000FFF7E4BFFD
:102FC000F8B50446254606F0A3F9224B45F83C3BEC
:102FD000214BA465C4E91734204BC4E91934204BB4
:102FE000E36604F1800019F0B7FE04F19C0019F0CB
:102FF000B3FE04F1B80019F0AFFE4FF6FF76194B9F
:10300000C4F8CC30A4F8D06004F1D40019F0A4FEC8
:103010004FF0FF37144B1549C4F8307128461D6036
:103020004DF062FBA4F87870A4F8946004F5A270E7
:1030300019F092FE04F5B07019F08EFE04F5BE7022
:1030400019F08AFE002384F89031C4F8B431204688
:10305000F8BD00BFAC2D0D08992701089D27010878
:10306000A12701080000FFFF88860020C49A0D08F0
:1030700010B5044606F04CF90A4B23600123A387E0
:1030800004F1400019F068FE04F1500019F064FEEC
:1030900004F1600019F060FE04F1700019F05CFEAC
:1030A000204610BD90370D082DE9F047044688B042
:1030B000FFF71EFCA44B236004F50C50203004F5F0
:1030C000005502F027F904F50B532C3304F5335661
:1030D000C5F8E83C062385F8EC3C4FF07C5705A981
:1030E00006F13800059756F053FC06F150008FF0BA
:1030F000DFF8002304F59A4985F8283D192304A92F
:1031000085F8343D04F53456C5F8309D04F5355046
:10311000049756F03DFC06F158008FF0C9F80126DF
:10312000182304F5365004F5375785F87C3D3837B9
:1031300085F8706DC5F8789D103061F0B7FC3846A1
:103140007EF0BCFB814B8DF8186006AEC5F8F83DEB
:103150003146381D4EF0DEF804F5385030304AF074
:10316000C1FF04F5395030307EF092FB784B794F37
:10317000C5F8703E04F53A5031460830069756F0CF
:1031800007FC04F53A5031461430069756F000FC1F
:1031900004F53A503146203004F53A5A06970AF1C0
:1031A000380A56F0F5FB6C4BC5F8B83E0AF114002E
:1031B0008FF07EF804F53B5704F53D58303708F1A1
:1031C0001408384614375BF0C5F9B845F9D104F551
:1031D00040580723C8F878300023A8F87C304FF413
:1031E000CB701AF043F9C8F8740004F542508FF020
:1031F0005FF804F5435004308FF05AF8574B1A68C3
:103200000AB9C3F800A004F5AC47554BC5F8B83E61
:10321000643704F54350C8F8EC7030307FF028FE76
:10322000504B07934FF07E554F4BC8F82451C8F8C8
:1032300030510694009304F5445096E80C004FF486
:1032400000713C3016F014FD04F55A50303070F027
:10325000A7FC04F5994003A95030039556F0BEFB36
:1032600004F5994003A96430039556F091FB04F5E9
:10327000994004F58045703019F06EFD05F60C5349
:103280000026C9F80060C9F80460C9F808601E602B
:103290005E609E6004F595531033C5F8183D04F543
:1032A0009A40002385F8393D4FF400413C3017F037
:1032B000A9FA04F59B403C3062F034F904F59C40D7
:1032C00040306EF0FBFD04F59C407C304EF058F928
:1032D000264BC5F87C3E04F59D40254B2549103012
:1032E00004F59D48186008F130084DF0FDF9FF2302
:1032F00085F8C03E85F8C83E1F4940464DF0F4F9B8
:103300001E4A136813B11E488FF0EAFD1D491E487E
:10331000C2F8008004F59D42583208604FF0140E48
:103320001FFA83FC0EFB0C010133097C0029F7D145
:10333000164BA3F800C0164BD3F80080B8F1000F6D
:103340002AD01448E0E700BFB0D80C08A8D00C0879
:10335000E8D00C080000A04098E20D08EC8A00209C
:1033600030D90C0895270108A0D80C08F8D00C0813
:10337000A490002064F70D084C890E0838910020B5
:1033800034D10C0860870020181B0D085C870020D2
:103390001887002055D10C0804F59D401A6003A938
:1033A000584B03936C3056F0F3FA04F59E400C3002
:1033B00005F0AEFF544BC5F80C3F04F59E404C3071
:1033C00005F0A6FF04F5A249504BC5F84C3F04F5A3
:1033D0009F4009F16009083004F5A045FFF7F0FDB2
:1033E000484605F095FF4A4BC5F8603109F13C00AD
:1033F0008CF042FC474BC5F89C3104F5A6402030C8
:1034000005F086FF444BC5F8203304F5A640643030
:1034100005F07EFF414BC5F8643304F5A74085F8FD
:10342000A083243005F074FF3D4BC5F8A43304F5A8
:10343000A740603005F06CFF3A4BC5F8E03305F269
:103440001C4304F5A8401E605E609E60343005F0A9
:103450005FFF354BC5F8343404F5A840C5F87084D7
:103460007C3005F055FF314BC5F87C3404F5A9409C
:10347000C5F8B884403005F04BFF2D4BC5F8C0347B
:1034800004F5AA40083005F043FF2A4BC5F808357B
:1034900004F5AA40443005F03BFF274BC5F84435FE
:1034A00005F2BC5304F5AB401E605E605830FFF778
:1034B000DFFD384605F02CFF204BC5F8643604F5D7
:1034C000AD40203005F024FF1D4BC5F8A03604F5B3
:1034D000AD40A5F8DC867030FFF7CAFD194BC5F882
:1034E000F036012385F8793704F5AF4318461E609E
:1034F0005E609E600C300AF04BFD204608B0BDE8CF
:10350000F08700BFCDCC4C3DA4290D08482A0D08FA
:10351000502E0D08E02E0D089C2F0D083C300D0894
:10352000DC300D0874310D08B0330D0850340D082F
:10353000E0340D0878350D0818360D08EC380D0804
:10354000883A0D0848380D0838B5054B1C682368C3
:103550000A461D68034B01462046A847002038BD97
:10356000E0840020802C002010B58FF017F9064C65
:10357000064B18602046FFF797FD2046044A054990
:10358000BDE81040B2F090BB802C0020E084002009
:10359000D4E200205D2801080120704790F89C309B
:1035A0008B4286BF283150F8210000207047000070
:1035B00090F89C308B4286BF283150F821000020C3
:1035C00070470000FA207047014B93F8AE02704735
:1035D000804C0020034BD3F82001431E5842584131
:1035E000704700BF805C0020034BD3F82001831E8E
:1035F00058425841704700BF805C0020034BD3F80D
:10360000100108B187F00ABE01487047805C0020B5
:103610001CD90C0838B5C36A2E4D43F4E052C2627F
:10362000026B42F4E0520263426B42F4E0524263A6
:10363000D5F8242D0446E2B143F4F843C362D5F82B
:10364000240D83F0FFF838B1236B43F480432363E8
:10365000636B43F480436363D5F8240D83F014FA5D
:1036600038B1236B43F400532363636B43F400537B
:103670006363194B1D6845B1192128464EF048FA7D
:1036800018B1E36A43F48073E362144B93F8F03C9F
:103690006BB1236B43F48073236345B11921284632
:1036A0004EF06EFA18B1636B43F480736363E36AA0
:1036B00043F08043E362236B43F080432363084B72
:1036C000D3F8103193F8C1301BB9636B43F08043DA
:1036D000636338BD806C002070870020804C002020
:1036E000805C002013B54FF44470CDE9002119F03F
:1036F000B7FE044628B1DDE900215DF035FE024B3E
:103700002360204602B010BD74DB0C080020704717
:10371000704700000320704708207047014B93F862
:10372000B0027047804C0020034B93F968030038C7
:1037300018BF0120704700BF804C0020014B93F957
:10374000B2027047804C00207047000070470000B4
:1037500008B50C4BD3F8240D70B910230A4AD2F8DF
:10376000102143F0400022B192F8CB200AB143F07F
:10377000C00040F0010008BD83F064F80028ECD0E0
:103780001823EBE7806C0020805C002038B5C578FA
:103790000B46352D044628BF352535220021184615
:1037A000B4F0F0FF2A4604F10C01BDE83840B4F053
:1037B0009FBF00001FB5184C94F8E610A4F16800F4
:1037C00011F01AFD78B194F8E610A4F1680011F038
:1037D00015FD40B194F8E610A4F1680004B0BDE80E
:1037E000104011F00DBD002301930293039313F0D9
:1037F00033FC01A913F0FCF920B101A82EF036FD2D
:1038000004B010BD23F0D2F890F8F432B02202FBDD
:10381000030090ED3B0AF3E7804C002008B50D4B08
:10382000D3F81001A8B1443055F0C0FF034693ED22
:10383000000ADFED090A9F20B7EE001A2AF0E4FE25
:10384000DFED067A20EE270ABDEEC00A10EE103A30
:1038500018B208BD805C0020000000000000C842D3
:103860002DE9F04FDFF8D880344F8DB004460425A1
:1038700008F5005617F8019BB8F9083309F1FF3A2B
:1038800043FA0AF3D90742D5207C57F023FC83463C
:10389000207C58F023FB00F121039B4505D2207CBE
:1038A0000DB0BDE8F04F56F06BBEBAF1030F2ED845
:1038B000DFE80AF00234393ED6F81C0D03689B6835
:1038C000984700F194035A69D3F800A0D3F804E0B4
:1038D000D8681969D3F818C008925A6A1B6ACDF8DB
:1038E0002520CDF8293062222123CDE9003206902F
:1038F0000791207CCDF80CA0192303AAC221CDF892
:1039000010E0CDF814C08DF8249057F04DFC013D27
:1039100015F0FF05AED10DB0BDE8F08FD6F81C0D47
:103920000368DB68CCE7D6F81C0D03681B69C7E7A2
:10393000D6F8243D03F52A73C5E700BF48DC0C0820
:10394000804C002013B504460748019108F0CCFFD5
:1039500030B90199204602B0BDE8104058F0FEBCD5
:10396000042002B010BD00BF087C0020014808F010
:1039700097BD00BF087C002037B504460D460648B9
:10398000019211468AF03CFF019A2946204603B075
:10399000BDE830405CF0B6BB1858002010B588B0C8
:1039A000044659F0D9FE0C4BD3F8100138B90B4A34
:1039B0000621204608B0BDE8104059F0B5BE694662
:1039C0001E2287F02FFC064A6B460621204659F03E
:1039D000ABFE08B010BD00BF805C002068D90C08A9
:1039E00022270D08034A92F8D03C013382F8D03CDC
:1039F00058F076BF804C002007B50846019119F0B9
:103A000081FA38B10448019902F0DEFC002003B0CD
:103A10005DF804FB0420FAE7EC840020F7B58B8BFB
:103A2000CD2B06460C4617461DD1D1ED067AFCEE8D
:103A3000E77ACDED017A9DF80430022B13D10E4DBB
:103A400095F8351E05F6BC5061F0A2FD58B195F809
:103A5000351E05F6BC5061F0A3FD20B994ED020AB5
:103A6000064802F091FC3A462146304603B0BDE8D4
:103A7000F04058F0C7BF00BF806C0020EC840020ED
:103A8000162A10B40C4605D0542A03D05DF8044B16
:103A900058F080BC0323237001205DF8044B70476D
:103AA00008B558F0D3FE40F41C6040F00D0008BD8E
:103AB00010B5044619F0DCFC204610BD10B50C4CC6
:103AC00094F9E030002B0FDBD4F8EC000368DB6CDA
:103AD000984758B9D4F8EC0003689B6C98470028C5
:103AE0000CBF0220032010BD0120FCE70420FAE7F0
:103AF000805C002010B44C69012C05D101465DF8B2
:103B0000044B034802F0F4BF5DF8044B58F002BFC9
:103B1000802C00202DE9F341B1F90430002B06463A
:103B20000C46154635DB4FF00008CDE900281A4F4A
:103B3000B1F902209FED190AD7F8D41C4FF47A731B
:103B40005CF0C8FD0123CDE900539FED140AB4F9E0
:103B50000020D7F8D81C4FF47A7330465CF0BAFDD9
:103B60009FED0F0AB4F90420D7F8DC1C4346304619
:103B7000CDE900585CF0AEFDCDE900589FED070A95
:103B8000B4F90620D7F8E01C4FF47A7330465CF0A5
:103B9000A1FD02B0BDE8F081804C00200000FA4495
:103BA00000007A44044B187820B9044B93F8E200E3
:103BB000C0F38010704700BF58860020805C002052
:103BC0000B4B93F8AD267AB993F8052192060BD1E9
:103BD00093F9E020002A09DB93F8E13013F0200F7D
:103BE00014BF042001207047052070470320704750
:103BF000805C002008B5074B93F9FC32032B03D0FF
:103C0000BDE8084059F008BE034A022159F08CFD76
:103C1000042008BD804C002080D90C08094BD3F843
:103C20006C23920701D458F0A9BB03F5005303F6A7
:103C3000F44393ED000ADFED047AB8EEC00A20EEFB
:103C4000270A7047804C00200AD7233C10B594B057
:103C5000044603A819F080F81C4BD3F8EC00036865
:103C600003A95B6D984778B3002103A819F00CF9FC
:103C700050B3247C8FF066F9059BDDED047A089340
:103C8000069B09930023F8EEE77A9FED117A0B93D8
:103C90000C930D930E930F931093119312934FF671
:103CA000F853ADF84C300023962267EE877A8DF8F2
:103CB0004E303323CDE90032079007AA5721204622
:103CC000CDED0A7A57F070FA14B010BD805C002078
:103CD0000AD7233C30B52DED0A8B774C0546D4F836
:103CE000EC00036899B05B6A984700285BD004F544
:103CF0000054D4F8B834062B00F2C980DFE803F092
:103D00000404045788AB53006C489FED6D8A0BF098
:103D100081FF9FED6C0A0168426883680D930BA8D0
:103D20000B910C922DF0A4FEF0EE489AB0EE40CA32
:103D3000F0EE60BAB0EE419AB0EE48AAF0EE488AD2
:103D4000F0EE48AAB0EE48BA40F6F8542D7C8FF059
:103D5000F9F800231593169301238C228DF85E3019
:103D60003323CDE900320B90B1EE499AF1EE688A27
:103D7000B1EE488A0BAA552128468DED0CCACDED2F
:103D80000DBA8DED0E9A8DED0FBACDED10AACDEDD9
:103D9000118A8DED12AACDED139A8DED148AADF82E
:103DA0005C4057F001FA19B0BDEC0A8B30BD4348B6
:103DB0000BF030FF9FED430A0168426883680D9362
:103DC0000BA80B910C922DF053FE3C48F0EE60BA1C
:103DD000B0EE419AB0EE40CA0BF020FF9FED390AD9
:103DE0002DF046FE3548B0EE40BAF0EE60AAF0EE97
:103DF000418A0BF017FF9FED330A2DF039FE4FF487
:103E00004064B0EE40AAF0EE609AB0EE418A9DE7C1
:103E10002A489FED2B9A0BF001FF9FED2A0A2DF007
:103E200027FE2648B0EE40BAF0EE60AAF0EE418AD6
:103E30000BF0F8FE9FED230A2DF01AFEF0EE49BAC2
:103E4000B0EE40AAF0EE609AB0EE418AB0EE49CAF8
:103E500040F607447AE71948DFED198A0BF0E2FED5
:103E60009FED180A2DF004FEF0EE68AAB0EE40AA0D
:103E7000F0EE609AB0EE418AB0EE68BAB0EE689AA1
:103E8000F0EE68BAB0EE68CA40F63F445EE79FEDD8
:103E90000C8A0024F0EE489AB0EE48AAF0EE488A68
:103EA000F0EE48AAB0EE48BAB0EE489AF0EE48BA42
:103EB000B0EE48CA4AE700BF805C0020FC800020CA
:103EC000000000000AD7233C2DE9F0412DED068BC0
:103ED0003B4D95F8E13099068CB004466AD505F55E
:103EE00080579FED380AD7F81C0DDFED378A6C300C
:103EF0002DF0BEFD8DED041A21EE281AD5F8EC60E8
:103F00008DED020ABDEEC11ACDED030A11EE103A95
:103F10001DB2336894F810809B6D304660EE289A8D
:103F200020EEA89A984707EE900AF8EEE77A304616
:103F300067EEA87AFDEEE77A17EE903A1CB2336886
:103F4000DB6D984707EE900AB8EE678AD7F8243DF4
:103F5000DFED1E7A93ED0FAA336828EE288A1B6ED8
:103F6000B4EEE78AF1EE10FA58BFB0EE678A304639
:103F70009847BCEEC88A0023089318EE103AB7227F
:103F80002AEE28AA20EE280AADF82C301A23CDE913
:103F900000323E2105AA4046CDED059A8DED069AE8
:103FA0008DED07AA8DED090AADF82850ADF82A402D
:103FB00057F0FAF80CB0BDEC068BBDE8F08100BFFD
:103FC000805C00209F0CB3450AD7233C00FF7F474D
:103FD0002DE9F04F2DED028B1A4B047CD3F81C3DDC
:103FE0008DB0D3F88480D3F88870D3F88C60D3F880
:103FF000905093ED258AD3F898B0D3F89CA0D3F8CD
:10400000DC908EF09FFF00238DF82C3016222523A4
:10401000CDE90032029002AA532120468DED078A95
:10402000CDF820B0CDF824A0CDF82890CDF80C80A4
:1040300004970596069557F0B7F80DB0BDEC028BC6
:10404000BDE8F08F806C002070B58A7A4B7A43EA25
:104050000223CA7A43EA02439D2B06460C4621D12D
:10406000134D95F8351E05F6BC5061F091FAC8B1B4
:1040700095F8351E05F6BC5061F09EFA022811D164
:1040800095F8351E05F6BC5061F08AFA50B9D4EDAA
:10409000057A9FED080A0848F8EEE77A27EE800ACD
:1040A00002F072F921463046BDE8704058F018BB66
:1040B000806C00200AD7233CEC840020054BD3F809
:1040C00010312BB193F8CA00002808BF02207047B6
:1040D00002207047805C002008B5034BD3F8EC0049
:1040E00003681B68984708BD805C0020024B93F86A
:1040F000E100C0F340107047805C002070B52C4E8A
:104100002DED028B0546D6F8EC0091ED018A03688F
:1041100086B05B6A0C46984750B9BDEEC88A18EE67
:10412000103ADB0704D4022006B0BDEC028B70BD50
:10413000D4E904012BF0F6FA0028F4D002A818F014
:104140000BFE02AA214628465CF034FA0028EAD089
:10415000184902A818F0E2FE03460028E3D1DFED7B
:10416000160A00900246B0EE600A144802A90BF04D
:1041700089FBD8B1D6F8EC0003685B6A984704461F
:1041800008B10020D0E70E480222042105F058FCB7
:1041900060B1DFED090A094800942346B0EE600AD9
:1041A000224602A90BF06EFB0028EAD10420BBE7EF
:1041B000805C00207079002000000000FC8000205E
:1041C000802C002008B591F82030032B1CD1D1EDB4
:1041D000027A9FED0E7A91ED060A0D4BF0EEE77A2A
:1041E000F4EEC77ADFED0B7AD3F8EC00F1EE10FABB
:1041F0004CBF0121002120EE270A10F095FA00287B
:1042000014BF0020042008BD0220FCE70000003499
:10421000805C00200000C84210B52DED028BD1ED6E
:10422000007AF5EEC07AF1EE10FA82B00C4604DAAC
:10423000042002B0BDEC028B10BD9FED197AF4EEA4
:10424000C77AF1EE10FAF3D891ED030A9FED158AC3
:10425000F0EEC07AF4EEC87AF1EE10FA19D5D4ED8A
:10426000037A1148D4ED010A94ED000AF4EEC87AFD
:10427000D4ED027AFDEEE77AF1EE10FACDED017A97
:104280009DF90410ACBF0122002201F0DFFF0020E5
:10429000CFE7F7EE000A2AF0B3F80028C8D0DEE72F
:1042A0000000B44300000034EC84002091ED010ACA
:1042B000B5EEC00AF1EE10FA08B501DC042008BD25
:1042C0009FED107A104BD1ED007AD3F8EC0020EE80
:1042D000070A9FED0E7A0368F4EEC77AF1EE10FA42
:1042E00005DDDB6E98470028E8D00020E7E79FED6A
:1042F000087AF4EEC77AF1EE10FACCBF9B6E5B6ED3
:10430000F0E700BF0000C842805C00209A99394065
:104310003333F33F08B5D1ED007A9FED157AF0EE17
:10432000E77AF4EEC77AF1EE10FA1DD5D1ED017AF5
:10433000F0EEE77AF4EEC77AF1EE10FA14D50D48F4
:104340000222032105F07CFB80B10A480121FDF720
:104350003FFF094890F8C83F012B03D000F6C47016
:1043600030F0FEFE002000E0022008BD0420FCE743
:1043700000000034802C0020806C002010B5D1EDAE
:10438000007AFCEEE77A17EE903A9CB2012C02D04C
:10439000022C06D04CB90648214666F0DFFF00200B
:1043A00010BD044803F05CF9F9E70420F8E700BF0A
:1043B000107B0020802C00201FB5D1ED017A0B7CF2
:1043C000FCEEE77ACDED027AD1ED007A0093FCEEB7
:1043D000E77AD1ED030ACDED037A91ED020A9DF85B
:1043E00008309DF80C20014602480EF059FF05B038
:1043F0005DF804FB802C002010B50A4C94F80531C0
:10440000DB070CD402220521A4F5405005F018FB6F
:1044100028B902221146A4F5405005F011FB0020F6
:1044200010BD00BF805C002010B5D1ED007AFCEE1D
:10443000E77A044617EE903A13F0FF030FD10F4BC3
:10444000D3F8EC0003689B6F984708B1002010BDBB
:104450000B4A2046062159F067F90420F7E7012BA3
:1044600009D1064BD3F8EC000368DB6F98470028AE
:10447000ECD1044AEDE70220E9E700BF805C0020B0
:10448000A4D90C08B4D90C089FED0B7A01F10C03E8
:10449000F1EC017AF4EE677AF1EE10FA0AD6F0EE5A
:1044A000E77AF4EEC77AF1EE10FA03DC9942EFD125
:1044B000012070470020704700007A4430B52DED90
:1044C000028B8DB00023054603930493059312F0ED
:1044D000C3FD03A912F08CFB58B312F0BDFD00F52B
:1044E0005A7393E8070006AC84E80700DDED060A7E
:1044F0009DED070A2D7CF1EE600AB1EE400AB1F0A5
:104500004BFF2046B0EE408A2DF0B0FEDFED0B7A77
:10451000089B0B93012228EE278A0C23CDE9003259
:10452000A82109AA28468DED098A8DED0A0A56F0C0
:104530003BFE0DB0BDEC028B30BD00BFE02E6542EE
:10454000242938B505460FD003D81B2907D10124EB
:1045500012E04029FBD0A1F14203012BF7D92846F4
:10456000BDE838405CF012BA0C2156F01BF8044646
:1045700010B12846FFF7A2FF204638BD38B5194CC8
:1045800094F80531DB070D460AD4D4F8103193F8BE
:10459000CB303BB901221146A4F50270FDF76EFC49
:1045A000002038BD94F9E030002B4FF0020212DAFF
:1045B0000521A4F5405005F043FA0028F0D095ED10
:1045C000000ADFED097AD4F8EC0020EE270A012179
:1045D00010F0AAF8E4E70921A4F5405005F030FAFC
:1045E000DEE700BF805C00200000C84210B5214C0F
:1045F00094F80531DB070ED4D4F8103193F8CB30A2
:104600004BB194F9E030002B07DA01220821A4F520
:104610000270FDF7E7FC002010BDD1ED007A9FEDA0
:10462000167AF0EEE77AF4EEC77AF1EE10FA0BD5CF
:1046300012480222112105F003FAA0B90222114604
:104640000E4805F0FDF9E6E7D4F8EC0003681B68B6
:1046500098470428DFD0D4F8EC0003681B6898471B
:104660001428E5D1D7E7064840F6C41108F03EFE0D
:10467000D1E700BF805C002000000034802C0020C7
:10468000A07F002073B58B8BC12B05460C4644D808
:10469000BB2B0DD8202B63D02ED8113B99B2052906
:1046A00018D92146284602B0BDE870405DF060BAD6
:1046B000BC3B052BF5D801A151F823F0FB470108BD
:1046C00005480108A3460108A346010893470108CD
:1046D0009F470108052BE4D801A151F823F000BF42
:1046E000E1470108A3460108A3460108F547010870
:1046F00007470108B5470108732B2CD006D8542B67
:1047000058D0552BCDD1022209216BE0B22BC8D154
:1047100002B0BDE87040FFF7C9BD4AF21146B3428E
:1047200054D00BD8D12B40D0B3F5967F53D0D02B9B
:10473000B7D102B0BDE87040FFF720BE4AF2124682
:10474000B3423ED04AF21346B342AAD102B0BDE80A
:104750007040FFF74BBF02B0BDE87040FFF75CBD93
:10476000D1ED007AF5EEC07AF1EE10FA4FDD9FED53
:10477000297AF4EEC77AF1EE10FA48D8FCEEE77A1F
:10478000254ACDED017A9DF80430A2F89A3B00202D
:104790002EE0214602B0BDE87040FFF7AFBC2146D5
:1047A00002B0BDE87040FFF73FBE02B0BDE8704008
:1047B000FFF702BE2146284602B0BDE87040FFF771
:1047C00001BD02B0BDE87040FFF7D8BE02B0BDE841
:1047D0007040FFF711BE02B0BDE87040FFF79ABD10
:1047E000022205210D4805F02BF90028CFD1042025
:1047F00002B070BD02220621F4E70221084806F04B
:1048000097FAF2E70221064806F05CFAEDE702208B
:10481000EEE700BF00007F43804C0020802C00208A
:10482000087C002008B591ED007AF6EE007AB4EE2F
:10483000E77AF1EE10FA06DD044801220521FDF7C2
:10484000D1FB002008BD0420FCE700BF785A0020FF
:1048500030B52DED028BCD7893B0272D28BF2725BD
:104860000C462722002108A8B3F08CFF2A4604F149
:104870000C0108A8B3F03CFF424BD3F8EC000368EE
:104880005B6A9847002841D09DF8465068063DD4A1
:1048900000244FF07E532906049307940694059450
:1048A00027D504A82CF08EFBEA0701940294039408
:1048B00005F006032ED4002B2ED10D9B01930E9BE9
:1048C00002930F9B039330480AF08AFD9DED100A76
:1048D000044630B340F2ED40B7EE001AFFEE000A96
:1048E00029F092FE2848234601AA04A90AF080FD77
:1048F0000CE0099B04930A9B05930B9B069304A869
:104900000C9B07932CF064FB0028CDD113B0BDECB9
:10491000028B30BD062BD6D001211B480AF0FCFCCF
:10492000F4E7DFED1A0A4FF49E60B7EE001A29F0A3
:104930006BFEF6EE000AB0EE408A29F061FDE8B9A0
:10494000B6EE000A124BB4EEC08AF1EE10FAD3F8BC
:10495000283D08DD38EE400A30EE008A93ED070A64
:1049600028EE000ABEE730EE480AD3ED087A30EEB2
:10497000000AF0EEE77A27EEC00AB3E79FED030ADC
:10498000B0E700BF805C0020FC8000200000000039
:10499000806C00202DE9F0439DB0814608460EA9A9
:1049A000FEF7F4FE844BD3F8EC0003685B6A98478B
:1049B00050B19DF86C30012B09D0DA1F022A06D9BC
:1049C0007E4801210AF0A8FC1DB0BDE8F083BDF8C7
:1049D0006840A20504F0070604F0380704F4E07507
:1049E00001D5002DF0D04FF00008CDF81480CDF89F
:1049F0001880CDF81C803EBB9FED716A9DED107A4A
:104A0000DDED117ADDED0F6A27EE067A67EEC67AE4
:104A100066EE866A083B012BCDED056A8DED067AC0
:104A2000CDED077A04D8674806AA05A9FDF74AFD27
:104A30009DF86C30073B022B06D8634885F046FB97
:104A4000014605A82DF034F8CDF82080CDF824805B
:104A5000CDF82880F7B9DDED147A129B0893F1EEBA
:104A6000677A139B099308A94846CDED0A7AFFF7A8
:104A70000BFD0028A4D09FED520A08A82DF04CF899
:104A80009DF86C30083B012B04D84E4809AA08A9B0
:104A9000FDF718FDCDF82C80CDF83080CDF83480AE
:104AA000EDB99FED476A9DED167ADDED177ADDEDE4
:104AB000156A9DF86C3027EE067A67EEC67A66EEC8
:104AC000866A083B012BCDED0B6A8DED0C7ACDED9E
:104AD0000D7A04D83B480CAA0BA9FDF7F3FC14F49B
:104AE000806233D1DFED397A9DED180A9DF86C10A4
:104AF00020EE270ADFED327A0839012920EE270A55
:104B00008CBF0021012114F4006305BFDFED2F7A73
:104B1000DDED190ADFED2E0A60EEA70A04BFDFED16
:104B2000287A60EEA70AAEB9002F35D1B3FA83F325
:104B3000B2FA82F25B0952090291019300920BAB27
:104B400008AA05A91D480AF055FD3DE79FED200A7A
:104B50000021D8E77FB9B3FA83F35B090120009302
:104B6000B2FA82F3CDE901105B0914480BAA08A937
:104B70000AF0D8FF28E7002D7FF422AF0120B3FA16
:104B800083F3B2FA82F2CDE900105B090B485209B7
:104B90000BA90AF06FFF17E7002D3FF411AFB3FA2E
:104BA00083F3B2FA82F2CDE900165B09520905A936
:104BB00002480AF0A1FD07E7805C0020FC8000208D
:104BC0000000C842802C002080790020E02E654241
:104BD000000000002DE9F047A2B08046084614A965
:104BE000FEF7D4FD7E4BD3F8EC0003685B6A984770
:104BF000C0B1BDF88040A30504F0070904F4E077D4
:104C000000D57FB10CAE304618F0A6F8B9F1000F10
:104C100029D1DDE915012AF085FD30B9714801215E
:104C20000AF07AFB22B0BDE8F0879DF8841009AA4B
:104C300040465BF0A9FC0028F0D0DDED177A9FED2F
:104C40006A7A099B009367EE877A10ADFDEEE77AEA
:104C5000DDE9151217EE903A284618F09DF895E810
:104C60000F0086E80F00002514F0380A0695079516
:104C7000089514D1DDED1A7A189B0693F1EE677A48
:104C8000199B079306A94046CDED087AFFF7FCFB78
:104C90000028C3D09FED540A06A82CF03DFF0995CB
:104CA0000A950B959FB99FED506A9DED1C7ADDED3D
:104CB0001D7ADDED1B6A27EE067A67EEC67A66EE90
:104CC000866A8DED0A7ACDED096ACDED0B7A14F482
:104CD000806805BFDFED457A9DED1E0A9FED440A11
:104CE00020EE270A04BFDFED407A20EE270A14F4F5
:104CF000006405BFDFED3D7ADDED1F0ADFED3C0A04
:104D000060EEA70A04BFDFED387A60EEA70AB9F1BA
:104D1000000F31D1BAF1000F52D13046CDED050A66
:104D20008DED040A18F048F803289DED040ADDED26
:104D3000050A3FF473AF10A93046CDED050A8DED9D
:104D4000040A10951195129518F096F900283FF471
:104D500065AFB4FA84F46409B8FA88F3DDED050AA6
:104D60009DED040ACDF804A000945B0906AA10A9E1
:104D70001C480AF0AFFC55E7BAF1000F0FD1012330
:104D8000B4FA84F4CDE901A36409B8FA88F31548AC
:104D900000945B0909AA06A90AF0C4FE42E7002FA5
:104DA0007FF43CAF0123CDE90073B8FA88F2B4FA7E
:104DB00084F30C485B09520909A90AF05BFE31E74C
:104DC000002F3FF42BAFB4FA84F3B8FA88F2CDF891
:104DD00000905B095209314602480AF053FD21E771
:104DE000805C0020FC8000200000C842E02E65426C
:104DF0000000000010B44B7A8C7ACA7A43EA04238C
:104E000043EA0243542B07D0562B09D0522B0BD127
:104E10005DF8044BFFF71CBD5DF8044BFFF7BABD0E
:104E20005DF8044BFFF7D6BE5DF8044B5CF07CB830
:104E30002DE9F0432DED028B00F540590446D9F8D9
:104E4000EC00DFED4A8A036891B05B69984704F58E
:104E500080470026002840F08480D7F8243DD3ED19
:104E6000DE7A93EDD88AFDEEE77A28EE288A17EEEF
:104E7000903A1DB204F5365801A940460EF0F4FFF1
:104E800018B953F061F83A4B01933722002102A878
:104E9000B3F078FCA3238DF8083095238DF8093002
:104EA0008EF058F8D7F81C3DCDF80B00D9F810015A
:104EB000D3F8DC20D3F8E030CDF80F104430CDF833
:104EC0001320CDF8173054F071FC0346DFED290AAA
:104ED00093ED000AB7EE001A9F2029F095FB10EE23
:104EE000103AD9F81001CDF81B3003681B699847B8
:104EF00010EE103A04F59A49CDF81F3018EE103A2A
:104F00004846CDF8233085F0E5F820EE280A4046E3
:104F100010EE103ACDF82730D7F8CC3CCDF82B3036
:104F2000019BCDF82F300EF0C1FF10EE103A48462D
:104F3000CDF83330CDF83760ADF83B5085F0D6F87A
:104F4000BDEEC00A372210EE103A02A904F57F60C8
:104F5000ADF83D3052F04AF911B0BDEC028BBDE81E
:104F6000F08308EE106A002584E700BF0AD7233CCF
:104F70002292CA7F0000000010B500F58044D4F8EA
:104F80001C0D7DF08FFFD4F8241DD4F81C0DBDE856
:104F900010407DF0EDBF000070B54FF48051044625
:104FA0000FF0AAF800284ED004F5804604F57F657E
:104FB000D6F81C0D03689B689847692100F194029C
:104FC000284651F0ABFFD6F81C0D0368DB68984704
:104FD0006A2100F19402284651F0A0FFD6F81C0D7A
:104FE00003681B6998476B2100F19402284651F031
:104FF00095FFD6F8242D6C21284602F52A7251F02F
:105000008DFF202120460FF077F8E0B104F54053E2
:10501000D3F8EC0003681B69984778B1D6F8242DC3
:10502000284690326E2151F079FFD6F8242D28467B
:10503000BC32BDE870406F2151F070BF20460BF0CC
:10504000DBFA0028EAD170BD08B512F005F8BDE81A
:10505000084011F07FBD00007FB50E464FF6FF718E
:10506000044615460FF048F8E0B1102200216846CA
:10507000B3F088FBA3238DF8003095238DF8013021
:1050800003238DF802308DF065FF1022CDF8030068
:10509000CDF8071004F57F6069468DF80B60039525
:1050A00052F024F904B070BD7FB50E464FF6FF7183
:1050B000044615460FF020F8E0B1102200216846A2
:1050C000B3F060FBA3238DF8003095238DF80130F9
:1050D00004238DF802308DF03DFF1022CDF803003F
:1050E000CDF8071004F57F6069468DF80B600395D5
:1050F00052F0FCF804B070BD30B52DED048B87B0D4
:1051000004460D46182200216846B0EE409AF0EEA3
:10511000608AB0EE418AB3F035FBA3238DF80030EE
:1051200095238DF8013006238DF802308DF012FFA3
:105130001822CDF80300CDF8071004F57F6069460A
:105140008DF80B508DED039ACDED048A8DED058A17
:1051500052F04CF807B0BDEC048B30BD10B54FF4E5
:10516000801104460EF0C8FF30B104F595501030A0
:10517000BDE8104010F0D8B910BD00002DE9F04393
:105180008FB01446054689463122002101A8DDE989
:1051900016769846B3F0F6FAA3238DF804309523DB
:1051A0008DF8053008238DF806308DF0D3FE236886
:1051B000049363680593A36806933B68CDF81D309C
:1051C0007B68CDF82130BB68CDF825303368CDF849
:1051D00029307368CDF80700CDF80B10CDF82D30CD
:1051E0003122B3688DF80F9001A905F57F608DF825
:1051F0001C80CDF8313051F0F9FF0FB0BDE8F083DD
:1052000070B52DED068B8CB0144605460E462C224B
:10521000002101A8B0EE409AF0EE608AB0EE418A1B
:10522000B0EE61AAF0EE429AB3F0ACFAA3238DF887
:10523000043095238DF805300B238DF806308DF062
:1052400089FEDFED1A7A94ED007ACDF8070027EE9B
:10525000277A29EE279A8DED077A94ED017ACDF819
:105260000B1027EE277A68EEA78A8DED087A94ED69
:10527000027A8DF80F6028EE278A67EE277A2C22B3
:1052800001A905F57F608DED049ACDED058A8DEDC0
:10529000068ACDED097A8DED0AAACDED0B9A51F073
:1052A000A5FF0CB0BDEC068B70BD00BFE02E6542C3
:1052B000A020704730B5154B89B004466946D3F835
:1052C000100104F57F651E2285F0ACFF6A46104987
:1052D000284652F027F904F54053D3F8EC00036850
:1052E0001B68984704F50053014693F86822284646
:1052F00052F03CF904F59550103012F013F904F512
:10530000907020F0BDFB09B030BD00BF805C002074
:1053100022270D082E4B2F4A70B5436000234361AE
:105320008361C361C3632C4B426303644FF08042CB
:105330002A4B43640446826358305DF05DF9284E81
:10534000284BA365A82560195DF00CFB665130352C
:10535000B5F56A7FF7D1244D04F56A705FF004F863
:10536000002104F2BC7088F04DFBC4F8705804F6BC
:105370007800A5F5BE6589F01BF89FED1C1ADFEDDE
:105380001C0A9FED1C0AC4F8085904F61C107EF094
:105390007BFB9FED161A9FED180AF0EE410A04F60A
:1053A00034107EF071FB9FED111A9FED130AF0EEA1
:1053B000410A04F64C107EF067FB20460F494BF083
:1053C00093F920460E494BF08FF9204670BD00BF7F
:1053D000F03800200000C8410AD7233C0000E0401C
:1053E0008C240D08A0240D080C840020000000006F
:1053F0009A99993E0000B44300804A4308180D086A
:10540000881A0D0870B54C4D4C49ADF50E7DD02273
:1054100006465AA8B3F06CF90FCD0EAC0FC40FCDF1
:105420000FC40FCD0FC495E80F0084E80F000024CF
:105430005AAB18190021B7EE000A10344AF010FEDA
:10544000D02CF5D13E4B0FCB02AC84E80F0001A964
:1054500020464AF0B9FD90B19DF90430DFED396A7C
:10546000E06807EE103AB8EEC77AF0EE007AE7EEA1
:10547000267AB7EE000A80EE270A4BF0D5FC00240E
:105480000EAB181900211034B7EE000A4AF0E8FDFF
:10549000402CF5D12C49902236A8B3F029F90022EE
:1054A000092136A84AF088FE96F9A469D6B9274D95
:1054B0000FCD1EAC0FC40FCD0FC40FCD0FC495E898
:1054C0000F0084E80F00324604211EA84AF074FE43
:1054D0009FED1F0A1F484BF0A7FC1F48B7EE000ABC
:1054E0004BF0A2FC1D4C9FED1E0A0FCC06AD0FC564
:1054F00094E80F0085E80F00002106A84AF0B0FDEF
:105500009FED170A002128464AF0AAFD04F1100178
:1055100060221EA8B3F0ECF800241EAB181900217D
:10552000B7EE000A10344AF09BFD602CF5D15EF016
:10553000A7FC0DF50E7D70BD10CA0C0840C90C0803
:1055400050CA0C08CDCCCC3D60CA0C08F0CA0C087F
:1055500000000000F0160D08FF160D0830CB0C08F7
:10556000000034422DE9F04790B00DF106011D20F6
:105570005EF07AFD002800F09E809DF80630614ABA
:105580000133DBB211210BA88DF806308CF0B6FE8A
:1055900000220DF107010BA84AF048FA9DF80630E9
:1055A000594A112105460BA88CF0A8FE00220DF1E6
:1055B00007010BA84AF03AFA9DF80630534A112128
:1055C00006460BA88CF09AFE00220DF107010BA8ED
:1055D0004AF02CFA9DF806304D4A03F03F031121A2
:1055E00007460BA88CF08AFE00220DF107010BA8DC
:1055F0004AF01CFA8046002D5DD0002E5BD0002FB3
:1056000059D0002857D028464AF028FC002852D10B
:1056100030464AF023FC00284DD138464AF01EFCA3
:10562000002848D140464AF019FC002843D1394CA3
:1056300094E80F000DF10C0C10348CE80F0094E886
:105640000F000DF11C0989E80F0002A960464AF01D
:10565000BBFC98B3BDF8084002A948464AF0B4FC28
:1056600000284AD0BDF8083054BB23B340F2E244CE
:105670009C420FFA84FA0FFA83F927D80DF10A0138
:105680003046ADF80A904BF0C5FE0DF10A012846F0
:10569000ADF80AA04BF0BEFE0DF10A013846ADF898
:1056A0000AA04BF0B7FE00230DF10A014046ADF809
:1056B0000A304BF0C9FE10B0BDE8F0870024CBE7FC
:1056C00040F2D662002B08BF1346D1E70DF10A0164
:1056D0003046ADF80AA04BF09DFE0DF10A012846B8
:1056E000ADF80A904BF096FE0DF10A013846ADF880
:1056F0000A904BF08FFE0123D6E7002CDBD040F25E
:10570000D663B5E710170D081C170D0828170D08EC
:1057100035170D08B0CB0C0837B500F50A517822C3
:105720002C31044650F02EF900220C2126484AF074
:1057300043FD2046FFF716FF0022B7EE000A0221C4
:1057400004F50B504AF0C0FD012504F505511F4A30
:1057500000950023103145204AF032FD1C4A1368A1
:10576000D90709D41B49156004F5035338330B607E
:1057700004F585530833CB6004F50C50154902221B
:10578000203001254AF06EFD134A0095002304F5F0
:105790007F61FD204AF014FD104B1A68D20705D432
:1057A0000F4A1D6004F58E54183414600C48012112
:1057B0004AF074FD4BF09EF90A4A138843F0010346
:1057C000138003B030BD00BF48170D08A4830E0836
:1057D000E484002000220020D8C90D08E8840020BD
:1057E000182200204C8700200F299DBF302303FB87
:1057F0000100503000207047014B93F9F3027047CD
:10580000804C0020024B93F8050100F00100704726
:10581000805C0020044BB3F8B832DB075ABF006944
:10582000C0F3401000207047804C0020014BD3F89B
:10583000E00C7047804C002008B503689B689847CF
:1058400030B9044B93F90401B0FA80F0400908BD67
:105850000020FCE7805C002038B50D1E2DDB174CC6
:1058600094F8EC2CEBB29A4227D3D4F8E83C01220E
:10587000595DA4F5005004F0E3F8F0B15DF03CF898
:1058800003215EF0AFF8C0B95DF036F80D215EF08F
:10589000A9F890B994F9D832EB40DB075CBF94F9D2
:1058A000F212E940A4F5005048BF0221BDE838409B
:1058B00058BF01F00101FCF7A1BC38BD804C0020AD
:1058C000022A10B50C4605D1BDE810400948352222
:1058D00004F0B6B8084BD3F8EC0003681B6898478F
:1058E000A04205D15DF008F8BDE810405CF08EBF25
:1058F00010BD00BF802C0020805C002029B102294F
:1059000007D1044BC3F8E4107047024B0122C3F8DF
:10591000E4207047805C002031B1022907D1044B9C
:10592000012283F8E8207047014B83F8E8107047A4
:10593000805C002010B500F50053DFED186AD3F845
:10594000D82CD3F8D43CB2F90820B3F908309FED35
:10595000147A07EE902AF8EEE77A0446C7EEA60A14
:1059600000F595500121103007EE903AF8EEE77AF5
:1059700060EE870A87EEA60A20EE070A11F00AFCFD
:1059800052F0E2FA262152F01BFA04F53A50054A89
:10599000BDE810400621383054F0D2BB0000C842A8
:1059A00035FA8E3C5C220D0800F58042002382F817
:1059B000383D044A00F53A5013720621024A383045
:1059C00054F0BEBBBD86002068220D0870B500F5FE
:1059D0008045044695F8381D002957D02C4B2D4A98
:1059E000D3F8EC00904204D1D3F8103193F8CB30C7
:1059F00023B92046BDE87040FFF7D6BF264E95F884
:105A0000390D04F54053012293F9E0303272D0BBD6
:105A1000002B3BDB85F8392D0139C9B204F5005361
:105A200085F8381DD3F8D82CD3F8D43CB2F9082027
:105A3000DFED1A6AB3F908309FED197A07EE902A64
:105A4000F8EEE77AB1FA81F1C7EEA60A04F59550AF
:105A50004909103007EE903AF8EEE77A60EE870ACF
:105A600087EEA60A20EE070A11F094FB95F8383D60
:105A700063B904F53A5033720A4ABDE87040062112
:105A8000383054F05DBB002BC6DAB2E770BD00BF02
:105A9000805C0020E4820020BD86002000007A4562
:105AA00035FA8E3C7C220D086D2900F3E380012934
:105AB00001DC5DF0C1BD8B1E6B2BFAD80FF2040C1C
:105AC0005CF823F0D35C0108CD5C0108D35C0108CD
:105AD000D35C0108B35A0108D35C0108B35A01082A
:105AE000B35A0108CD5C0108B35A0108D35C010820
:105AF000CD5C0108CD5C0108B35A0108D35C0108F4
:105B0000D35C0108D35C0108B35A0108B35A0108F9
:105B1000CD5C0108D35C0108CD5C0108B35A0108D3
:105B2000CD5C0108CD5C0108B35A0108B35A0108E5
:105B3000B35A0108B35A0108B35A0108CD5C0108F1
:105B4000D35C0108B35A0108B35A0108B35A0108DB
:105B5000D35C0108B35A0108CD5C0108B35A0108AF
:105B6000B35A0108D35C0108CD5C0108B35A01089F
:105B7000B35A0108B35A0108D35C0108D35C010889
:105B8000D35C0108B35A0108B35A0108D35C010879
:105B9000B35A0108B35A0108D35C0108D35C010869
:105BA000D35C0108B35A0108B35A0108D35C010859
:105BB000D35C0108B35A0108B35A0108B35A01086B
:105BC000B35A0108B35A0108B35A0108D35C01085B
:105BD000D35C0108D35C0108D35C0108D35C0108E5
:105BE000D35C0108B35A0108CD5C0108CD5C010803
:105BF000B35A0108B35A0108B35A0108B35A01084D
:105C0000B35A0108B35A0108D35C0108CD5C0108FE
:105C1000B35A0108B35A0108B35A0108B35A01082C
:105C2000B35A0108B35A0108B35A0108B35A01081C
:105C3000B35A0108B35A0108B35A0108B35A01080C
:105C4000B35A0108B35A0108D35C0108B35A0108DA
:105C5000B35A0108B35A0108B35A0108B35A0108EC
:105C6000B35A0108B35A0108B35A0108B35A0108DC
:105C7000CD5C0108A12921DC96297FF71AAFA1F19B
:105C800097030A2B3FF615AF0FF2040C5CF823F0D4
:105C9000D35C0108D35C0108B35A0108D35C010846
:105CA000B35A0108B35A0108B35A0108B35A01089C
:105CB000CD5C0108CD5C0108D35C0108B42908D093
:105CC000DB2903D0B2297FF4F4AE704700235DF0E6
:105CD00085BC704770B563298AB0034668DC01292A
:105CE00073DD881E612870D8DFE810F07C00840026
:105CF000940099006F00B3006F006F000C016F00FB
:105D00006F008B001F016F000A013C0143016F000F
:105D10006F004B01520159016F006A0173016F005E
:105D20006F006F006F006F007C0189016F006F00D2
:105D30006F008B016F006F006F006F008D016F00AF
:105D40006F006F006F006F006F006F006F006F00DB
:105D500095016F006F004501470149016F006F0019
:105D60006F006F006F006F006F006F006F006F00BB
:105D70008F0191019301970199019B016F00BC0173
:105D80009D016F006F006F006F006F006F006F006C
:105D900001026F006F006F006F006F006F006F00F7
:105DA0006F006F006F006F006F006F006F000D02DB
:105DB000B22900F068810EDC9A2900F0B0819F2999
:105DC00000F09D81982900F0A08118460AB0BDE836
:105DD00070405DF06FB9B42900F0C680DB29F4D1C2
:105DE000012433E0022AFBD135220E21B04803F012
:105DF00027FEF5E7111E18BF0121AD48FCF7FEF99B
:105E0000EEE7012A04D0022A14BF00210221F4E7A0
:105E10001146F2E706211846FFF752FDE0E7022A95
:105E2000DED1A44DD5F8EC000368DB6A9847044640
:105E30000028D5D0A5F58053D3F8DC3CB3F9083061
:105E4000002BCDD1A5F54050FFF774FD20460AB0D8
:105E500070BD022AC4D1974E974AD6F8EC109142F1
:105E6000BED0D6F8102192F8CB20002AB8D006F583
:105E70008054A6F58056B4F9F82F2AB9D6F8DC3C40
:105E8000B3F90830002BABD01C22002103A805ADCC
:105E9000B2F078FC284616F05FFFB4F9F83F93B9EA
:105EA0001623ADF80E30D4F8F43C8448642BB8BF08
:105EB000642303A906932CF085FD20B152F044F829
:105EC000272151F07DFF04F54F6494E80F0085E829
:105ED0000F00D6F8DC3C7948B3F90830002BCCBF72
:105EE0001023152303A9ADF80E302CF06BFD00280C
:105EF0003FF476AF52F028F8272151F061FF6FE7A9
:105F0000032188E7022A6E4D03D0002385F8F03C78
:105F100066E71921A5F596504BF0FAFD04460028D6
:105F2000F3D0012385F8F03C90E7012A0BD0022A38
:105F300011D0002A7FF454AF614B83F81C2352F038
:105F400003F82B21D9E75E4B019283F81C2351F013
:105F5000FBFF2C21D1E75A4B83F81C2351F0F4FFAF
:105F60002D21CAE70F2156E7564811468BF0C4FB96
:105F700036E709214FE704214DE705214BE71721BB
:105F800049E7901E414241414F4865F0E7F927E754
:105F9000022A7FF425AF464801F062FB20E7012A80
:105FA00006D0022A07D0002A7FF41AAF1146EBE789
:105FB00011460192E8E74448012165F0CFF9EAE78C
:105FC000424B911ED3F81C3D4A424A4183F820209F
:105FD00006E7931E594259413C4BD3F81C0D7EF005
:105FE0005FFEFDE6334B013A93F8E210012A8CBFC5
:105FF0000022012262F3041183F8E210F0E611217D
:1060000009E7122107E7152105E7002103E7102121
:1060100001E70221FFE60121FDE61621FBE607214B
:10602000F9E60B21F7E6022A284B0ED1012483F86A
:10603000E84E51F089FF4A2151F0C2FE5AF054FF58
:10604000234A062154F07CF800E7002283F8E82E6A
:1060500051F07AFF4B2151F0B3FE5AF045FF1D4A33
:10606000062121E0012A09D0022A0AD0002A7FF461
:10607000B7AE012118480DF02FFFB1E601920021C3
:10608000F8E71146F6E75AB3022A7FF4A9AE094BA6
:10609000D3F8EC0003689B6F984700287FF4A0AE0C
:1060A0005AF022FF0D4A042154F04AF898E600BF46
:1060B000802C0020805C0020087C0020447C002094
:1060C000804C00201C7E0020107B0020806C002073
:1060D00094220D08A5220D08005A0020B7220D08B1
:1060E000184BD3F8EC000368DB6F984778E6184646
:1060F0001146FFF703FC144804F054F870E611460B
:10610000FFF70AFC6CE61B2185E6022A7FF468AEE5
:106110000E48FCF76BFE5AF0E7FE0D4AA0E7114669
:106120005CF0B2FE0B487BF00DFC044600283FF407
:1061300057AE044A92F8E33043F0020382F8E330AA
:1061400084E600BF805C00208C7B0020802C002037
:10615000D0220D08785A002010B50446044883F078
:10616000B7FF04F10801BDE8104029F059BA00BF9B
:106170008079002038B504462DED028B114883F05C
:10618000ADFF05462BF0B6F90F48B0EE408A0DF092
:106190004FFF90B1DFED0D7AB4EEE78AF1EE10FA21
:1061A0000BDDD5ED000A95ED010AB0F0F5F8DFED55
:1061B000087A20EE270A84ED080ABDEC028B94EDE4
:1061C000080A38BD80790020802C002000401C4641
:1061D000E02E6542074B93F9D902022805D0032827
:1061E00006D0003818BF0120704781F001007047C9
:1061F00004207047804C002003688B4216D004298D
:10620000C0E9001302D007290ED07047084B9FED5C
:10621000097A03F59663D3ED007AF8EEE77A67EE34
:10622000877AC0ED087A704700238362704700BF09
:10623000803C00200AD7233C08B50246FFF7CAFF7E
:10624000BDE8084001461046FFF7D6BF70B52DEDFA
:10625000048B0446F0EE408AB0EE608A0D46164686
:106260008CF070FE9FED329ADFED329AE06176B3EA
:10627000236843B9304B03F59663D3ED007AF8EE0B
:10628000E77AC4ED097A68EE898A002DB7EE000A34
:10629000FFEE007AB8BFB0EE670A68EE808AC4ED00
:1062A000058A264BB4EEE98AF1EE10FAD3F81C0DFC
:1062B00030DA7DF0D3FC20EE090A84ED060ABDEC4D
:1062C000048B20460321BDE87040FFF795BF94ED95
:1062D000090A98EE890A28F041F9002D84ED050A93
:1062E0000BDAB4EEE90AF1EE10FADADBDFED147A3C
:1062F00030EE670A84ED050AD3E7D2D0DFED117ADC
:10630000B4EEE70AF1EE10FACBD8DFED0D7A30EEFD
:10631000270AEFE77DF0A2FCB4EE480AF1EE10FA8E
:1063200048BFB0EE408A28EE098A84ED068AC6E7A7
:106330000000C84200000034803C0020806C002037
:1063400000A00C47000000B410B52DED028B0446F0
:10635000B0EE608AF0EE408A8CF0F4FDDFED090AC1
:10636000E06168EEA08A68EE200AC4ED098ABDECFF
:10637000028BC4ED0A0A20460621BDE81040FFF753
:106380003BBF00BF0000C84210B52DED028B044694
:10639000B0EE408A8CF0D6FD94ED090ADFED097A63
:1063A000E061A8EE270A28F0C3F8BDEC028B0023B9
:1063B00084ED090AA36220460621BDE81040FFF7DC
:1063C0001BBF00BF0000C84270B54B68154D0646A4
:1063D0000C4673B98B6863B9C96851B91248FFF7A5
:1063E0002BFF95F8351E05F6BC50BDE870405FF0F8
:1063F00037BA95F8351E0D485FF0D2F848B906F166
:106400000801204616F038FE18B107480221FFF7B0
:10641000F3FE95F8351E05482246BDE870405FF052
:1064200013BA00BF806C0020EC8400203C7A00206E
:1064300008B50721FFF7E0FE80ED0A0A08BD00005D
:1064400008B50368032B23D1D0ED057A9FED127AAE
:10645000F0EEE77AF4EEC77AF1EE10FA1AD50F4BA8
:1064600090ED090A03F59663D3ED007AF8EEE77A2A
:1064700037EEC00A28F072F8DFED097AB0EEC00AF4
:10648000B4EEE70AF1EE10FA94BF0120002008BD37
:106490000120FCE70020FAE700000034803C0020E7
:1064A0000000484330B50368023B85B00446082B22
:1064B0006DD8DFE803F0050D30374B613F616100B7
:1064C000FFF74AFE84ED090A94ED090A05B030BDD4
:1064D0008CF038FDE369DFED310AE061C31A07EEA5
:1064E000903AF8EE677A94ED050A67EEA07AD4ED5B
:1064F000060AF12020EEA71A67EEE00A28F084F8D9
:10650000D4ED057A77EEC07AC4ED057AD4ED097A38
:1065100037EE800AD6E7FFF72DFEDFED217A20EE79
:10652000270ACFE71F4BD3ED4E7AF8EEE77AC0ED9E
:10653000097AC9E71C4DD5F8300D81F063FF0028BA
:10654000C2D0D5F8303D1B6B6362BDE78CF0FAFC1E
:10655000E3699FED127AD4ED0A6AE061C31A07EE8F
:10656000903AF8EE677A67EE877A94ED097AA6EEAC
:10657000A77A84ED097AA7E70B4B9FED0C0AD3F8B5
:106580001C0D6C302BF074FA84ED091A9CE7064B55
:10659000D3F8243DD3F84433D6E700BF6F12833AD3
:1065A0000000C842805C0020806C00209F0CB34536
:1065B0000368092B08D8DFE803F0050A050505057F
:1065C000070705100023836290ED0A0A7047044B09
:1065D000D3F8243DD3F84833F5E7C36AF3E700BFA7
:1065E000806C0020F8B50023214FCB6297F805316D
:1065F000204E13F0010F04460D462DD1D7F8EC00C4
:1066000003685B6F984738B3D7F8EC0003F0CEFB14
:10661000DFED197A85ED0B0AB0EEC00AB4EEE70A99
:10662000F1EE10FA03D409213046FFF7E5FD1148D9
:10663000FFF738FF0F4884ED000AFFF7B9FF336812
:1066400084ED010A0A2B0FD8DFE803F00C101010BC
:106650001010100C100C0C003368092BE7D1054802
:106660000021E2E70223A3602046F8BD0123FAE7F8
:10667000805C0020EC84002000000034034B0122E9
:106680001A6000229A60DA601A617047EC84002078
:1066900013B501A904460DF067FB04F5804320B94A
:1066A000012283F8652E02B010BDDDED017ADFED29
:1066B000096A03F65862B8EEE77AD2ED007A67EE1F
:1066C000A67AB4EEE77AF1EE10FA54BF0122002266
:1066D000E7E700BF0000C8422DE9F04F2DED068B23
:1066E00000F5005B00F595599BF92A338DB00546FE
:1066F00000F5804409F1100933B100F54058D8F88D
:10670000103193F8CB707FB90021A4F8DC1E484605
:1067100010F030FF94F8DD1E48460DB0BDEC068B3E
:10672000BDE8F04F10F030BF8CF00CFC0190D4F8B5
:10673000240D9FED948A90EDDBAA80F083F809AEDA
:10674000002800F0CA80D4F8243D03F55C7393E878
:10675000070086E8070030468DED0B8A2BF086FD9A
:10676000B0EE409A28460DF063FC05F59A4A0028E1
:1067700000F0B680504683F0B1FC07C886E80700F9
:1067800030468DED0B8A2BF071FDF0EE409AD8F873
:10679000EC0003681B689847122840F0AA80002389
:1067A00084F8DC3ED8F8EC0003685B69984728B1B0
:1067B000DBF8DC3CB3F90830002B0DDC98F9E03055
:1067C000002B09DA019BC4F8E03E504683F082FCBE
:1067D00004F6E46383ED000A94F8DC3E5BB1019BB0
:1067E000D4F8E00E181A41F28833984240F28F80B4
:1067F000002384F8DC3ED4F81C0D9FED630A6C3056
:106800002BF036F98DED090ACDED0A0A8DED0B1A44
:1068100096E8070006AB03AE9FED5C0A83E807002D
:1068200086E8070030462BF023F92846B0EE408A70
:10683000F0EE608A8DED060ACDED070A8DED081A9F
:106840000DF0F6FB002874D0DFED517AF4EEE79AF4
:10685000F1EE10FA94BF01250025D4F8240D7FF045
:10686000F1FF30B1DFED4A7AB4EEE79AF1EE10FABB
:1068700009D9002D64D1D8F8EC0003681B6898474B
:10688000022864D00027D4F8240D80F0FDF80546D6
:10689000002873D0B5EEC0AAF1EE10FA6DD5DFED89
:1068A0003D7AB4EEE7AAF1EE10FAACBF012600265D
:1068B000504683F01BFC5EB9DFED377AB0EEC00ABC
:1068C000B4EEE70AF1EE10FA5AD8002D08BF0027FF
:1068D00094F8DC1E84F8DD7E19E7B0EE489A41E7B3
:1068E00028460DF075FB00287FF444AFDFED259AB4
:1068F0004DE7D8F8103193F8CB30002B3FF452AF6E
:1069000098F9E030002BBFF64DAF012348E7504621
:1069100083F0E0FB04F6E463D3ED007A30EE670A1F
:10692000DFED1E7AB4EEE70AF1EE10FA3FF760AF42
:1069300061E728460DF04CFB0546002884D18CE722
:10694000D4F8240D7FF07EFF002894D19BE7B0EEB1
:10695000680AAFF0CFFAF0EE408AB0EE480AAFF026
:10696000C9FADFED0F7A20EE280AB4EEE70AF1EE5D
:1069700010FACCBF0127002785E700252E4697E7B0
:106980003746A5E7000000009F0CB345D302373916
:106990000000FA420000C8C20000704200004842F5
:1069A00055CF7D3F38B504460DF042FB04F59555B3
:1069B000103548B920460DF00BFB014620B928469A
:1069C000BDE8384010F022B804F54054D4F8EC008B
:1069D00003689B6C984720B9D4F8EC000368DB6C23
:1069E00098470146EBE7000030B5044689B0684699
:1069F00004F5955516F0B0F9103504A816F0ACF969
:106A00006946284610F0BCF898B104A9284610F051
:106A100007F970B1059B019323680022DB6C69467E
:106A20002046984728B104F52B5001211C3087F0EF
:106A3000B5FA09B030BD000000F5805292F82C255F
:106A4000D2070BD400F54052D2F8102192F8CB10A7
:106A500009B1FFF7C9BF03689B6C18477047000076
:106A600030B587B0044602A8019116F075F904F517
:106A7000955002A9103010F083F8019A18B900253A
:106A8000284607B030BD236802A9DB6C2046984732
:106A900005460028F3D004F52B5001211C3087F067
:106AA0007DFAEDE7F0B5044685B004F595566846E5
:106AB00010360F46154616F04FF96946304610F06D
:106AC000AFF810B9002005B0F0BD394630460FF0E0
:106AD0000FFF0028F6D0002DF5D004F5805428468D
:106AE00094F82C3543F0020384F82C35EBE70000D2
:106AF0002DE9F04F2DED0A8BBDB0044624220D4642
:106B000018A80021B1F03EFE2422002121A8B1F0F6
:106B100039FE242200212AA8B1F034FE04F54056A3
:106B20002422002133A8B1F02DFE0023CDE90D333E
:106B30000F9396F8E13013F0080839D104F50059A5
:106B400043F0080399F8D02C079286F8E13017F04B
:106B50005BFA90F9213003B390F84033EBB104F2C3
:106B60008457384617F060F9C34694F8A6355FFAA3
:106B70008BF18B421FD9384617F034F90BF1010B1A
:106B800082460028F1D1C94A0221284656F0CCFDA0
:106B900096F8E1306AF3C30308E0C54A02212846AB
:106BA00056F0C2FD96F8E1306FF3C30386F8E1308A
:106BB0004FF001083EE304F53753383301211846FE
:106BC0000BEE903AFAF7F6FF824608B9B94ADBE7CE
:106BD00020460CF04FFFD9F8DC3CB3F908A0BAF11D
:106BE000000F01D0B44AD9E796F9E030002B01DB61
:106BF000B24AC9E7204601F0AFFE04F544533C33E6
:106C0000184652460CA90CEE103A13F0CFF90028A2
:106C100014BF022301230393F123CDE9133A8F21FB
:106C20000A23CDE9003113AA287CADF854A0032330
:106C30004D2154F0B9FAA24B9FEDA28A01225A725B
:106C40000621A14A284656F06FFD039B022B0CBF7C
:106C50009E4A9F4A062128464FF0000A56F064FDDE
:106C600089F8E6A25146384617F028F894F8A63578
:106C70005FFA8AF18B420CD913AA38468DED138A3C
:106C80008DED148A8DED158A0AF1010A16F098FE31
:106C9000ECE7384617F0C8F84FF0000A4FF07C0BCD
:106CA00094F8A6255FFA8AF94A4519D94946384623
:106CB00016F078FDC0B20BFB00403CAA0C2300F29A
:106CC000146003FB092C07C8ACF1900C8CE807009A
:106CD0003CAA02EB890909ED2F8A0AF1010ADFE7D4
:106CE00041F288310AA823F073FFD6F810019FED16
:106CF000759A03689FED77AA9B6ADFED77AA98479C
:106D0000D6F81001012184F091F9744B1B680293AD
:106D1000D86A036801211B6898478CF013F9059025
:106D20008CF010F9F0EE499A0690002604F500590F
:106D3000079A99F8D03C934240F0D88094F8C6184E
:106D4000384617F04FF8002800F0D08004F5405B7B
:106D5000DBF8103193F8CB300493002B00F0C680A1
:106D600041F288310BA823F033FF8CF0EBF8059B40
:106D7000C01A132840F2D9808CF0E4F80590204620
:106D80000CF078FE5DF018FC82465DF0ABFBD9F8A4
:106D9000DC3CDBF81001B3F9083000EE103AB8EE35
:106DA000C00A20EE0A0A85F0B3FD50465DF0A2FB52
:106DB000384617F039F81CEE100A13F013FBD9F817
:106DC000DC3CDFED400AB3F9083000EE103AB8EED3
:106DD000C00AA22020EE0A0AB7EE001A27F014FC1F
:106DE000B4EEE90AF1EE10FA1CEE100A4FF00002C0
:106DF0000CA958BFF0EE409AF0EE408A13F0D6F896
:106E000008B900230C939DED0C8ADFED357AB4EEC2
:106E1000498AF1EE10FAF4EEE78A48BFB0EE498AEB
:106E2000F1EE10FA80F28F809FED2E9ADFED2E8A20
:106E30004FF0000A94F8A6355FFA8AFB5B4540F2F2
:106E400096814FF00C0918AB09FB0BF903EB090015
:106E5000B0EE490A2AF00CFE59463846CDED110A2B
:106E60008DED121A8DED100A16F09CFC7C23C0B239
:106E700003FB0040B0EE680A00F214602AF0F8FD4F
:106E80003CAB13A910A899448DED130ACDED140A5B
:106E90008DED151A2AF0C0FD0AF1010A09ED240A48
:106EA00049ED230A09ED221AC4E700BFCD240D08DD
:106EB000BC240D083F3B0D08DB240D08ED240D0814
:106EC000BD86002000000000F8240D080D250D08E7
:106ED000CFCD0C086F12833A0000C842E084002036
:106EE00000000034A4707D3F0AD7233C04F54059CC
:106EF000D9F8100103689B6A9847D9F8100100215E
:106F000084F094F8029BD86A036800211B689847B4
:106F1000002E40F05F812846C94A052156F004FC46
:106F20003146384616F0CAFE70E1029B986A036843
:106F300005215B6898470BA823F056FEB0EE498AFE
:106F4000B0EE489AF2E64FF000094FF00C0B04F552
:106F5000B86A94F8A6255FFA89F39A4222D91946AD
:106F60003846089316F01EFC089B0BFB03F13CAB64
:106F70005A18A2F16C034FF07C0CC0B2CDE9083274
:106F80000CFB00A018AB194454302AF05BFD089BA1
:106F9000099A09F1010902ED1B0AC3ED010A83ED0B
:106FA000021AD6E7039B012B4FF0000A46D19FED52
:106FB000A5BA9FEDA59A4FF00C0B94F8A6355FFA91
:106FC0008AF6B34240F286800BFB06F63CAB03EB3D
:106FD0000609A9F14803089321ABB0EE680A981995
:106FE0002AF056FD089B09ED120AC3ED010A83ED54
:106FF000021A33ABB0EE4B0A98192AF039FD2AABCE
:1070000098198DED100AB0EE490ACDED110A8DEDFB
:10701000121A2AF02DFD13A910A88DED130ACDED3B
:10702000140A8DED151A2AF00DFD0AF1010A09ED79
:10703000090A49ED080A09ED071ABEE79FED819A92
:107040009FED81BAF0EE088A94F8A6355FFA8AF9C6
:107050004B4564D99DED0C0AB4EEE80AF1EE10FA46
:1070600035DB0C2303FB09F93CAB03EB090621AB31
:1070700003EB09002AF00CFD33AB46ED110A06EDD7
:10708000101A06ED120A03EB0900B0EE490A2AF0C5
:10709000EFFC2AAB03EB09008DED100AB0EE4B0AB2
:1070A000CDED110A8DED121A2AF0E2FC13A910A8F9
:1070B0008DED130ACDED140A8DED151A2AF0C2FCE0
:1070C00006ED090A46ED080A06ED071A049E0AF1C4
:1070D000010AB9E74FF000094FF00C0A94F8A63501
:1070E0005FFA89F6B34241D933AB0AFB06302BF085
:1070F000BDF81BEE900AF0EE408A7AF01FFC07EE16
:10710000900AB8EE677A3CABC8EE877A03EB860646
:1071100009F1010967EEAA7A46ED2F7ADEE74FF012
:10712000000A4FF00C0B94F8A6355FFA8AF94B452C
:107130001DD933AB0BFB09302BF098F8C8EE297A38
:107140000AF1010A1BEE900A67EE808A7AF0F6FBDC
:1071500007EE900AB8EE677A3CABC8EE877A03EB8D
:10716000890967EEAA7A49ED2F7ADCE7049E8BF055
:10717000E9FE069BC01AB0F5FA7F27D98BF0E2FE34
:1071800004F50053DDED0D7AD3F8DC3C0C9A1B8935
:107190001392FCEEE77A339A1492ADF85C30349A8D
:1071A000159217EE903A359A1692ADF85E30F022AD
:1071B0001423CDE90032B121069013AA287C53F0A4
:1071C000F3FF74F0C5FB297C74F0B4FA0BA823F02C
:1071D0000BFDB5E60399384616F070FD00264FF01A
:1071E0000C0A94F8A635F1B28B4207D933AB0AFBEF
:1071F0000132384616F0E4FB0136F2E7384616F065
:10720000F1FB124A0621284656F08EFA104B002553
:1072100020465D7201F092FB04F50B50263049F0D8
:1072200039FB99F8E13065F3C30389F8E1300AA826
:1072300023F0DAFC40463DB0BDEC0A8BBDE8F08F90
:10724000A5D40E08A4707D3F0AD7233C15250D0850
:10725000BD860020F0B5534FD7F8983CDA0785B0CB
:10726000044600F19C8000F54055D5F8103193F8A4
:10727000C120002A40F0938093F8CB30002B00F01F
:107280008B8095F9E030002BC0F2868000F58046B7
:1072900096F8E83E002B40F08280D6F81C0D9FED5A
:1072A000420A6C302AF0E4FBCDED020A60EEA00A3F
:1072B000DFED3E7A8DED010AE0EE000A8DED031A56
:1072C000F4EEE70AF1EE10FA66DCD6F81C3D9FED0D
:1072D000387AD3ED377AF4EEC77AF1EE10FA04D5A6
:1072E000D5F810311B7A002B56D0B5EE007AF4EEAB
:1072F000C77AF1EE10FA4FD404F59A4082F0F6FE08
:10730000DFED2C7AB4EEE70AF1EE10FA44D8D6F8A5
:107310001C3D9FED297AD3ED367A67EE877AB3EE7E
:107320000E7AF4EEC77AF1EE10FA35DA234AB4F9A0
:10733000A410138801339BB2138019B9B4F8A210BA
:10734000A4F8A410B4F8A410994228D800261680F6
:1073500050F0FAFD0122192150F052FDD5F810012C
:1073600003685B699847431C04F53A50144A314658
:10737000383052F0E5FED5F81031012283F8C120F3
:10738000D7F8983C5B070AD504F58550083005B05E
:10739000BDE8F04068F0DEB8084B00221A8005B066
:1073A000F0BD00BF804C00209F0CB3454054094AFB
:1073B0006666663F000000B4E02E65422685002028
:1073C0002C250D0870B52DED028B4A4BD3F8983C57
:1073D0009B0784B004461FD400F58045DFED468A44
:1073E000D5F81C0D03681B699847D0ED017AF4EEBF
:1073F000E87AF1EE10FA0FDB04F5405304F59D46F0
:10740000D3F8102192F8C1106C3649B1002303A9BA
:107410003046039352F0CCF904B0BDEC028B70BD42
:1074200092F8CB20002AF1D093F9E030002BEDDB6D
:1074300095F8E83E002BE9D1D5F81C0D03681B69CF
:107440009847D0F8A430D5F81C0D039303681B6946
:10745000984704F58C7200F1A401304652F0A6FA68
:10746000DDED037AB0EEC08AF0EEE77AF4EEC87A8A
:10747000F1EE10FA03D503A9304652F099F9D5F888
:107480001C0D03681B699847D0ED040AF4EEE80A66
:10749000F1EE10FAC0DBF6EE087A60EEA77AF4EEB1
:1074A000C87AF1EE10FA1DD58BF04CFDD5F8F83EF8
:1074B00042F21072C31A9342AED9DFED107AC5F8CA
:1074C000F80E68EE277A04F53A5417EE900AF9F7A9
:1074D0001BF83834CDE90001094A0021204652F05A
:1074E0002FFE99E79DED030A26F08AFF0028DBD1E5
:1074F00092E700BF804C0020000000340000C8422A
:1075000048250D0810B5044600F59D40103063F085
:1075100037FF04F59D400121BDE8104030306CF08C
:10752000FBB90000F8B500F58045044695F9903E9A
:1075300043B300F5405695F8A42E96F8E030DB43AF
:10754000C3F3C01363F3C30285F8A42E00F59D476F
:1075500000F59A4082F0CAFDDFED3D7A103720EE4B
:10756000670A384663F08CFF95F8E83E53B9384611
:1075700063F032FFD6F8103193F8CB301BB9354B9E
:1075800000221A80F8BD95F8A43EDB07FAD4D6F89D
:10759000EC0003689B6B98470028F0D096F9E03028
:1075A000002BECDB2B4E33884BB9B5F9963E33B14B
:1075B000642213FB02F3D5F8F42C9A42E2DB38463E
:1075C00063F07AFFD5F81C3D9FED237AD3ED367A30
:1075D00067EE877AB3EE0E7AF4EEC77AF1EE10FA20
:1075E00005D83388002BCDD0013B3380CAE7B4F9EE
:1075F000A4301BB9B4F8A230A4F8A4303388B4F88E
:10760000A420B4F9A400154993423CBF0133338050
:107610003388D5F8CC2C012B01D10A60B2E7096878
:107620009142ACDD18B9B4F8A220A4F8A420B4F8B3
:10763000A4209A42A6D80023338050F085FC022271
:107640000C2150F0DDFB2046BDE8F840FFF75ABFA3
:107650000AD7233C24850020E02E654220850020A7
:1076600008B500F5804292F9903E6BB300F54053A7
:1076700093F9E030002B0EDA00F53A50134A062158
:10768000383052F05DFD50F05FFC0322BDE8084049
:107690000F2150F0B5BBB2F9963E8BB1D2F8F42C65
:1076A000642113FB01F39A420ADA00F53A50084AC2
:1076B0000121383052F044FD50F046FC0222E5E74B
:1076C000BDE80840FFF71EBF08BD00BF60250D08DC
:1076D00072250D08F0B52DED028B00F540555C4E7E
:1076E000D5F8103193F8CB308DB0044643B195F9FD
:1076F000E030002B04DB00F5005393F902332BB983
:10770000002333800DB0BDEC028BF0BD00F5804747
:1077100097F8E83E002BF3D101F084FB00287DD1DF
:10772000D5F8EC0003689B6B98470028E8D004F577
:107730009940503052F092F82AF098FDF0EE087A15
:10774000B4EEE70AF1EE10FAF0EE408AD8DA04F56A
:10775000805303F59F6203F2FC43D3ED007A92ED70
:10776000000A20EE270AAEF0AFFDDFED3A7A20EEF8
:10777000270AB2EE0E7AB4EEC70AF1EE10FABFD9BC
:10778000D7F81C3D93ED368A28EE278AF3EE0E7A61
:10779000B4EEE78AF1EE10FAB2D904F59550002361
:1077A00009A9103009930A930B930FF045FA0028AA
:1077B0003DD13388B4F9A42001339BB23380002A31
:1077C00040D0B4F8A420B3EB420F9BDB50F0BCFBDD
:1077D00001220C2150F014FB1F4B002218EE900ADE
:1077E000CDE90623F8F790FE1C4BCDE904010022F9
:1077F00018EE100ACDE90223F8F786FE04F53A5494
:107800003834CDE90001164A2046002152F098FC98
:1078100001220C211348FAF7E5FB73E7D5F8EC00D9
:107820000368DB6C984700287FF47AAF68E709A803
:107830002AF01CFDF2EE047AB4EEE70AF1EE10FA3B
:10784000B7DB5DE7B4F8A220A4F8A420B9E700BF35
:107850001C850020E02E65420000084000003E40EC
:1078600088250D08785A0020F0B52DED028B8BB0DD
:10787000002307930893099305AB0446019300F591
:10788000955007AB009302AA04AB03A910300FF088
:10789000EBF804F50056054686F8AC0E28B900252D
:1078A00028460BB0BDEC028BF0BD8BF03FFBD6F849
:1078B000B03E9FED327AC31A07EE903AF8EE677A3F
:1078C000074667EE877A04F53A5006AA02A90830FF
:1078D000CDED067A52F06AF804F53A5006AA03A9EB
:1078E00014308DED020A52F061F804F53A5006AA00
:1078F00004A920308DED030A52F058F896EDC18AA4
:10790000C6F8B07EB5EEC08AF1EE10FAC7D9DDED4B
:10791000080A9DED070AAEF073FBDDED090AAEF033
:107920006FFBD6F8302EDDED037AB4EEC08AF1EEAF
:1079300010FA94BF012300231AB196F8342ED2070F
:1079400012D438EE087AB4EEE77AF1EE10FA0BD8DA
:107950000233DBB2DDED027AB4EEE78AF1EE10FA23
:1079600009D8002B9BD09BE7B4EEE78AF1EE10FA22
:10797000F0D80133EDE7012B92D890E7BD3786357B
:1079800070B500F54055044695F8053143F0040301
:1079900085F8053150F0D8FA0122112150F030FA63
:1079A000D5F8103193F8CB30002B43D0D5F8EC004C
:1079B00003681B68984709280AD1204608F01CFE76
:1079C00030B104F5A9404030BDE8704008F0FCBD7E
:1079D000194BD3F8EC0003681B69984704F5005372
:1079E00040B993F90133032B24D10621204608F036
:1079F000EFFD0DE093F901130229F6D195F8053159
:107A0000DB07F2D40622204602F01AF80028ECD058
:107A10000A4BD5F8EC0001225A7303681B6C984797
:107A2000034604F53A50064ABDE87040022138305A
:107A300052F086BB70BD00BF805C0020BD86002078
:107A4000BC250D0808B500F5405292F805315907DC
:107A500017D56FF3820382F805310A4B5A7B42B186
:107A6000002200F53A505A730221074A383052F08A
:107A700067FB50F069FABDE808400022112150F080
:107A8000BFB908BDBD860020E0250D08F0B505464C
:107A900085B005F595576846103715F05DF96946CC
:107AA00038460FF0BDF880B105F50053D3EDC17A2B
:107AB000374CF5EEC07AF1EE10FA08D8354A0023BB
:107AC00028462380D373FFF7BDFF05B0F0BD2846DD
:107AD000FFF7CAFE064628460CF07AFA10B9284687
:107AE0000CF052FAA378002E18BF00200343DBB23B
:107AF000A370002BE9D06378A8BB83BB2378013344
:107B0000DBB2082B237003D14EB338460FF018F8C0
:107B10002378092B02D138460FF00AF82378092B75
:107B20001DD94FF48573238050F00EFA02221021E4
:107B300050F066F98BF006FA6368C01A47F23053CA
:107B4000984209D905F53A50134A0221383052F0CB
:107B5000F7FA8BF0F7F960602846FFF711FF0D4B3D
:107B60006278DA73B1E72678002EF8D0013EF6B2DB
:107B70002670002BF3D0002EF1D1667050F0E4F99E
:107B80003246102150F03CF92846FFF75BFFE6E74C
:107B900028850020BD860020F8250D0800F54053FB
:107BA00093F805315B0701D5FFF7EABE7047000087
:107BB00073B5044600F5955001A9103004F5005541
:107BC0000EF09CFDD5F8743E834206460CD004F5B9
:107BD0008043D3F81C0D7DF005FCC5F8746E50F0A1
:107BE000B3F93E2150F0ECF804F5805695F9781E73
:107BF00096F9C02596F8C03591421BD0FF2B19D0BD
:107C000004F58043D3F81C0D7DF0ECFB96F8C035ED
:107C100085F8783E50F098F995F8782E182150F0B4
:107C2000EFF804F53A5095F9783E034A04213830CC
:107C300052F086FA02B070BD08260D082DE9F04317
:107C40008FB005468BF07EF90023059306930793CA
:107C5000089309930A930B930C930D9305F595588C
:107C600004AB019308F1100803AB009306460BAB7D
:107C700008AA05A940460EF0D7FEDFED487A9DED33
:107C8000077AB4EEE77AF1EE10FA074632DB9DEDA3
:107C90000A7AB4EEE77AF1EE10FAACBF01240024C0
:107CA00005F50059404699F8AC3E002B08BF002767
:107CB0000EF0CCFE8046FFB9444699F9343C012BC6
:107CC0002BD174B105F54053D3F8102192F8CB4075
:107CD0003CB1D3F8EC0003685B69984780F0010081
:107CE000C4B299F87C3ECBBBCCB9C9F8806E0FB05A
:107CF000BDE8F0830024D3E7002CDDD005F53A5031
:107D0000143051F053FD90ED007AF7EE007AB4EEA6
:107D1000E77AF1EE10FAD0DCCEE70024E1E7D9F8FB
:107D2000800E301AB0F57A7FE1D9C9F8843E01247B
:107D300005F5804389F87C4ED3F8243D83F80C4444
:107D400050F002F922461D2150F05AF8144A05F568
:107D50003A500221383052F0F3F9C8E714B1C9F8AB
:107D6000846EC4E7D9F8840E43F69823361A9E42EF
:107D7000BDD905F58043C9F8804E89F87C4ED3F80B
:107D8000243D83F80C44C9F8844E50F0DDF82246B7
:107D90001D2150F035F8034AD9E700BF0000003438
:107DA00020260D083A260D080B4B10B5012204467B
:107DB0005A728BF0C7F804F58042D2F8D43EC31A49
:107DC000142B07D9C2F8D40E04F59350BDE8104027
:107DD00044F03EBF10BD00BFBD8600202DE9F74333
:107DE000044604F5405600F50B5000233C300DF1DD
:107DF00007018DF8073049F0BBFAD6F8100190F969
:107E0000C030026883B3083BDBB2012B95692BD9E4
:107E10003221A84704F1100012F05EFC204B04F55B
:107E20003A581F684FF0000908F13808F86A0368EB
:107E3000DB69984701281ED18BF084F841F2873323
:107E4000A0EB09029A42054605D9164A062140468A
:107E500052F076F9A9462046FFF7A6FFB86A0368F4
:107E600003215B689847E1E704F500539269B3F892
:107E700010139047CEE70121D6F8100183F0D6F811
:107E8000D6F810010368DB6A98475BF093FFF86A45
:107E900003681B68012103B0BDE8F043184700BF29
:107EA000E084002058260D0870B5044600F53A50CD
:107EB0002DED028B184A194E9FED198A0621383094
:107EC00052F03EF92046FFF789FF2046FFF76CFF8E
:107ED00020460BF0CFFD3368986A036803215B6886
:107EE00098475CF069FB05465CF0FCFA04F500532A
:107EF000D3F8DC3CB3F9083000EE103A04F54053F7
:107F0000B8EEC00AD3F8100120EE080A84F000FD94
:107F100028465CF0EFFAD8E77C260D08E0840020C4
:107F20006F12833A2DE9F047044600F53A502DEDE3
:107F3000028B2A4ADFF8AC900621383052F000F963
:107F40002046FFF74BFF5CF037FB04F54056054633
:107F50005CF0C8FAB7EE000AD6F8100184F0D8FC3D
:107F600028465CF0C7FA8AF0EDFF41F2873A0746EF
:107F70008AF0E8FFC01B5045D9F8008017D99FED63
:107F8000188A28465CF0AEFAB0EE480AD6F810011E
:107F900084F0BEFC28465CF0ADFA2046FFF704FFF3
:107FA000D8F82800036803215B689847E9E728466A
:107FB0005CF098FAB7EE000AD6F8100184F0A8FC3D
:107FC00028465CF097FA2046FFF7EEFED8F8280026
:107FD000036803215B689847CAE700BFAC260D0819
:107FE00000000000E0840020F7B500F5405304468F
:107FF000D3F8103193F9C030032B2BD0364E6525C2
:1080000000F58047013D15F0FF050CD0D7F8D03EB4
:108010004BB93368986A036814215B689847204617
:108020000BF028FDEEE704F5375001213830F9F761
:10803000C1FD04F5005378B993F9FC3253B1092B13
:1080400008D08DF8070004F50B500DF107013C3006
:1080500049F08EF903B0F0BD93F9FC22032A34D81D
:10806000DFE802F002252D30D3F8DC3CB3F908201C
:1080700040F2B5339A422ADD04F50B5001250DF18B
:1080800007013C308DF8075049F072F904F53A5079
:10809000124A0221383052F053F8114B5D720E4BE8
:1080A0001C68A06A036805215B689847F9E7D3F864
:1080B000DC3CB3F9082040F2B5339A4207DD204694
:1080C000FFF7F2FE2046FFF72DFF092AC2D000235A
:1080D0008DF80730B7E700BFE0840020D0260D08F8
:1080E000BD86002000F53A500B46024A0421383084
:1080F00052F026B8F0260D0810B504464FF024FFC4
:10810000002205214FF07CFE04F53A50034ABDE8F9
:1081100010400421383052F013B800BFFC260D087F
:1081200013B50B464AB100F53A5000920421054AB6
:10813000383052F005F802B010BD02B0BDE8104072
:10814000FFF7D0BF14270D0808B500F53A50064ACE
:108150000421383051F0F4FF4FF0F6FEBDE808403E
:10816000002208214FF04CBE28270D0838B50446E0
:108170000D468AF0E7FE04F540533DB9D3F8FC20E4
:10818000C3F800010AB9C3F8FC0038BDD3F80021D8
:10819000801A642884BF0022C3E93F22F5E700006B
:1081A00037B5044600F59A4081F086FF04F5405249
:1081B000C0F3803592F8E230C3F34001A9421DD0EC
:1081C00065F3410304F53A5482F8E23038346DB176
:1081D0004FF0BAFE02220B214FF012FE084A022194
:1081E000204603B0BDE8304051F0AABF4FF0ACFECE
:1081F0002A460B214FF004FE024AF0E703B030BDDF
:1082000040270D085C270D0838B50A460C460621A4
:10821000054601F015FC28B1054A137843F0080320
:10822000137038BD21462846BDE8384008F0D0B963
:10823000DC86002038B50A460D461521044601F0BB
:10824000FFFB28B1094A137843F00803137038BDC7
:1082500004F53A5004213830054A51F071FF29469F
:108260002046BDE8384008F0B3B900BFDC860020E6
:108270006C270D0838B50A460D461521044601F055
:10828000DFFB28B1094A137843F00803137038BDA7
:1082900004F53A5004213830054A51F051FF29467F
:1082A0002046BDE83840FFF7AFBF00BFDC860020A6
:1082B00094270D0838B50A460D461B21044601F0E7
:1082C000BFFB28B1094A137843F00803137038BD87
:1082D00004F53A5004213830054A51F031FF29465F
:1082E0002046BDE83840FFF78FBF00BFDC86002086
:1082F000AA270D0838B50A460D461121044601F09B
:108300009FFB28B1094A137843F00803137038BD66
:1083100004F53A5004213830054A51F011FF29463E
:108320002046BDE8384008F053B900BFDC86002085
:10833000BC270D0810B500F5405494F8E2309A06B9
:1083400023D4D4F8EC0003681B689847032808D0AE
:1083500005D802280ED194F8E000C00914E01B28CB
:10836000F9D194F8E00000F0A000A0F18003584299
:10837000584109E0B4F8E00020F4FE4020F07F000E
:1083800080B2003818BF012010BD0120FCE70000BA
:1083900038B500F54055044695F80531184A43F0C4
:1083A000080300F53A5085F805310221383051F0C4
:1083B000C7FE4FF0C9FD012217214FF021FD2046D5
:1083C000FFF7B8FF40B104F537500122BDE838404F
:1083D00015213830F9F706BED5F8EC0003681B68A4
:1083E0009847062806D104F5AB405830BDE8384020
:1083F00009F0FABA20460B21BDE83840FFF704BF68
:10840000D0270D0870B500F54055D5E93F239B1ADC
:1084100041F288329342064611D9D5F8EC00036840
:108420001B6D9847044695F80531C3F3C003A3427A
:1084300013D034B13046BDE87040FFF7A9BF002427
:10844000F1E74FF081FD224617214FF0D9FC95F856
:10845000053164F3C30385F8053170BD0B4610B5D3
:1084600011460446072B07D8DFE803F02A04131649
:10847000191C242708F0ACF804F50053D3F8383C55
:108480009B061DD504F585500830BDE8104067F007
:1084900061B8FFF7B9FEEFE7FFF7ECFEECE7FFF797
:1084A000C9FEE9E700F53750012214213830F9F709
:1084B00099FDE1E7FFF7FEFEDEE7FFF71BFFDBE7D5
:1084C00010BD0000F8B5044604F500574FF03CFD20
:1084D000012205214FF094FC97F8E632072B98BF54
:1084E000304A204694BFD55C0125FFF723FF68B1D1
:1084F0002D4A2E492046FFF713FE04F5375001227E
:1085000010213830F9F76EFD002514E004F54056CF
:10851000D6F8EC000368DB6C984798B196F8AD3656
:1085200083B196F9AC36012B0CDC214A2149204657
:10853000FFF7F6FD0125294620460322BDE8F84055
:10854000FFF78CBFD6F8EC000368DB6C984718B1D6
:10855000D7F8383C190715D4D6F8EC0003681B6827
:108560009847032803D1D7F8383CDA070DD4D6F85A
:10857000EC0003685B6A984768B90C492046FFF72E
:10858000B1FDD8E70A4A0949D1E70B4A0749204615
:10859000FFF7C6FDB8E7D7F8383C5B07EDD5074ACB
:1085A000F4E700BFB0280D08F0270D081AF80D08F1
:1085B000FA270D080D280D081D280D082D280D0877
:1085C00038B5044615464FF0BFFC012206214FF096
:1085D00017FC2046FFF7AEFE98B104F53750012294
:1085E00007213830F9F7FEFC144A15492046FFF7F9
:1085F00097FD0025294620460422BDE83840FFF7B4
:108600002DBF04F54053EDB2D3F8EC000368DB6CEA
:10861000984768B104F50053D3F8383C1B0707D5D9
:1086200035B1084A06492046FFF77AFD0125E1E702
:1086300003492046FFF756FDDCE700BFF0270D0891
:108640004A280D08FA270D082DE9F041044604F5E3
:1086500000574FF079FC012208214FF0D1FB5AF06E
:108660004BF897F8D532072B98BF384A04F5405697
:1086700098BFD55CD6F8103193F8CB8088BF02251F
:10868000B8F1000F0BD132492046FFF72BFD002532
:10869000294620460522BDE8F041FFF7DFBE20460F
:1086A000FFF748FE60B104F537500122122138303F
:1086B000F9F798FC274A26492046FFF731FDE6E7FF
:1086C000D6F8EC000368DB6C984768B196F8AD36D5
:1086D00053B196F9AC36012B06DC1F4A1F492046E0
:1086E000FFF71EFD0125D3E7D6F8EC000368DB6C2D
:1086F000984718B1D7F8383C190713D4D6F8EC00CE
:1087000003681B689847032803D1D7F8383C9A07B9
:108710000BD4D7F8383CDB0609D40D492046FFF7C7
:10872000E1FCB5E70C4A0A49D9E70D4AC3E7D6F898
:10873000EC000368DB69984706460028EDD1094A3A
:1087400003492046FFF7ECFC3546A1E7B8280D08A1
:10875000F1130D08F0270D08FA270D0844280D081D
:1087600052280D0867280D08F8B500F50055044695
:1087700095F9D532B3B300F54056376F97B38AF009
:10878000E1FB05F5496595ED000ADFED177A9FEDF0
:10879000171ADFED170AC71B20EE270A8D2025F0D8
:1087A00033FFBCEEC00A10EE103A9F420CD296F88E
:1087B00005319A0716D520460021F9F76DFD2046B0
:1087C000BDE8F840FFF7C0BC0CD996F805319B070F
:1087D00008D420460121F9F75FFD2046BDE8F840A6
:1087E000FFF732BFF8BD00BF00007A440000804FA1
:1087F000000000002DE9F341074600F59A4081F0A2
:108800005BFC07F54054C0F3804801908AF09AFB66
:1088100094F808314345454606460DD007F53A50D1
:1088200084F808813830002D41D03C4B3C4AC4F8D4
:108830000C61022151F084FC94F8083107F50058CE
:1088400043B394F809312BBBB8F9A63C9FED350A28
:108850009FED351ADFED350A07EE903AF8EEE77A2C
:1088600040F2571027EE800A25F0CEFEBCEEC00A7B
:10887000D4F80C0110EE103A361A9E420AD90123A0
:1088800007F53A5084F80931294A244B022138303F
:1088900051F056FC98F9A53C002B94F805310DDCFD
:1088A0006FF3451384F8053102B0BDE8F0811B4B2E
:1088B000204AC4F80C8184F80981BAE7C3F3401256
:1088C000AA42F1D065F3451384F805319B06EBD538
:1088D000194BD3F8EC0003681B6998470028E3D0D4
:1088E0004FF032FB01221F214FF08AFA3846FFF782
:1088F00021FD48B107F5375001222121383002B05F
:10890000BDE8F041F9F76EBB98F8A51C3222384655
:1089100002B0BDE8F041FFF7A1BD00BF80280D08FF
:108920008F280D0800007A440000804F00000000EE
:10893000A5280D089A280D08805C002008B5044B76
:1089400001221A708AF0F2FA024B186008BD00BFCB
:108950003185002034850020014B00221A707047B9
:10896000318500202DE9F04104468AF0DFFA2A4BD8
:10897000B4F8BE201988294E914205460ED01A80BF
:10898000274B18603378A3B1002434704FF0DCFA21
:1089900022461321BDE8F0414FF032BA3378214F1F
:1089A000DBB93B782BB11E4B1F4A1B68C31A93429D
:1089B00001D8BDE8F0810123337004F54053D3F8AA
:1089C000100190F8CB3013B103689B6A98474FF0C1
:1089D000BBFA012213214FF013FA3B78002BE8D0A9
:1089E0003378002BE5D00E4A10491368EB1A8B42FE
:1089F000DFD904F540541560D4F8100190F8CB305D
:108A0000002BD6D0002182F011FBD4F810010368AE
:108A1000BDE8F0415B6A18473285002030850020B0
:108A2000348500203185002080841E0040420F00E4
:108A30002DE9F84300F5405500F500580446D5F8F7
:108A4000EC0098F88C710368DB6C9847014650B9CC
:108A500095F9E030002BA5BFD5F8103193F8CB0085
:108A6000012180F0010104F5055909F1100948467A
:108A700067F078FDD5F8103193F8CB300646002B1F
:108A80007BD0002865D03E4B93F9E030002B04DB0F
:108A900002463C49484667F03FF998F9567157B18C
:108AA00095F9E030002B0EDA04F5375001220F2142
:108AB0003830F9F797FA4FF047FA3246BDE8F843F5
:108AC00009214FF09DB9D5F8EC0003685B69984720
:108AD00058B195F9E130002B07DA95F80531DA073E
:108AE00003D498F88C31DB07DED53146484667F071
:108AF0009FFDDFED257AB4EEE70AF1EE10FA05DD11
:108B00000A220921204600F09BFFD4E7023F032FF1
:108B100011D801A353F827F0018B0108298B010814
:108B2000478B01084D8B01080A221521204600F0D1
:108B300087FF0028BFD10A220621204600F080FFCF
:108B40000028B8D1DCE70A221121F6E70A22152114
:108B5000F3E797B198F88C317BB9094B93F9E03082
:108B6000002B06DB04F53A50084A0521383051F055
:108B7000E7FA4FF0E9F90022A0E7BDE8F88300BF6B
:108B8000805C0020C0280D080000C842C9280D08DC
:108B900070B500F5005300F59A4586B093F87C1E39
:108BA0000446284681F036FA02A814F0D5F804F5F8
:108BB000955002A910300DF0E3FF04F58043049AAC
:108BC000C3F8F82C059AC3F8FC2C284681F074FAF7
:108BD00082061AD5284681F07DFA04F59945FDEE06
:108BE000C07A703504F5805417EE901A0222284698
:108BF00017EE906A14F0B6F894F82C35DB0706D41B
:108C000001223146284614F0ADF806B070BD0121AE
:108C1000284614F039F90028F2D0F6E770B500F5CF
:108C2000804486B0B4F8043F8B420D46164603D10B
:108C3000D4F8003F934221D08AF084F9D4F8FC3E66
:108C4000C31A132B1AD9C4F8006FA4F8045FC4F830
:108C5000FC0E4FF079F904468AF07CF9084B094A7A
:108C60001B68CDE90453084B0193084B0093CDE9F1
:108C70000201074B074920464EF0F2FE06B070BDD8
:108C800038850020E0280D08F8280D0870FE0C0833
:108C9000ACE10C08F3280D0838B500F540540D463A
:108CA00094F8E130C3F380138B420BD021B14FF025
:108CB0004BF911214FF084F894F8E13065F38613F5
:108CC00084F8E13038BD0000F0B52DED048B00F5DF
:108CD00040568BB0D6F8103193F8CB30054600F5EE
:108CE0008044002B67D096F9E030002B63DBD6F888
:108CF000EC0003685B699847002861D1D4F81C0D2B
:108D00009FED440A6C3028F0B3FE0AAACDED080AA4
:108D10008DED091A8DED070A12E9070004AB01AFCA
:108D200083E8070087E80700384628F0EDFBD4F811
:108D30001C3D05F599405030D3ED368AB0EE409A8F
:108D400050F08CFD29F092FAD4F8243DD6F8EC00CE
:108D5000D3EDDB9A0368DB6CB0EE408A9847DFED19
:108D60002E7AB4EEE79AF1EE10FA02DC96F8E830CB
:108D70000BB100283AD0DFED297A68EEA78AF3EE2E
:108D80000E7AF4EEE78AF1EE10FA2FDCF0EE087AB4
:108D9000B4EEE78AF1EE10FA28DCF5EEC09AF1EEB7
:108DA00010FA23DAD4F81C0D03689B6F98470BB0B8
:108DB000BDEC048BF0BDD4F81C0D03689B6F0FE075
:108DC00005F50055D4F81C0DD5F8DC2C0368B2F974
:108DD0000820002A03DCD6F8E420022AEED1DB6F5B
:108DE0000BB0BDEC048BBDE8F0401847D4F81C5D17
:108DF000DFED0B0A2B68D3F88060D4F8243D40F2F5
:108E0000AB1093EDC90AB7EE001A25F0FDFB28461A
:108E1000B047CCE79F0CB3450080BB44E02E6542D1
:108E20000000000000F5405090F8E8007047000096
:108E30002DE9F04100F54055064695F8E030B1EBDC
:108E4000D31F0C4648D0254B00221A6000293FD082
:108E50004FF07AF812214EF0B3FF95F8E03064F34A
:108E6000C71385F8E03084F0010872F0B1FE414686
:108E700072F08AFE06F50057B8F1000F06D097F899
:108E80006A321BB98AF05EF8C7F86C0287F86A820A
:108E900014B3B7F8B8325B071ED5D5F8103193F884
:108EA000CB30CBB1D5F8EC0003685B69984798B933
:108EB000D5F8EC00036820219B69984760B106F55E
:108EC00037500122BDE8F0410D213830F9F78AB85A
:108ED0004FF03AF81C21BEE7BDE8F081388500204C
:108EE0002DE9F04F2DED0A8B00F540558DB0D5F8EA
:108EF000103193F8CB60044600F580471EB901217C
:108F0000FFF796FF0BE095F9E020002A65DAD5F827
:108F1000EC0003689B6C98470646002841D04FF050
:108F2000000B95F9E020B14E002AC0F25381D6ED36
:108F3000007AB4F9A420B8EE677A1AB9B4F8A2207E
:108F4000A4F8A420B4F8A430DFEDA96A07EE903AA3
:108F5000F8EEE77A67EEA67AB4EEE77AF1EE10FA69
:108F6000ACBF012100212046FFF796FE95F9E020D5
:108F7000002A95F8E120B8BF4BF0010B530697F893
:108F8000E82E48BF4BF0020B0AB14BF0080B3268D9
:108F9000594620460DB0BDEC0A8BBDE8F04FFFF7F7
:108FA0003DBED5F81031204693ED0C8AF9F744FA0E
:108FB000B4EEC80AF1EE10FAB1D5D5F8103193F835
:108FC000A130032BABD14DF0CBFA4FF480114222EC
:108FD0004DF07EFA3146204692E797F8E8AEBAF1B6
:108FE000000F03D0814A0023136098E7D7F81C0DC7
:108FF00093F8079003685B6F984780460090D5F818
:10900000EC0003685B69984720B1D5F8E430022B87
:1090100000F0E280B9F1000F0CBF4FF0000B4FF4ED
:10902000007BB7EE00BAB8F1000F02D04BF4806BB2
:10903000009604F59D4808F1300840466AF08CFC23
:109040000130D7F81C0D9FED6B0A9FED6BCADFED69
:109050006B8A0CBF012302236C3008EE103A28F013
:1090600007FD0CABCDED0A0A8DED0B1A8DED090A4B
:1090700013E907000DF10C0E0DF1180C8CE8070038
:109080008EE80700704628F03FFAD7F81C2DDFED78
:109090005C7A92ED36AA2AEE27AAB4EECC0AF3EE59
:1090A0000EBAF1EE10FA04F59940B4EEEBAAC8BF7F
:1090B0004BF4807B5030F1EE10FAC8BF4BF4807B4C
:1090C000F0EE40AA50F0CAFB29F0D0F8B8EEC88AFA
:1090D00004F59A40B4EEC80AF1EE10FA98BF4BF0CE
:1090E000800BF0EE409A81F001F868EE288AB0EE2D
:1090F000C09AB4EEE89AF1EE10FA204648BF4BF061
:10910000400B0AF0A1FD002846D14BF0200B019640
:1091100040466AF021FC01284FD14BF0100BB246BB
:109120003249B9F1000F53D0009B002B50D0F4EE20
:10913000CCAAF1EE10FA4BDCB4EEEBAAF1EE10FA89
:1091400046DCF4EEC89AF1EE10FA41D8B4EEE89A93
:10915000F1EE10FA3CD5019BD3B3BAF1000F37D032
:109160000A68B4F9A40007EE902AB8EE677A18B935
:10917000B4F8A200A4F8A400B4F8A43007EE903A22
:10918000F8EEE77A67EE8B7AB4EEE77AF1EE10FA52
:1091900019D501320A60C4E604F53350383050F076
:1091A00005FBDFED187A90ED007AB4EEE77AF1EE88
:1091B00010FAAAD400230193AAE740466AF0CCFB38
:1091C0000130ADD1A9E701212046FFF731FEA8E625
:1091D0000022DFE70121C6E6B9F1000FB0EE08BAC0
:1091E0000CBF4FF0000B4FF4007B1FE738850020C9
:1091F000CDCC4C3E9F0CB3450080BB440000C84220
:10920000E02E65420000484310B500F5B052044618
:1092100007CA88B002AB83E807009FED1D7ADDED39
:10922000047A77EE877A9FED1B7ACDED047AD4ED40
:109230002B7AF0EEE77AF4EEC77A04F59940F1EE76
:1092400010FA00F150000BD5B4F9A22007EE902AD5
:10925000F8EEE77AF7EE006A86EEA77A84ED2B7ACD
:10926000D4F8AC200192194601AA50F0C5FB204663
:10927000FFF736FE2046FEF755F92046FEF72AFA9C
:109280002046FDF7E7FF2046FEF79CF808B010BD2A
:109290000AE81C410000003410B504462DED028B95
:1092A0001D205AF047FF60B304F54053D3F8EC009B
:1092B00000F0C4FA192108EE100A04F5546048F0D1
:1092C0001DFC02281AD00338012808D804F53350B1
:1092D000383050F06BFA90ED008ABDEEC88AB8EED7
:1092E000C88A9FED090A28EE000ABDEC028B04F53E
:1092F0009D403030BDE810406AF0B4BB9FED038A5A
:10930000EDE7BDEC028B10BD0AD7233C0000000046
:10931000134A0260134A426002F1740181601249EB
:10932000C16002F52A510161083941612439816126
:10933000A2F6FC71C1610D49016202F664614162ED
:1093400002F62821816202F62C21C16202F5236116
:1093500002F634224263064A01638263704700BF0B
:10936000A83C0D082C4F0020A87900209C790020F3
:10937000982D0020172952D8DFE801F0100C14189E
:10938000221F2A1C5126512E51513236393D41514E
:109390005144484D00F59E400C30704700F5AC40FC
:1093A0006430704700F59E404C30704700F59F4098
:1093B0000830704700F5A640F2E700F5AA40F7E74D
:1093C00000F5A8407C30704700F5A9404030704758
:1093D00000F5AB405830704700F5A7402430704787
:1093E00000F5A7406030704700F5A240FAE700F5AD
:1093F000AA404430704700F5A6402030704700F581
:10940000AD40FAE700F5AD407030704700F5005010
:10941000D0F8900B704700F5A8403430704700201A
:109420007047000073B50B6805461B6C08460C4678
:1094300016469847034605F53A500F4A0096042110
:10944000383050F07DFE4EF07FFD236805461B68E6
:10945000204698470A21024628464EF0D1FC074B89
:1094600093F8E1309B0641BF054A137843F00403AB
:10947000137002B070BD00BFFC280D08805C002096
:10948000DC86002038B50C4A182305460C464CF003
:10949000B5FE78B121462846FFF76CFF30B1014692
:1094A000064A2846FFF7BEFF002038BD28464CF08C
:1094B000EDFDF9E70120F8E77C290D081C290D08CE
:1094C00010B500F50053002283F88C2D094B04469B
:1094D00093F8E01000F5804304F54054D3F81C0DD8
:1094E000C9097AF02BFCD4F8EC000368BDE8104001
:1094F000DB681847805C002070B505460868036883
:109500005B690C461646984790B1306803685B6902
:10951000984768B905F54053D3F8102192F8CB204D
:1095200032B193F9E030002B02DB2846F8F79AFFBE
:1095300004480BF055F920680368BDE870409B684B
:10954000184700BF1486002070B500F5405504464A
:10955000D5F8EC000B4E0368DB6998473074D5F8FA
:10956000EC0003681B689847F070D5F8EC000368BE
:109570005B6C9847014604F59350BDE8704043F09A
:1095800081BB00BFBD86002070B52DED028B244B42
:1095900093F80531DB0782B006460D461446B0EE5F
:1095A000408AF0EE608A06D500232B60236002B06B
:1095B000BDEC028B70BD59F09FF9037F002BF3D0F7
:1095C000F36A9FED181A1B689FED170AB3F908306C
:1095D00007EE103AB36A1B68B3F9083007EE903A09
:1095E000B8EEC77AF8EEE77A67EE000A68EE811AFD
:1095F00027EE800A28EE011A01A9684625F0F8FE38
:10960000DFED0A6A9DED007ADDED017A27EE267A1C
:1096100067EEA67A85ED007AC4ED007AC7E700BF51
:10962000805C00200AD7233C530469390000C842FB
:1096300070B52DED028B88B0002302930393364B57
:1096400093F8053113F0010F0646B0EE408A06ADDF
:1096500002AC03D159F050F9037F5BB994E80300E1
:1096600085E803009DED060ADDED070A08B0BDECB4
:10967000028B70BDB36ADFED296A1B68B3F908304D
:1096800007EE903AF36A1B68B3F9083007EE103A18
:10969000B8EEC77AF8EEE77A27EE267A67EEA67A72
:1096A000F1EE476ACDED026ADFED1D6ACDED037A7A
:1096B000B0EEC77AB4EEE67AF1EE10FA06D5F0EE27
:1096C000E77AF4EEE67AF1EE10FAC7D403AA21465F
:1096D0001448F8F7F7FEDDED027A9DED037AF0EE1F
:1096E000E77AB0EEC77AF4EE477AF1EE10FACCBF23
:1096F000B0EE670AB0EE470A204627F053FE04A8F2
:109700008DED040ACDED050A27F0FEFE204688EE19
:10971000000A27F077FEA1E7805C00205304693936
:1097200000000034802C0020094B93F9E020002A2F
:109730000CDAB5EEC00AF1EE10FA07D9D3F8103101
:1097400093F8A100C31E584258417047002070474B
:10975000805C0020436A1B6893F8CB3043B1054B13
:1097600093F8E00000F0A000203818BF01207047F7
:1097700001207047805C002010B5436A04461868D9
:10978000D1B1022181F062FC236A9FED0C1A1868A6
:109790000368F0EE410ADB6AB0EE410A9847236A9B
:1097A000074A1868D2EDAD0A03689FED040A5B6EA4
:1097B000BDE81040002118470121E3E70000000048
:1097C000804C002010B5436A04461868002930D048
:1097D000022181F03BFC236A18687AF07FFA636A01
:1097E0001B6893F8A130012B04D8236A0121186863
:1097F0007BF00EF8636918687EF01AF963691868DF
:109800007EF076F963699FED0C0A18687EF09CFB88
:10981000636918687EF00AFC236A9FED071A1868CE
:109820000368BDE81040DB6AF0EE410AB0EE410A81
:1098300018470121CDE700BF0000000013B5044622
:1098400001A90C480AF090FA10B1019802B010BDBD
:10985000636918687CF0F6FF18B9074BD3F8F40C6D
:10986000F4E7064801AA032113F0B2FA0028F4D065
:10987000EBE700BF802C0020806C00207079002076
:1098800070B504462DED028B00296AD18368B3F9C7
:109890006E58642DB8BF6425FFF7D0FFA8426268F8
:1098A000A4BF324B93F8E150B2F93430ACBFC5F3EA
:1098B00080150125002BDBBF63691B685B4293EDBC
:1098C000C48AC8BF07EE903AB2F93230C8BFB8EECA
:1098D000E78A002BB8BF5B429BB25B4207EE903A2F
:1098E000A368F8EEE77AB3F96E68F4EEC87AF1EEA1
:1098F00010FAD8BFB0EE678A2046642EB8BF64263F
:10990000FFF79CFF6369A26B1B68D2ED001A93ED11
:10991000C61AD3ED0E0A311A00EE101AB8EEC00ABC
:1099200025F054F96368B3F93230002BB8BF5B42BD
:109930009BB25B4201EE103A40F29720B8EEC11A9A
:10994000F0EE480A24F060FE6369294618687DF04D
:109950001DF8BDEC028B6369BDE8704018687EF0AD
:1099600065BB9FED030A0025EEE700BF805C002089
:1099700000000000436A186803681B69184700006C
:1099800038B52DED028B03680446D3F88030984734
:10999000236B2A481B68F0EE408AB3F908500AF09E
:1099A000F5F84FF47A72041E4FF000012846D8BF34
:1099B0004FF4FA7424F066FE8442B6EE000A2ADD03
:1099C00007EE900AB8EEE77A07EE904A27EE007AA3
:1099D000F8EEE77A87EE278A4FF46D7038EEC00A0A
:1099E000F5EE087AB1EE400A80EE270AB7EE001ACB
:1099F000FEEE000A24F008FEF7EE007A77EEC07A59
:109A000028EE000A20EE080A20EE080AA7EE880ACF
:109A1000BDEC028B38BD031B07EE103AC4F57A7417
:109A2000B8EEC77A07EE904A27EE007AF8EEE77AAA
:109A300087EE278A38EE008ACEE700BF802C002010
:109A40002DE9F04F2DED028B00F5804900F54058CF
:109A500099F8084F89F8082F0546D8F8EC000368F4
:109A600083B01B680F4616469847B84221D105F5CA
:109A700000551A2E85F8686207D130B905F66C4595
:109A8000D9F81C3D2A68C3F8FC208C4B93F8E130D0
:109A9000980606D40124204603B0BDEC028BBDE835
:109AA000F08FB442F6D0864A137843F00203137065
:109AB000F0E7022E0CD01B2F12D105F59F40314646
:109AC000083003B0BDEC028BBDE8F04F01F066B981
:109AD00039462846FFF7D6FC04460028EBD1DAE7E2
:109AE00039462846FFF746FC0446019018B9284637
:109AF0004CF0CCFACFE7D8F8103193F8CBB003682C
:109B00005B699847019A05F5A74324338BF0010A56
:109B10009A4208BF0120BBF1000F08D101980368E9
:109B200051465B689847044648BB664A22E098F96C
:109B3000E030002B80F2B380002800F0B080DFF826
:109B40007CB1DBF8EC0003685B69984704460028A9
:109B500040F0A5800198FFF713FFABF54050B0EE41
:109B6000408AF8F769FCB4EEC08AF1EE10FA40F3CF
:109B70009680554A01992846FFF754FC8BE705F576
:109B8000435101AA2C31284605F50054FFF7B4FCD7
:109B90000198C8F8EC0084F8686203681B6898476D
:109BA0003246014605F57F604DF0E0FC05F53A5080
:109BB0000021383057F0B4FF94F9563123B105F540
:109BC0000550103066F058FDD8F8EC0003681B68AB
:109BD0009847C21E5042504104F63C4289F8AC0DF1
:109BE000D9F81C3D1268C3F8F82004F66C42D9F885
:109BF0001C3D1268C3F8FC20012F01D00B2F06D1A9
:109C000004F65444D9F81C3D2268C3F8FC202846C9
:109C1000FFF79AFC294B93F8E1309B063FF543AFE1
:109C200038E705F5005393F85021002A3FF476AF4A
:109C3000B3F86C21D1077FF571AF93F88C21002A1E
:109C40003FF46CAFD8F8102192F8CB20002A3FF4F3
:109C500065AF93F868320A2B7FF460AF98F9E03073
:109C6000002BFFF65BAF194A01992846FFF7DAFB94
:109C7000002410E716480AF0EDF90028D1D1D8F8F1
:109C8000EC0003685B6998470028CAD00198036814
:109C90005B69984704460028C3D10E4A6AE70198D9
:109CA00003681B6998470028E4D009480AF0C0F906
:109CB00004460028DED1084A5CE700BF805C002033
:109CC000DC86002046CF0E0844290D0868290D08BF
:109CD000802C002056290D08B6820E080148FFF797
:109CE000AFBE00BF802C002013B504468DED010AE5
:109CF00069F0CAFD6369A26B1B6892ED001A93EDCF
:109D00000E0AD3EDC60A01A968F04CFC9DED010ACC
:109D100002B010BD436A186803685B6A1847000008
:109D200038B5436A1C6894F8CB10054661B92046E3
:109D300081F08CF96B6A1B6893F8A10018B10128B7
:109D400014BF0320022038BD164803783BBBFFF741
:109D5000EBFC20BB144A92F8E03003F0A003202B68
:109D600017D0B5EEC00AF1EE10FA10D592F8E23035
:109D70005B070CD40121204681F068F96B6A1B68EF
:109D800093F8A130012B0CBF02200320DBE7022156
:109D9000F1E72046022181F059F90420D3E70120A0
:109DA000D1E700BF14860020805C002010B52DEDA7
:109DB000028B134B93F80531DB07044604D59FED66
:109DC000110ABDEC028B10BD58F096FD037F002BED
:109DD000F5D0636B186858F0B9FEA368DFED0A7A16
:109DE00003F5156292ED008A03F65413D3ED000AD1
:109DF00028EE278A25F0B6FA28EE000AE1E700BF30
:109E0000805C0020000000000000C8420148F8F714
:109E100083BB00BF802C00200148F9F717B800BFB2
:109E2000802C00200148FFF70BBE00BF802C0020D3
:109E300070B52DED028B7D4D95F8E1308CB000268C
:109E4000044658060496059603D5636918687CF0A5
:109E50006DFB95F80531D9075DD463689B899A0736
:109E60001BD573484FF0A2FCDFED727A90ED007ABB
:109E7000B4EEE77AF1EE10FA0FDD4EF065F83D2111
:109E80004DF09EFF6C4809220521FFF7D9FD20B94E
:109E9000092202212046FFF7C5FF636893F9543079
:109EA000CBB365489FED658AF8F7D0FFE3689FED77
:109EB000647A1B68D3ED0A7AF4EEC87AF1EE10FAF0
:109EC000B8BFF0EE477AB6EE000A27EE800A2046C9
:109ED000FFF7AEFB8DED040AB0EEC00AB4EEC80A7F
:109EE000F1EE10FACDED050A06D5F0EEE00AF4EE3B
:109EF000C80AF1EE10FA0ED495F8E2301B0704D42C
:109F00004EF022F849214DF05BFF95F8E23043F026
:109F1000080385F8E23095F8E3306FF3820385F8A3
:109F2000E330606909960A9609AD2A4604A90068DB
:109F300001237CF065FB636918687DF0D9FD6369D6
:109F400018687CF0B1FEA3688DED060ACDED070A16
:109F50008DED081AD3ED007AF5EEC07AF1EE10FA25
:109F600052DD384B9FED388AB3F9A83200EE903AB3
:109F7000F8EEE00A2046CDED030AFFF75FFCA36888
:109F8000DDED030AD3ED001A9FED2A0AB7EE002A91
:109F900007EE900A31EE822AB8EEE71A22EE082A7E
:109FA00061EE881A24F070FADFED287A20EE270A95
:109FB000DFED277A20EE270AACF022F9DFED257AD3
:109FC00020EE270A06A820EE088A27F09DFAB4EEB4
:109FD000C08AF1EE10FA17D5C8EE006A63699DEDEC
:109FE000067ADDED077A27EE267A67EEA67A8DED02
:109FF000067ACDED077A1B68D3F88823C3F894233B
:10A00000D3F88C23C3F89823236A13491C68284685
:10A01000FCF7E8FA0B9B009395E80C0006A9204694
:10A0200079F00EFF0CB0BDEC028B70BD805C00209F
:10A030006479002000002F44802C002000000034B0
:10A0400000007A43804C00200000C8420AD7233C1D
:10A0500035FA8E3C0AE81C41EC84002013B5044616
:10A060000191FFF7E5FE0199204602B0BDE81040DE
:10A07000FFF706BC0148FEF7DBBE00BF802C0020C6
:10A0800000487047385B00200148F8F733BA00BF3A
:10A09000802C002030B50F4D87B000230446694660
:10A0A000D5F8240D0093019302937CF015FED5F8AA
:10A0B000240D02A97CF064FE009B0393019B049392
:10A0C0000222029B059303A9204613F051F9204672
:10A0D00007B030BD806C0020014B01221A70704720
:10A0E0003C8500200020704700207047002070470A
:10A0F0000020704700207047002070470020704704
:10A100000020704700207047002070479FED010A33
:10A11000704700BF0000000000207047002070471B
:10A1200000207047012070470020704700207047D2
:10A1300001207047002070470120704701207047C0
:10A1400000207047012070470120704700207047B1
:10A150000048704794290D080048704794290D085D
:10A16000836893F86439DB0706D5002380F83C3018
:10A17000024B0222C3F8E42001207047805C0020DB
:10A1800090F83C3043B9836893F86439DB0742BFE9
:10A19000034B0122C3F8E420002380F83C307047D1
:10A1A000805C0020012380F83C3070472DE9F043AB
:10A1B0002DED0C8BF0EE409A20EE000A97B00025B2
:10A1C000A0EEA00A04468946B0EE41CAF0EE60AAAD
:10A1D00090461F46019502950395049505950695B1
:10A1E000ACF024FAF7EE00CAB4EEEC0AF1EE10FA85
:10A1F000C8BFCCEE807AA36803F5126203F624137D
:10A2000092ED009A9FEDC5DAD3ED000AC4BF69EE66
:10A21000A79A6AEEA7AAB0EE690A25F0A3F8A36888
:10A2200029EE0D9A03F5126203F62413D2ED008A8B
:10A23000D3ED000A29EE009AB0EE6A0A25F092F8F2
:10A24000A36868EE8D8A03F6381203F63C13D3ED4B
:10A25000000A92ED008A68EE808AB0EE4C0A25F082
:10A2600081F8636828EE0D8A93F9703028EE008A31
:10A27000002B00F0D980236A9FEDA90A18686C3082
:10A2800027F0F6FBB0EE60AACDED080A8DED091AB5
:10A290008DED070A24F062F9BDEEC0BAA14940F67F
:10A2A000B8321BEE100A24F0DDF9434207EE903A73
:10A2B0006368F8EEE77A93ED1A7A67EE877AB0EE84
:10A2C0004A0ACDED017A24F049F9FDEEC0BA40F614
:10A2D000B83294491BEE900A24F0C4F942426368F4
:10A2E000039507EE902A93ED1B7A93F97030F8EE00
:10A2F000E77A022B67EE877ACDED027A6ED18A4B30
:10A30000B3F9A8320AEE103AB8EECBBAB8EECAAA40
:10A31000236AB4EECABAF1EE10FA1A683DDDA368FA
:10A32000DFED820AA16B92ED051AD1ED001A03F55B
:10A33000126393ED007A27EE0D7A3AEE4B0AC7EEE0
:10A34000200A24F043FCDDED017A37EE800A8DED22
:10A35000010AB8EEEB0A236AB4EECA0AF1EE10FA6B
:10A360001A6834DDA368A16B92ED061AD1ED001ACC
:10A3700003F51263D3ED000A20EE8DDADFED6B0AF0
:10A380003AEE400ACDEE200A24F020FCDDED027A00
:10A3900037EE800A8DED020A20E0B1EE4A0AB4EEF3
:10A3A000C0BAF1EE10FAD4D5A368A16BDFED5F0A55
:10A3B000D1ED001A92ED051A03F5126393ED007AC0
:10A3C00027EE0D7A30EE4B0AC7EE200AB9E7B1EE60
:10A3D0004AAAB4EECA0AF1EE10FAC3D4236AD3F83B
:10A3E00000C00CF184030FCB12AD85E80F000EAE58
:10A3F0000AAD86E80F0085E80F0004AB01AA2946E4
:10A4000060467AF0B9F9636893F97030022B16D17F
:10A41000DDED047A39EE279ADDED057A78EEA78A2C
:10A42000DDED067A38EE278A89ED009AC8ED008ABC
:10A4300087ED008A17B0BDEC0C8BBDE8F083F0EE21
:10A44000E99AF0EEEAAAF4EEE9AAF1EE10FA48BFB2
:10A450006D46CDED009ACDED0AAAD5ED007ADFED7F
:10A46000340AB0EECCCAF4EECC7AF1EE10FAD8BFD2
:10A4700035468DED0ECA95ED007ADFED2E7A87EE2A
:10A48000270AAD20B7EE001A3CEEC00A24F0BCF853
:10A49000E369D3ED937A04A820EE270A27F0E8FABF
:10A4A000F0EEC07A8DED061AB0EEC91A31EE671AD9
:10A4B0008DED040AB0EEC11A39EE000ACDED050AA1
:10A4C000B520F1EE410A24F09FF8B0EE409A9DEDE0
:10A4D000050AB0EEE81AF0EEC07A31EE671A38EEEF
:10A4E000800AB0EEC11AF1EE410ABA2024F08CF8CD
:10A4F000F0EE408A9DED060AB0EEC81AF0EEC07A82
:10A5000031EE671A38EE000AB0EEC11ABF20F1EE44
:10A51000410A24F079F8B0EE408A85E70000C8428D
:10A520009F0CB34548F4FFFF804C002000007A44A4
:10A530000000000000A08C4510B52DED028B836A51
:10A54000044686B0186858F001FBE36A1868B0EE5C
:10A55000408A58F0FBFA636B8DED010A186858F0D9
:10A56000F5FA05ABB0EE401A03A92046DDED010A6D
:10A5700004AAB0EE480AFFF719FE636A186890F85B
:10A58000CB1000293AD180F061FD2046FFF7F8F9A1
:10A59000636A1B6893F8A1100129B0EE408A3DD090
:10A5A000032944D051B9236A012118687AF0E6FFE3
:10A5B000236A186879F07CFB9FED208A236AA268E1
:10A5C000186892F8642903689DED030ADDED040A1A
:10A5D0009DED051A92074CBFDB6B9B6B9847236A76
:10A5E000174A1868D2EDAD0A036800215B6EB0EE21
:10A5F000480A984706B0BDEC028B10BD114B93F989
:10A60000E120002A06DBD3F8E430022B04D190F8D5
:10A61000A1300BB90121B6E70221B4E7236A18681B
:10A620007AF0ACFF236A186879F058FBC4E7D9794F
:10A630000029C3D12046FFF71DFDBFE70000000041
:10A64000804C0020805C0020836893ED140AB5EEF6
:10A65000C00AF1EE10FA01DCFFF78CB97047000078
:10A6600070470000002070470120704702207047AB
:10A67000002070470020704701207047002070477D
:10A6800081F00100704700000120704701207047F1
:10A69000004870472C2A0D0800487047382A0D08DA
:10A6A00038B54369044618687CF0EEF918B9636957
:10A6B00018687DF06DFB636920461D68FFF7E4FCB8
:10A6C0006368B3F93820B3F9363000EE903A43426C
:10A6D00001EE102A00EE103AB8EEC11AF8EEE00AC8
:10A6E000B8EEC00A28467CF0BBF8636920461D68B6
:10A6F000FFF7CAFC6368B3F93820B3F9363000EECF
:10A70000903A434201EE102A00EE103A2846B8EE85
:10A71000C11AF8EEE00AB8EEC00A7CF01BF901207D
:10A7200038BD000030B52DED028B0446436985B07D
:10A730001D68FFF7A9FC6368B3F93820B3F9363018
:10A7400000EE903A434201EE102A00EE103AB8EEC5
:10A75000C11AF8EEE00AB8EEC00A28465B4D7CF05C
:10A760007FF82046FFF758FBB5F9A83208EE103AFB
:10A77000236A186803689B6E9847B8EEC88AF0EEA3
:10A78000400A02AA01A9B0EE480A2046FEF7FCFEE4
:10A790002046FFF70BFB236B1B68B3F90830F0EE84
:10A7A000408A00EE103A2046B8EEC00AFFF72EFBB2
:10A7B0002046B0EE408A8DED030AFFF765FC636822
:10A7C000B3F9363001EE103A434200EE903AB8EE5B
:10A7D000C11AF8EEE00A2B20B0EE480A23F014FF6D
:10A7E00020468DED030AFFF79BFA042813D8DFE813
:10A7F00000F0032F252A4B00236A186879F058FAD5
:10A80000236A002118687AF003F863699FED300A23
:10A8100018687DF099FB236ADDED020A18689DED4A
:10A82000010A0368B0EE681ADB6A98476369186822
:10A830007DF0FCFB05B0BDEC028B30BD236A01212D
:10A84000186879F0E5FF236A186879F047FADCE7C1
:10A85000204D2B7863B963689FED1F1ADFED1C0A4A
:10A8600093ED040A452023F0CFFE284609F0A0FF0F
:10A8700020469DED030AFFF737FA16488DED030ACF
:10A8800003A909F0CFFFC6E7636A0221186880F0C8
:10A89000DDFBB5F9A832114800EE103A02AA01A971
:10A8A000B8EEC00A67F0AEFB20469DED030AFFF745
:10A8B0001BFA0B488DED030A09F072FA63699DEDEE
:10A8C000030A18687CF052F8A5E700BF804C00200E
:10A8D000000000001486002000007A44C07A0020A6
:10A8E000005A00200020704790F8B931002B14BFA7
:10A8F0001B20032070470000002070470120704794
:10A9000090F89001062804D0A0F10A03584258415B
:10A9100070470120704700000120704701207047F8
:10A9200090F8B901034A044B002814BF104618469A
:10A93000704700BFD02A0D08D2950E0890F8B901D3
:10A94000034A044B002814BF10461846704700BF46
:10A95000DC2A0D08D2950E0890F890010B3818BF2C
:10A960000120704790F8B9312BB9044BD3F8880C0B
:10A9700000F0010070470020704700BF804C0020AD
:10A9800090F8903123B9034B187880F0010070479C
:10A9900000207047F885002038B590F89041012CD0
:10A9A000054601D0002038BDC368186803681B69DC
:10A9B00098470028F6D1EB681B68204683F8B84812
:10A9C000F1E70000C3681B68002283F8B828012063
:10A9D0007047000070B52DED028B002380F8B9316F
:10A9E000B0F87030012B84B004460D4601D8002920
:10A9F00046D0636A254E1B6893F8CB3073BB24485E
:10AA0000072384F890310368022B02D10021FBF761
:10AA1000F3FB9FED208AE368F0EE480A1868B0EE79
:10AA2000481AF0EE481AB0EE480A01257EF084FD7F
:10AA300084ED738A84ED748A84ED758A84F8B85144
:10AA400004F59A7027F0FCFC134805F0D9F896F845
:10AA5000E2306FF3C30386F8E23011E096F9E0309C
:10AA6000002BCCDA04F13C0029F0DCFD054600287F
:10AA7000C5D12046FFF704FB084A02214FF060FBD6
:10AA8000284604B0BDEC028B70BD00BF805C002086
:10AA9000EC84002000000000FC800020E42A0D0867
:10AAA00038B5094D95F8C83F012B044603D105F68A
:10AAB000C47027F02DFD95F8351E04485AF086FD28
:10AAC000002384F8B93138BD806C00203C7A002026
:10AAD00010B52DED028B094B0446D3F8280DB0EECE
:10AAE000408A7EF0C1F89FED060A28EE008A012018
:10AAF00084ED748ABDEC028B10BD00BF806C002019
:10AB00000AD7233C10B52DED028B094B0446D3F830
:10AB1000280DB0EE408A7EF0B7F89FED060A28EEC9
:10AB2000008A012084ED758ABDEC028B10BD00BF48
:10AB3000806C00200AD7233C10B52DED028B094B09
:10AB40000446D3F8280DB0EE408A7EF0ABF89FEDB6
:10AB5000060A28EE008A012084ED738ABDEC028B80
:10AB600010BD00BF806C00200AD7233CC3681B685F
:10AB700018697CF0CBB9000038B5D0F894310446A0
:10AB80000D461BB988F0DEF9C4F8940188F0DAF9B3
:10AB9000D4F89431C01A4FF47A73B0FBF3F0B4F8E0
:10ABA0009231984209D32046FFF76AFA2B88044A6B
:10ABB00006214FF0C5FA012038BD0020FCE700BF98
:10ABC000002B0D0890F89031052B05D1054BD3F8DB
:10ABD000303DD8687CF012B9C36818680368DB6838
:10ABE000184700BF806C002008B590F89031052B05
:10ABF0000BD1094BD3F8303DD868243026F084FCC3
:10AC0000BCEEC00A10EE100A08BDC36818680368DD
:10AC10009B689847F4E700BF806C002090F8903163
:10AC20008B4206D00B2B80F8901102D10148FCF723
:10AC3000B5BF7047802C002073B501231E4E80F8ED
:10AC40007530D6F8EC30834205460A4614D101240B
:10AC500085F8B941D6F8EC00019203681B68984763
:10AC6000019A014615484CF081FC96F8E1309A06AD
:10AC70001BD4204602B070BD01910321FFF7D2F82A
:10AC8000019A04460028E2D185F875004DF05CF980
:10AC90001B220A214DF0B4F896F8E1309B06E8D566
:10ACA000074A137843F0040303E0054A137843F09E
:10ACB00002031370DDE700BF805C0020703C0020C1
:10ACC000DC86002030B585B004460D460146684656
:10ACD000FFF7E0F9694604F13C002AF055FAC8B9DB
:10ACE0004DF032F91B220A214DF08AF80D4B93F8F2
:10ACF000E1309B0604D50C4A137843F0040313702B
:10AD00002046FFF7BDF9094A04214FF019FA002047
:10AD100005B030BD2946204605B0BDE83040FFF7FC
:10AD20008BBF00BF805C0020DC860020142B0D0848
:10AD300030B585B004460D4601466846FFF7AAF9CE
:10AD4000694604F13C002AF043FAC8B94DF0FCF81A
:10AD50001B220A214DF054F80D4B93F8E1309B066D
:10AD600004D50C4A137843F0040313702046FFF710
:10AD700087F9094A04214FF0E3F9002005B030BDFE
:10AD80002946204605B0BDE83040FFF755BF00BF5B
:10AD9000805C0020DC860020502B0D087FB5054626
:10ADA0000E4605F13C0401466846FFF773F9694613
:10ADB00020462AF00DFAC0B9204669462AF0E4F987
:10ADC000044690B94DF0C0F81B220A214DF018F846
:10ADD0000D4B93F8E1309B060FD42846FFF750F94E
:10ADE0000A4A04214FF0ACF904E031462846FFF747
:10ADF00023FF0446204604B070BD054A137843F093
:10AE000004031370E9E700BF805C0020882B0D0865
:10AE1000DC86002030B5044685B00F4809F008F9FB
:10AE20000546B0B1072384F89031002301930293C3
:10AE30000393E36801A918687DF0B0FEE368186821
:10AE4000036801A95B680022984704480021FBF7CA
:10AE5000D3F9284605B030BD802C0020EC840020BA
:10AE6000F0B5424FD7F8FC2CD7F8F83C2DED028B0B
:10AE70001343D7F8F42C134387B005460C460CD186
:10AE80004BF06EFB40F275124FF4801107B0BDEC31
:10AE9000028BBDE8F0404BF01BBB80697FF01AF9D4
:10AEA0002046B0EE408A11F087FF03283AD1EB68C4
:10AEB00001A918687DF04EFF064698B3DDED017AD2
:10AEC0006368009338EE678A294BDFED2A7A93F99D
:10AED000E0309FED290A2948002BA8BFB0EE670A91
:10AEE00038EE008A009BBDEEC88A002118EE102AB9
:10AEF0009342ACBF00930092FBF77EF96B69186830
:10AF00007CF046FFDDED007A1D48B8EEE70A3146D9
:10AF100009F008FF00212846FFF780FE07B0BDECCE
:10AF2000028BF0BD94E80F0002AE86E80F00D7F860
:10AF3000F83C04936A46D7F8FC3C0593022130465E
:10AF400011F046FF78B94CF0FFFF022215214CF0BA
:10AF500057FFDDED037AF8EEE77A77EE887AFDEEBB
:10AF6000E77ACDED007A0026AEE700BF806C0020C6
:10AF7000805C0020000000000000C842EC8400203B
:10AF8000F885002030B52DED028BC36887B00446EC
:10AF900018680D467DF0D2FE00284BD194F8902120
:10AFA00000230093019302936AB93148039303A9E4
:10AFB0000493059309F0E8FE28B1039B0093049BDA
:10AFC0000193059B029394ED730A9FED2A8AE3682F
:10AFD000DDED000A9DED011ADDED021A1868B4EEF0
:10AFE000C80AF1EE10FAAABFDFED237A9FED230A1B
:10AFF00020EE270A7EF0A0FAD4ED747AF4EEC87A37
:10B00000F1EE10FA07DBE3689FED1B0A186827EEE4
:10B01000800A7DF029FED4ED757AF4EEC87AF1EE5F
:10B0200010FA07DBE3689FED140A186827EE800A20
:10B030007DF02AFEE368294618687EF0A5F90546EA
:10B0400088B10F4B1B68022B09D0032B03D10D4B8A
:10B0500093F9D9321BB10A480021FBF7EDF8012121
:10B060002046FFF7DBFD284607B0BDEC028B30BD64
:10B07000F8850020000000340000C84200000000F5
:10B08000EC840020804C002010B52DED028BC368AD
:10B09000DFED348A1B684269D3ED0A0A9FED328ADC
:10B0A00093ED060AF4EEE80A0446F1EE10FA106891
:10B0B000B8BFF0EE480A7BF0B9F9E36862691B6833
:10B0C0001068D3ED0A0A93ED060AF4EEE80AF1EEF1
:10B0D00010FAB8BFF0EE480A7BF020FA63691868EE
:10B0E0007BF0B0FB18B9636918687CF0EBFBE36890
:10B0F00062691B68106893ED080A93ED0C1AD3ED92
:10B10000070AB0EEC00A7BF0ABFBE36862691B681C
:10B11000106893ED080A93ED0C1AD3ED070AB0EE10
:10B12000C00A7BF017FC636918687BF0ADFC18B9A6
:10B13000636918687CF02CFE00210C48FBF75CF872
:10B140000B4868F027FD0B4AB2F8E23023F4816324
:10B15000A2F8E230BDEC028B20460221BDE810408F
:10B16000FFF75CBD0000003400007A43EC8400204F
:10B17000307B0020805C002010B50C4B0446D3F8D7
:10B18000300D90ED0B0A90F8502000F11C017DF07D
:10B190004DFA07480368022B02D00821FBF72CF870
:10B1A00020460521BDE81040FFF738BD806C002027
:10B1B000EC840020F0B52DED028B4A4DDFED4A8A7C
:10B1C000B0EE408A8FB00446D5F8300D0E461746D3
:10B1D0007DF0A2F8F0EEC87AF4EEE87AF1EE10FA1B
:10B1E00007D49FED420AD5F8300D28EE000A7DF015
:10B1F000F9F8D5F8300D90ED0B0AB0EEC00A0FB19A
:10B20000B1EE400A7DF0DEF80023D5F8300D07934B
:10B2100002AA07A9089309937DF000F9DFED347ABB
:10B220009DED027AB4EEE77AF1EE10FA56DD0222D5
:10B2300007A90AA812F09CF871680191304611F034
:10B24000BBFD019902460AA811F08CFDE3680AA92A
:10B2500018687EF099F810B92648FDF799F8A069AA
:10B260007EF036FF02684368D5F8300D049303A9D9
:10B270001C30039226F07AF805A88DED050ACDED75
:10B28000060A26F041F91C4B1B68022B1BD0D5F88F
:10B29000303D1948D3ED0A7AF4EEE87AF1EE10FA6F
:10B2A000B8BFD3ED047AF4EEC07AF1EE10FA4FF0A5
:10B2B000000110D5DFED117AB4EEE70AF1EE10FAD5
:10B2C00009DDFAF7B9FF04212046FFF7A7FC0FB00C
:10B2D000BDEC028BF0BDFAF78FFFF4E72046FFF7D5
:10B2E0004BFFF4E7806C0020000000340000C842EF
:10B2F00000009643802C0020EC8400200000FA43DC
:10B3000070B52DED028B294BDFED298AD3F8284D3E
:10B31000D3F8245DD4ED0A0A9FED268A94ED060A3F
:10B32000F4EEE80AF1EE10FAB8BFF0EE480A06466D
:10B3300028467BF07BF8D4ED0A0A94ED060AF4EE79
:10B34000E80AF1EE10FAB8BFF0EE480A28467BF0A2
:10B35000E5F828467BF076FA10B928467CF0B2FA78
:10B3600094ED080A94ED0C1AD4ED070AB0EEC00A69
:10B3700028467BF075FA94ED080A94ED0C1AD4ED8A
:10B38000070A2846B0EEC00A7BF0E4FA28467BF0B4
:10B390007BFB10B928467CF0FBFC07480021FAF73C
:10B3A0002BFFBDEC028B0123337070BD806C00203D
:10B3B0000000003400007A43EC84002008B5074800
:10B3C000D0F8883C9B0704D50121A0F50050F6F782
:10B3D000FFFEBDE80840024809F004BB804C002095
:10B3E000F885002030B589B00446FEF7B3F930B1D6
:10B3F0000021204609B0BDE83040FEF7E3B9636A9A
:10B40000022118687FF022FEE368186803685B6910
:10B41000984701461048FCF7A9FE636918687CF05C
:10B4200005FE236A1D68636918687BF03DFC05AC66
:10B4300020460A498DED020ACDED030A8DED041A6E
:10B44000FBF7D0F8079B009394E80C0002A928466C
:10B4500078F0F6FC09B030BD802C0020EC84002090
:10B4600038B50446FEF776F9054628B12046002196
:10B47000BDE83840FEF7A6B9636A022118687FF07C
:10B48000E5FD29462046BDE83840FEF7E7BD00004F
:10B490000148002106F0C2BE5882002030B5174D89
:10B4A0009FED170A05F5804389B00446D3F8300DA7
:10B4B0007DF01CF901462846FCF758FE63691868C0
:10B4C0007CF0B4FD236A1D68636918687BF0ECFBAF
:10B4D00005AC20460B498DED020ACDED030A8DED3A
:10B4E000041AFBF77FF8079B009394E80C0002A96D
:10B4F000284678F0A5FC09B030BD00BF802C0020A4
:10B5000000000000EC84002030B589B00446FEF74E
:10B5100021F930B10021204609B0BDE83040FEF7E6
:10B5200051B9636A022118687FF090FDE3681868DA
:10B5300003685B69984701461048FCF717FE63698A
:10B5400018687CF073FD236A1D68636918687BF0D6
:10B55000ABFB05AC20460A498DED020ACDED030A8E
:10B560008DED041AFBF73EF8079B009394E80C005E
:10B5700002A9284678F064FC09B030BD802C002078
:10B58000EC84002030B52DED028B83B00446FEF72D
:10B59000E1F820B9636A1B6893F8CC3043B9002105
:10B5A000204603B0BDEC028BBDE83040FEF70AB97F
:10B5B00094F89831DA071DD4E3681D682B68284693
:10B5C0009B689847D5ED097A94F89831B4EEE70A6C
:10B5D000F1EE10FA4CBF0122002262F3000384F85E
:10B5E000983107D4204603B0BDEC028BBDE8304053
:10B5F000FFF7F8BE94F898319B0734D4E368DFED89
:10B60000458A1B686269D3ED0A0A9FED438A93ED70
:10B61000060A1068F4EEE80AF1EE10FAB8BFF0EE90
:10B62000480A7AF003FFE36862691B681068D3ED8B
:10B630000A0A93ED060AF4EEE80AF1EE10FAB8BF32
:10B64000F0EE480A7AF06AFF636918687BF0FAF84E
:10B6500018B9636918687CF035F994F8983143F0AB
:10B66000020384F898312D4BD4F8A021D3F8F43C90
:10B670009B1A07EE903AB8EEE78AF1EE047AB0EE44
:10B68000C87AB4EEE77AF1EE10FA38D594F898312A
:10B6900043F0040384F89831204684ED678AFEF76E
:10B6A000C7FB6369A26B1B68D2ED001A93EDC61A43
:10B6B000D3ED0E0AB1EE480A23F088FA63691B68DD
:10B6C00040F2AA4093EDC31AD3EDC40A22F09CFFC6
:10B6D0002046FEF709FB12488DED010A08F060FBD9
:10B6E00063699DED010A18687BF040F96369186889
:10B6F00003B0BDEC028BBDE830407CF097BCD4EDCC
:10B70000677A68EE277AF5EEC07AF1EE10FAC3D5C3
:10B71000BCE700BF0000003400007A43806C0020CA
:10B72000005A002030B52DED028B83B00446FEF7A1
:10B7300011F820B9636A1B6893F8CC3043B9002133
:10B74000204603B0BDEC028BBDE83040FEF73AB8AE
:10B750006369DFED347A1B6894ED710A93EDC31AC7
:10B76000D3EDC40A20EE270A40F2C44022F04CFF79
:10B770002046FEF7B9FA236A186803689B6EB0EE9C
:10B78000408A9847284BB3F9A83207EE903AB4F8AC
:10B79000BC316425F8EEE77A13FB05F3B4EEE70A53
:10B7A00007EE103A94F9BE31F1EE10FAD8BFF0EE80
:10B7B000407A13FB05F39FED1D0AF8EEC76A07EE0A
:10B7C000103AF4EE407AB8EEC77AF1EE10FA58BFAC
:10B7D000B0EE670A6846CDED006A8DED017A25F07E
:10B7E000E5FE236ADDED010A1868B4F8C03102688D
:10B7F0009DED000A126B13FB05F301EE103A0121D7
:10B80000B8EEC11A90476369B0EE480A18687BF039
:10B81000ADF8636918687CF009FC03B0BDEC028BDD
:10B8200030BD00BF0000C842804C002000007A44B8
:10B830002DE9F0432DED028BB64F85B00446D7F8C5
:10B84000EC00FDF787FF48B1D7F8EC00002105B008
:10B85000BDEC028BBDE8F043FDF7B4BF07F58056A1
:10B86000D7F8100102217FF0F1FBD6F81C3D93EDD3
:10B87000378A87F067FBB7F8E03003F48143054669
:10B880007BB1D6F8240D7AF051FE2378022B08D133
:10B8900055F02AFBA04BA14A06214EF051FC032390
:10B8A000237063F07DFE63F067FE48B163F078FEBD
:10B8B00063F06CFE20B12378012B10D9022B1DD030
:10B8C0002378082B00F28581DFE813F0210039008E
:10B8D00063000A013E0145015A015C012A0055F04E
:10B8E00003FB8D4B8E4A06214EF02AFCD6F8243DF0
:10B8F000D3F85433636108232370E1E755F0F4FA79
:10B90000854B884A06214EF01BFC0323F4E7D6F84A
:10B91000280D03681B69984710B12046FFF7F0FC1B
:10B920002378082B00F27381DFE813F05C016401D7
:10B9300064017A017A017A017A0182018201A560AB
:10B94000D6F8243D9FED787AD3F854336361774B72
:10B9500003F6C842D2ED007AF4EEC77AF1EE10FA9F
:10B960004EDB9FED737A67EE877AD6F8283D93ED2C
:10B97000087AB0EEC77AF4EE477A4FF07E53F1EED4
:10B9800010FA48BFB0EE677A2361022384ED067A8D
:10B990002370D4ED016A9FED647AD6F8243DF0EE71
:10B9A000E67AF4EEC77AF1EE10FA0AD4D4ED057A0D
:10B9B00093EDD56A77EEC67AF4EEE76AF1EE10FA07
:10B9C00029D4DFED5C6AD4ED067A67EEA67AD3ED72
:10B9D000DB6AF4EEE76AF1EE10FA26DCA368D4ED38
:10B9E000047AEB1AB3F5FA6F21D2B4EE678AF1EE5E
:10B9F00010FAC8BFB0EE678A84ED048AE5608FE76D
:10BA0000B3F9DE32002BB8BF5B429BB207EE903A2F
:10BA1000F8EEE77AA9E70623237055F065FA3E4B66
:10BA2000454A04214EF08CFB7AE7A56078E7DFF801
:10BA3000FC8008F6BC43D3ED006A67EEA67AF4EE0C
:10BA4000C87AF1EE10FAD9D408F54C69D9ED007A2C
:10BA5000F4EEC77AF1EE10FA22DB98F8F03C33B935
:10BA60000623237055F040FA2B4B344AD9E7A8F54A
:10BA7000005008F0E9F898B198F9063D83B9B8F993
:10BA8000F23CD9ED007ADFED2A6A07EE103A67EE54
:10BA9000A67AB8EEC77AB4EEE77AF1EE10FAADDC2A
:10BAA000E068281AB0F5FA7F7FF63AAF03232370D7
:10BAB00008F6BC4855F018FA98ED007AD4ED047AEF
:10BAC00067EE277A054617EE900AF4F71DFD124B34
:10BAD0001B4ACDE90001062128464EF031FB1FE745
:10BAE000D6F8240D7CF0D0F963F05AFD63F044FDE4
:10BAF00068B155F0F9F9084B124A06214EF020FBC7
:10BB000063F04EFD63F026FD0423237008E7052350
:10BB1000FBE700BF805C0020D42B0D08E22B0D0852
:10BB2000EC2B0D08032C0D0800000034804C002085
:10BB30000000C842333373BF152C0D08302C0D089C
:10BB4000602C0D08882C0D0863F02AFD63F014FDAD
:10BB5000C0BB05232370404BE068DFED407AD3ED96
:10BB6000006A9FED3F7A2D1AA6EEA77A07EE905A4B
:10BB7000F8EE677AF4EEC77AF1EE10FA3FF5D0AE40
:10BB800007232370D6F8243D9FED367AD3EDC37A90
:10BB9000D3EDC66A67EE877AB6EE007A67EEA77ACB
:10BBA00067EE877A87EEA67AD4ED057A77EEC77AC4
:10BBB00093EDD57AF4EEC77AF1EE10FA3FF6B0AE17
:10BBC0000823A2E763F0ECFC63F0E0FC0028C0D19E
:10BBD000A6E64AF0C5FC40F29C524FF480114AF0B0
:10BBE00077FC9DE6204805B0BDEC028BBDE8F04334
:10BBF000FFF7F8BBD7F8EC00FEF71AF994ED060A48
:10BC00000121B1EE400AD6F8240D7AF0BFFED6F835
:10BC1000240D05B0BDEC028BBDE8F0437CF006BA04
:10BC2000D7F8EC00FEF704F99FED100A0021EAE7CF
:10BC30009FED0E8AD7F8EC008DED038AFEF7F8F839
:10BC4000D6F8240D0123B0EE480A03AA04F114012A
:10BC50007BF0A2FCDBE700BF4459002000007A44DF
:10BC60000000FA43CDCCCC3D087C00200000000051
:10BC700030B590F8B83185B00446F3B1684611F09C
:10BC80006BF8414869460AF0CBFF50B104F13C0023
:10BC900029F066FA002384F8B83104F59A7026F08A
:10BCA000CFFB94F890310B2B2DD8DFE803F0294B14
:10BCB0004F534B572C5B5F632C6700F59A7026F04F
:10BCC000BFFB04F13C0590B194F84030012B0ED13C
:10BCD00094F89031012B0AD1284629F0AFF850B1E1
:10BCE0002046FEF7CDF9294A02214EF029FA2846CE
:10BCF00029F0D2F8D5E72046FEF7C2F9244AF3E747
:10BD00002046FFF75BFB94F844303BB994F846308B
:10BD100023B994F840309A1E5342534194F8B92104
:10BD200082B37BBB84F8B9311A4BD3F8EC000368BB
:10BD30001B689847014618482D2205B0BDE83040E1
:10BD40004BF014BC2046FFF74DFBDCE72046FFF725
:10BD500087FBD8E72046FFF79BFBD4E72046FFF799
:10BD60009DFBD0E72046FFF7CFFBCCE72046FFF74F
:10BD700009FCC8E70948FFF75BFDC4E72046FFF769
:10BD8000D1FCC0E705B030BD303F0020A42C0D0829
:10BD9000CC2C0D08805C0020703C00203C850020ED
:10BDA0002DE9F0412DED028B074684B008460E4682
:10BDB00011F002F8032880466D4628D1FB68186808
:10BDC0007CF022FE012822D12148294607F0CCFF31
:10BDD0000446B0B17B69DDED007A1B68F8EEE77AC6
:10BDE00093EDF27A77EEC77A4246FDEEE77A17EEE8
:10BDF000901AC829CDED007AB8BFC821304610F09E
:10BE0000B1FF204604B0BDEC028BBDE8F081114BC0
:10BE10000FCB85E80F00304610F0CEFF01462846D4
:10BE200011F032F804460028EBD07B69DDED017A91
:10BE30001B68B8EEE78AD3EDF27A284638EE678AB7
:10BE400010F0BAFFBDEEC88A024618EE101AD5E708
:10BE5000802C00207079002010B543699FED126A94
:10BE60001B68D3EDF06A93EDF17AD3EDF27A86B0E8
:10BE700066EE866A27EE067A67EEC67A68460C4654
:10BE8000CDED006A8DED017ACDED027A25F0B4FD9D
:10BE900003A920468DED030ACDED040A8DED051AA8
:10BEA00011F0BAFA06B010BD0AD7233C30B50832FB
:10BEB00004461D460FCA84E80F00134301BFAB6858
:10BEC000A360EB68E360636885B093B9204610F027
:10BED00073FF03AA0146284610F07AFF60B1039968
:10BEE0000191204610F068FF01990246204610F0AB
:10BEF00039FF204605B030BD696801912846F1E759
:10BF000030B50B6985B004460BB94B6953B30023B8
:10BF1000C4F8B43108310FC96D4685E80F002946D1
:10BF20002046FFF73DFF98B9124B0122D3F8F41CCD
:10BF3000284610F017FF4CF007F8022215214BF0AD
:10BF40005FFF2046FEF79CF80B4A02214EF0F8F8FE
:10BF500029462046FFF716F810B90848FCF718FAEA
:10BF600005B030BD0123C0F8B43105B0BDE83040A4
:10BF7000FFF78AB8806C0020002D0D08802C00206F
:10BF800070B51A4B04460E460FCB88B06D4685E857
:10BF90000F0020462946FFF75FFFE36818687CF032
:10BFA000CDFE98B1E368186803681B69984768B1CB
:10BFB000E368294618687CF033FD38B94AF0D0FAB6
:10BFC00040F295624FF480114AF082FA214604A8AB
:10BFD0002B463246FFF76AFF04A92046FEF7D2FF40
:10BFE00010B90348FCF7D4F908B070BD707900208F
:10BFF000802C002070B5154B0C4606460FCB88B040
:10C000006D4685E80F0029463046FFF725FF2B4691
:10C010002246314604A8FFF749FF6288A388122A06
:10C020004FEA132305D1227ED20744BF03EB8303DB
:10C030005B00227A07EE903AC2F34002B8EE670A3C
:10C0400004A93046FFF7B6F808B070BD707900203B
:10C0500038B504460D46FFF793FF0023C4F894312A
:10C06000AB88A4F8923138BD7FB50D460446FFF782
:10C0700087FF05F108010FC96E4686E80F001343DC
:10C0800006D1234BD3F8F82CD3F8FC3C029203934F
:10C0900004F5D0720121304610F09AFE94F89831E0
:10C0A00070B923F0050343F0050384F89831204666
:10C0B000FDF7E6FF174A06214EF042F804B070BDC6
:10C0C00023F0070384F898310023C4F89C31E36817
:10C0D00062691B68106893ED080A93ED0C1AD3EDA2
:10C0E000070AB0EEC00A7AF0BBFBE36862691B681E
:10C0F000106893ED080A93ED0C1AD3ED070AB0EE21
:10C10000C00A7AF027FC08212046FEF787FDD5E714
:10C11000806C00202C2D0D082DE9F0438DB06D466C
:10C1200088461C46074613460A4601462846DDE96E
:10C130001469FFF7BBFE95E80F0084E80F0007A81D
:10C1400010F00AFEB8F80430F3B9B8F80010013165
:10C1500005AA89B207F13C0028F01CFAA0B12346D9
:10C1600005AA39462846FFF7A1FE95E80F0086E8A4
:10C170000F00BDF81630A3F152025342534189F823
:10C1800000300DB0BDE8F08394E80F0086E80F00A2
:10C190000023F4E770B58B8892B004460D4616462E
:10C1A000002B47D10DA810F0D7FD298801310BAA2B
:10C1B00089B204F13C0028F0EDF900283AD0BDF82E
:10C1C0002E1052291CD019D8112913D80F2913D990
:10C1D00033462A46214603A8FFF768FE03AB2146F3
:10C1E00007A80BAAFFF762FEE36807A918687DF0AD
:10C1F0000BF901E01329EBD012B070BD5E29FAE70C
:10C2000007AD03A810F0A8FD284610F0A5FD0DF11C
:10C210000B03CDE90053324603AB0BA92046FFF7D1
:10C220007BFFE0689DF80B3000682A4603A97DF08B
:10C23000C1F8E1E70120DFE770B5214B04460E4667
:10C240000FCB88B06D4685E80F0020462946FFF7E2
:10C2500003FEE36818687CF071FD98B1E368186824
:10C2600003681B69984768B1E368294618687CF041
:10C27000D7FB38B94AF074F940F216624FF48011D6
:10C280004AF026F9214604A82B463246FFF70EFE57
:10C2900004A92046FEF776FE20B90A48FCF778F894
:10C2A00008B070BD0023C4F89431B388A4F892316B
:10C2B00004AA31462046FFF76DFF0028F0D1ECE7D5
:10C2C00070790020802C0020F0B5324B04460E46D9
:10C2D0000FCB91B004AD85E80F0020462946FFF74B
:10C2E000BBFDE36818687CF029FD98B1E368186825
:10C2F00003681B69984768B1E368294618687CF0B1
:10C300008FFB38B94AF02CF94FF4DF624FF48011FB
:10C310004AF0DEF80CAF08A810F01EFD384610F009
:10C320001BFD0DF10F03CDE900732A4608AB314622
:10C330002046FFF7F1FEE0689DF80F3000683A46AE
:10C3400008A97DF07DFB20B91348FCF721F811B056
:10C35000F0BD0023C4F89431B388A4F8923108AA40
:10C3600031462046FFF716FF0028EDD00B4B1B6827
:10C37000022B09D0032B03D1094B93F9D9321BB1FE
:10C3800006480021F9F758FF01212046FEF746FC38
:10C39000DDE700BF70790020802C0020EC840020B5
:10C3A000804C002037B504460D4686F0CBFDC4F81E
:10C3B000A801D5ED027AF5EEC07AF1EE10FA17DD9C
:10C3C0009FED137A67EE877AFCEEE77AC4ED697A1F
:10C3D0002046FDF755FED4F8A4214FF47A73B2FB42
:10C3E000F3F30C4A062103B0BDE830404DF0A8BE7F
:10C3F00063F0C6FB0023009395F90D2095F90E30EC
:10C4000095F90C1063F058FBC4F8A401E0E700BFF5
:10C4100000007A44442D0D0810B5B1F90A30A0F897
:10C42000BC3191F90C3080F8BE31B1F90D30A0F873
:10C43000C031B1F90F3007EE903AF8EEE77A0446D2
:10C44000C0ED717A86F07EFD0B21C4F8C80120464C
:10C45000BDE81040FEF7E2BB38B504460D4686F055
:10C4600071FDC4F8B001D5ED027A9FED047A67EE54
:10C47000877AFDEEE77AC4ED6B7A38BD00007A4426
:10C480004A7C06480B46003A91F91010D3ED030A96
:10C4900093ED020A18BF0122F9F7D8BEEC84002000
:10C4A00070B51B4E0446D6F8EC00036886B01B68D6
:10C4B0000D469847042806D16B88102B0FD0732B9C
:10C4C00020D000201CE0D6F8EC0003681B689847D9
:10C4D0000328F6D194F89031062BF2D1ECE705F160
:10C4E00008010FC902ACDFED0B0A84E80F0000233E
:10C4F00009480093B0EE600A1A46214603F0C2F9DB
:10C5000006B070BD20462946FFF7BAFF0120F7E7C5
:10C51000805C002000000000FC80002038B5D1F8CD
:10C52000093007EE903AF5EEC07AF1EE10FA0546C2
:10C530000C4605DD0B7A022B03D01ED9032B0ED03F
:10C5400038BD154B9FED150AD3F8280D27EE800A4C
:10C550007CF08AFBD4F80930C5F8D031F0E70E4BF7
:10C560009FED0E0AD3F8280D27EE800A7CF08CFB95
:10C57000D4F80930C5F8D431E2E7074B9FED070A3C
:10C58000D3F8280D27EE800A7CF08CFBD4F8093014
:10C59000C5F8CC31D4E700BF806C00200000C84251
:10C5A00038B5114D0C4605F6BC5095F8351E58F0BF
:10C5B000EFFF58B195F8351E05F6BC5058F0F0FF66
:10C5C00020B994ED040A0948F9F7DEFE94ED041A47
:10C5D000D4ED020A94ED030A95F8351E0448BDE82F
:10C5E0003840002259F014B8806C0020EC84002000
:10C5F0003C7A0020F0B50B69214F85B005460E4608
:10C600000BB94B6953B300233B7006F108030FCB02
:10C610006C4684E80F0021462846FFF7C1FB98B915
:10C62000184B0122D3F8F41C204610F09BFB4BF072
:10C630008BFC022215214BF0E3FB2846FDF720FD81
:10C64000114A02214DF07CFD21462846FEF79AFC56
:10C6500038B90E48FBF79CFE05B0F0BD3846FEF732
:10C660004FFEB38807EE903AF8EE677A0921284624
:10C67000C7ED017A05B0BDE8F040FEF7CFBA00BFC4
:10C680003C850020806C0020542D0D08802C00205B
:10C6900010B5044C237813B1034867F075FA20787D
:10C6A00010BD00BFF8850020307B002000780728EF
:10C6B00094BF00200120704713B5094B0191044637
:10C6C000D3F8280D03681B69984730B101992046BB
:10C6D00002B0BDE81040FEF74FBA02B010BD00BF77
:10C6E000806C002090F8983113F0010018BFC3F35C
:10C6F00080007047094A034692F8150668B192F81F
:10C700001426043A012A07D85B6A1B6893F8A10033
:10C71000431E58425841704700207047807C0020DB
:10C7200010B5044686F00EFCD4F8B031C01AD4F827
:10C73000AC3123EAE37398424FF0000084BFC4F8A1
:10C74000AC01012010BD000010B503680446DB6D8C
:10C750009847D4F8AC3123EAE37398424FF00000D5
:10C760003CBFC4F8AC01012010BD000008B504486E
:10C770000321F9F741FDBDE808400148F9F760BE23
:10C78000EC84002070B51C4B0446D3F8280D0368D8
:10C790001B690E469847054610B90025284670BD0E
:10C7A000D4F894315BB986F0CDFBB4F89231C4F87B
:10C7B000940123B1114A537843F00103537086F07A
:10C7C000C1FBD4F89421B4F89231801A4FF47A72F4
:10C7D000B0FBF2F09842E0D323B9084A537843F013
:10C7E000010353702046FDF74BFC3388044A0621B1
:10C7F0004DF0A6FCD2E700BF806C0020DC86002054
:10C80000002B0D0810B590F89031042B0446164B00
:10C810000AD1D3F8280D03681B69984718B1204640
:10C82000FEF7AAFC002010BD0A79D3F8303DDFEDF9
:10C830000F6A93ED0E6A07EE902A0A7E920748BFB0
:10C840009FED0B7AF8EE677A48BF67EE877A86EE3F
:10C85000267AB0EEC77AB4EEE77AF1EE10FAACBF02
:10C8600001200020DFE700BF806C0020DB0FC94003
:10C870000000803B13B5094B01910446D3F8280D05
:10C8800003681B69984730B10199204602B0BDE8A2
:10C890001040FEF771B902B010BD00BF806C0020DF
:10C8A00010B5044686F04EFBD4F8A831C01AD4F86F
:10C8B000A43198424FF0000084BFC4F8A4010120C5
:10C8C00010BD000038B505460C4686F03BFBD5F898
:10C8D000C831C01A23894FF47A725343984294BFE7
:10C8E0000020012038BD0000C368186808B190F826
:10C8F000B808704710B5012104460A4805F00EF843
:10C9000028B120460321BDE81040FEF787B949F061
:10C9100027FEBDE8104040F26B124FF4801149F041
:10C92000D7BD00BF5882002090F89031022B04D070
:10C93000032B04D1034804F0C1BF0120704700203D
:10C94000704700BF5882002038B50C4BD3F8885C84
:10C9500090F89031032B044605F004050AD10848ED
:10C9600004F0C4FF94F8903135B110B9023B58423D
:10C97000584138BD0020F5E70120FAE7804C00203F
:10C980005882002010B50F4A137843F080031370CB
:10C990000D4B93F9E020002A044609DBFEF73AFA32
:10C9A00070B920460822BDE810400921FDF73ABAC7
:10C9B000BDE8104001220E21A3F50270F5F712BB6D
:10C9C00010BD00BFDC860020805C0020F8B5D0F8E8
:10C9D000B44105465CB1012C1AD049F0C1FD40F6C6
:10C9E00043024FF4801149F073FD012407E0184B16
:10C9F000D3F8280D03681B69984710B90024204616
:10CA0000F8BD2846FEF740FB0123C5F8B431F6E730
:10CA1000104F97F9E030002BF0DA436A1B6893F867
:10CA2000A160012EEAD13C3027F00AFE044600281E
:10CA3000E5D1D7F8103193F8CB3033B132460D2120
:10CA4000A7F50270F5F7CEFAD9E73446D7E700BF6D
:10CA5000806C0020805C002038B56E4BD3F8EC2051
:10CA60006D4B9A4204460D4601D0002072E04B887F
:10CA70005E2B55D8512B0CD8103B9AB20F2A29D9CE
:10CA80002046FDF7FDFA6B88644A04214DF058FBFF
:10CA900059E0523B0C2BF3D801A252F823F000BF0F
:10CAA000F7CB010881CA0108B9CB0108CDCB010839
:10CAB00081CA010881CA010881CA010881CA010826
:10CAC00081CA010881CA010881CA0108FDCB010899
:10CAD000D5CB01080F2BD3D801A252F823F000BF09
:10CAE000C7CB01086BCA0108DDCB0108E3CB010805
:10CAF000F1CB0108CDCB0108B9CB010881CA0108EF
:10CB000081CA010881CA010881CA010881CA0108D5
:10CB100081CA010881CA010881CA0108E9CB01085C
:10CB2000732B74D006D8702B6ED0722BA8D1FFF760
:10CB30000BFE44E04AF2CF62934262D0A0D8B32BFE
:10CB400009D8B12B9CD92046FDF79AFA298851F0D3
:10CB5000E3FC012038BDBC3B9AB2132A90D8132BBA
:10CB60008ED801A252F823F047CB010847CB010829
:10CB700081CA010881CA010881CA010881CA010865
:10CB800081CA010847CB010881CA010847CB0108C7
:10CB900081CA010881CA010881CA010847CB01087E
:10CBA00081CA010881CA010881CA010847CB01086E
:10CBB00081CA010847CB01082046FFF769FD00281C
:10CBC0003FF453AFBFE7FFF7DDFDF8E72046FFF77F
:10CBD000FDFEF4E71248FFF769FDF0E7FFF712FEEC
:10CBE000EDE7FFF769FDEAE7BDE83840FFF77ABDFA
:10CBF000FFF780FDE3E7FFF73DFEE0E7FFF750FEBC
:10CC0000DDE7FFF75FFEDAE7FFF78AFDD7E7FFF71B
:10CC1000ADFDD4E7805C0020087C0020882D0D0845
:10CC20003C85002090F89031032B0BD0062B06D0CA
:10CC3000012B0AD1C368186803681B6818470448A9
:10CC400002F012BA034804F0C3BE0020704700BFD0
:10CC5000FC800020588200208B88012B05D00B69B6
:10CC60003BB94B692BB9CB681BB904480021F9F7D4
:10CC7000F7BE024800220831F9F714BF802C0020CB
:10CC800010B54B885E2B04460A464DD8512B05D86B
:10CC9000103B99B20F2921D900209DE0523B0C2B6B
:10CCA000FAD801A151F823F013CE010899CC01085C
:10CCB000CDCD0108E3CD010899CC010899CC01083C
:10CCC00099CC010899CC010899CC010899CC0108AC
:10CCD00099CC01081BCE010823CE01080F2BDBD80D
:10CCE00001A151F823F000BFDBCD0108EDCD010813
:10CCF000F5CD0108FDCD01080DCE0108E3CD0108F9
:10CD0000CDCD010899CC010899CC010899CC010836
:10CD100099CC010899CC010899CC010899CC01085B
:10CD200099CC010805CE0108B32B00F0848016D8F9
:10CD3000732B7DD00ED8702B77D0722BACD1D1ED68
:10CD4000027A9FED447A67EE877AFDEEE77AC0EDCE
:10CD50006B7A40E0B22B9FD1FFF7E0FB3BE0CD2B9D
:10CD60002CD8BB2B98D9BC3B112B95D801A151F8DD
:10CD700023F000BFD7CD0108D7CD010899CC010819
:10CD800099CC010899CC010899CC010899CC0108EB
:10CD90003DCE010899CC01083DCE010899CC01088F
:10CDA00099CC010899CC01083DCE010899CC010825
:10CDB00099CC010899CC010849CE01084AF2CF620A
:10CDC00093427FF469AFFFF727FB04E002F108010B
:10CDD0002046FEF745F8012010BD1146FFF72CFA5A
:10CDE000F9E711462046FFF78BF8F4E71146FFF705
:10CDF000C7F8F0E71146FFF7FDF8ECE71146FFF73B
:10CE000027F9E8E71146FFF72FF9E4E7FFF772FD8E
:10CE1000E1E71146FFF758FADDE71146FFF7C2FADE
:10CE2000D9E71146FFF7E6FBD5E7FFF715FBD2E799
:10CE3000FFF726FBCFE7FFF70FFFCCE7064802F12D
:10CE40000801F9F7C1FAC6E711462046FFF7A8FB2B
:10CE5000C1E700BF0000C842EC840020704700001A
:10CE6000704700007047000090F8280080F0010033
:10CE700070470000024B436040F605030381704792
:10CE80000001020490F85501704700000F20704720
:10CE90000020704700207047002070470020704736
:10CEA00000487047342E0D0800487047402E0D088A
:10CEB00008B5094800F50053D3F8DC3CB3F9083055
:10CEC00000EE103AB8EEC00AF5F726FBBDE80840C0
:10CED0000248FCF709BF00BF802C0020E07D002045
:10CEE00010B514482DED028B1C4600F5005300F5DB
:10CEF0008040B3F9A832D0F81C0D08EE103A036850
:10CF000082B09B6ECDE900219847B8EEC88AF0EE5A
:10CF1000400ADDE90021B0EE480A0748FCF734FB7F
:10CF20000548FCF743FF84ED000A02B0BDEC028B1C
:10CF300010BD00BF802C0020E07D0020F8B51C4D06
:10CF400005F5005405F580462846D6F8247DF5F70A
:10CF5000D1FAB4F9E43201EE103AB4F9E23200EE5B
:10CF6000903A434200EE103AB8EEC11AF8EEE00AE9
:10CF7000B8EEC00A384679F073FC2846D6F8246D1E
:10CF8000F5F7B8FAB4F9E43201EE103AB4F9E23246
:10CF900000EE903A434200EE103A3046B8EEC11A25
:10CFA000BDE8F840F8EEE00AB8EEC00A79F0D2BC6D
:10CFB000802C002038B5144C04F5804504F57F64BE
:10CFC000D5F81C0D03689B689847692100F194020D
:10CFD000204649F0A3FFD5F81C0D0368DB6898478D
:10CFE0006A2100F19402204649F098FFD5F81C0D03
:10CFF00003681B6998476B2100F194022046BDE845
:10D00000384049F08BBF00BF802C0020014807F05A
:10D010000FB800BF802C00203C3084F059BB0000CA
:10D0200008B549F09DFABDE8084072224FF480111E
:10D0300049F04EBA08B549F093FABDE808406622B7
:10D040004FF4801149F044BA08B549F089FABDE8B7
:10D05000084080224FF4801149F03ABA73B51F4D51
:10D060000646D5F8EC0003681B6B9847044680B36E
:10D0700095F9E130002B2FDBD5F8103193F8CB4038
:10D080003CB395F8E03003F0A003202B24D1D5F871
:10D09000EC0003681B689847052808D0D5F8EC0019
:10D0A00003681B689847A0F110035C425C410C4A7E
:10D0B00002F550630193A2F500532146D3F8F43DE5
:10D0C0000093D2F8243DD2F81C2D304684F0AEFAFD
:10D0D0000446204602B070BD0024FAE7805C0020C0
:10D0E000806C00203C30FFF7B9BF000038B5114D0F
:10D0F00004461148F5F7AAFE95F9E030002B14DA42
:10D10000236A93F8A120012A06D0D5F8EC0000216B
:10D11000BDE83840FCF756BB0D21A5F50270F4F7C9
:10D1200061FF95F9E030002BEFDB2046BDE8384089
:10D1300084F0B8BD805C0020802C00203C30FFF7DC
:10D14000D5BF0000012070470120704701207047C3
:10D150000120704711207047012070470020704760
:10D16000002070470020704700487047842F0D084A
:10D17000004870478C2F0D0838B5436904461D6878
:10D1800080697CF0ABFF25F071F8DFED1B0A2846C3
:10D1900079F04CF96369A0691D687CF09FFF25F068
:10D1A00065F8DFED150A284679F0B8F96369186863
:10D1B0007AF088FB6369DFED110A18689FED0E1A9B
:10D1C000B0EE600A79F04CFB6369DFED0C0A186879
:10D1D0009FED091AB0EE600A79F0BCFB636918682C
:10D1E00079F052FC18B9636918687AF0D1FD002310
:10D1F0002364012038BD00BF00803B4400007A4317
:10D2000070B52DED028B88B00446FCF7A3FA70B11F
:10D2100020460021FCF7D6FA63699FED310A1868B1
:10D2200008B0BDEC028BBDE870407AF08DBE636A39
:10D23000022118687DF00AFF2A4B93F8E1305B0663
:10D2400003D56369186879F071F99FED258A6069E3
:10D250008DED018A8DED028A8DED038A8DED048AB4
:10D2600003AA01A90068012379F0CAF96369186863
:10D270007AF03EFC236A1D682B68DE6C63691868CF
:10D2800079F012FD0122CDED060A8DED071A05A9F0
:10D290008DED050A2846B0EE480AB0476369B0EE46
:10D2A000480A186879F062FB636918687AF0BEFE74
:10D2B000236C8BB185F046FEE36BC01A236C984259
:10D2C0000AD309480C220521FCF7BAFB20B906480D
:10D2D0000C220221FCF7B4FB08B0BDEC028B70BD40
:10D2E00000000000805C0020802C002038B504463F
:10D2F0000D4685F027FEC4E90F0538BD07207047AD
:10D3000001207047002070470020704701207047BF
:10D310000048704724300D08004870472C300D0835
:10D3200070B52DED028B0025C36880F83C501B685A
:10D33000DFED488AD3ED0A0A42699FED478A93EDF3
:10D34000060AF4EEE80A0446F1EE10FA88B0106816
:10D35000B8BFF0EE480A79F069F8E36862691B68C3
:10D360001068D3ED0A0A93ED060AF4EEE80AF1EE2E
:10D3700010FAB8BFF0EE480A79F0D0F86369204699
:10D380001E68FCF781FE6368B3F93820B3F93630C4
:10D3900000EE903A434201EE102A00EE103AB8EE49
:10D3A000C11AF8EEE00AB8EEC00A304679F058FA31
:10D3B000636920461E68FCF767FE6368274CB3F973
:10D3C0003820B3F9363000EE903A434200EE103A7E
:10D3D00001EE102A3046B8EEC11AF8EEE00AB8EEB7
:10D3E000C00A79F0B7FAD4F8300D7BF03BF9D4F8E5
:10D3F000306D338B1B0723D504A80FF0ADFC09F06B
:10D400002BFE9FED170A044606F11C0024F030FBAA
:10D4100001AA04A920468DED010ACDED020A8DED89
:10D42000031A09F0E7FD80B10322294604A80FF092
:10D4300099FC0C4B186804AA90F8791058F004FA7B
:10D4400009480821F8F7D8FE012008B0BDEC028B8E
:10D4500070BD00BF0000003400007A43806C0020E3
:10D460000AD7233C68900020EC84002030B52DEDD5
:10D47000048BC3689FED898A1B684269D3ED0A7AE1
:10D48000DFED870A93ED060AF4EEC87AF1EE10FAA2
:10D490000446A8BFF0EE670A106889B078F0C6FFAE
:10D4A000636920461D68FCF7EFFD6368B3F9382017
:10D4B000B3F9363000EE903A434200EE103A01EEF6
:10D4C000102A2846774DB8EEC11AF8EEE00AB8EEF9
:10D4D000C00A79F0C5F9D5F8300D7BF005FAA5F54D
:10D4E000805393F80531D90747D4D5F8303D1A8BCE
:10D4F000D20742D593ED0A9AB4EEC89AF1EE10FA2B
:10D50000B8BF93ED049AE36A186855F01FFBD5F88D
:10D51000283DD3ED067AA36B20EE270AD3ED007ADF
:10D52000F0EE498AE0EE278AB0EE490AF5EEC08AAD
:10D53000F1EE10FAD8BFDFED5C8AF0EE680A20F059
:10D540005FFF28B9D5F8300DB0EE680A7AF04AFFCF
:10D55000636893F95130272B0FD0A36A186855F0F0
:10D56000F5FAF0EEC07AF4EEC87AF1EE10FAB0EE09
:10D57000407A20D5002384F83C30236B1B68B3F934
:10D58000083000EE103A2046B8EEC00AFCF73EFC28
:10D590002046FCF7A9FB2046B0EE408AFCF7DAF8FB
:10D5A000002848D00021204609B0BDEC048BBDE81E
:10D5B0003040FCF707B9D5F8303D9FED3C0AD3ED7C
:10D5C0000F7AD3ED0B6AA36B27EE800AF4EEC86ADC
:10D5D000D3ED007AF1EE10FA67EE277A10DB9FEDBB
:10D5E000341ADFED310A552037EE800A21F00CF8AD
:10D5F000012384F83C30D5F8300D7AF0E3FEBCE727
:10D600009FED2C7AF4EEC76AF1EE10FA05D89FED83
:10D61000261ADFED290A5920E6E7F0EEE66AF4EE75
:10D62000C86AF1EE10FAE3D594F83C30002B08BF3D
:10D63000B0EE670ADCE7636A022118687DF006FD38
:10D640001E4806F0ADFBB0EE480AD5F8300D7BF071
:10D650004DF801461A48FAF789FD636918687AF0AF
:10D66000E5FC236A1D686369186879F01DFB05AC49
:10D67000204614498DED020ACDED030A8DED041A02
:10D68000F8F7B0FF079B009394E80C0002A9284626
:10D6900076F0D6FB09B0BDEC048B30BD0000003441
:10D6A00000007A43806C002000000000E02E6542FC
:10D6B0000000B442000000B40000B4C2005A0020D0
:10D6C000802C0020EC84002008B5064BD3F8303DB8
:10D6D000D868243023F018FFFCEEC07A17EE900AC9
:10D6E00008BD00BF806C0020024BD3F8303DD868E5
:10D6F00079F084BB806C00200B20704701207047BC
:10D700000020704701207047002070470048704794
:10D71000C4300D0800487047CC300D080120704718
:10D7200008B5DFED237AF4EEE70AF1EE10FA2DEDFD
:10D73000028BF0EE408AB0EE608A35DDDFED1D7AB7
:10D74000F4EEE70AF1EE10FA2ED5F6EE007A70EE5E
:10D75000E77ADFED196A9FED190ADFED190AF0EE9D
:10D76000E77A87EEA67A8720B7EE001A30EE470AEE
:10D7700020F04AFFDFED137A9FED131ADFED130A55
:10D7800020EE270A8A2020EE280A20F03DFF30EE06
:10D79000080ABDEC028BDFED0A0ABDE808408D20C7
:10D7A000B7EE001A20F030BF9FED050AEFE700BF8B
:10D7B000AC1C5A3ED578493F8FC2753E9A99993F25
:10D7C00000000000FAEDEBBA9A99993E9A9999BE39
:10D7D00030B52DED048B7D4BB3F9A83200EE903AB5
:10D7E000F8EEE00A83B0044601AA6946B0EE600A8A
:10D7F000FBF7CAFEA0697CF071FCE369D0ED008AFA
:10D80000D3ED946AD3ED977A90ED016AA3689FED0A
:10D81000701ADFED700A27EEE80A68EEA68A03F6B2
:10D820003813E6EE278A05463B20DFED6B7AB0EE33
:10D83000E87AB4EEE77AF1EE10FA58BFB0EE677A04
:10D84000DFED667AC7EE275AF7EE007A77EEE57AD3
:10D850009DED007A67EE877A93ED007A67EE877A1E
:10D860009FED5F7AA6EE260A87EE879A20F0CCFE1F
:10D870003C209FED571ADFED570AB0EE408AB0EE1C
:10D88000680A20F0C1FE626B564B1268DFED567AD3
:10D89000B2F90820D3ED006A9FED541ADFED540A67
:10D8A00007EE102AB8EEC77AF0EE408A27EE277A04
:10D8B000DFED507AA6EEA77A4520F4EE007AA7EEC7
:10D8C000678ABAEE000A28EE000A83ED007A8DED31
:10D8D000000A20F099FEDDED017A9FED477A474B73
:10D8E0008DED000AF0EEE77AF4EEC77AF1EE10FA69
:10D8F00051D593ED007ADFED427A77EE277AB2EEDA
:10D90000007AF4EEC77AF1EE10FA58BFF0EE477ADB
:10D91000C3ED007A67EEA87ACDED017A636A1868E4
:10D9200090F8CB10002939D17DF090FB636A1B6819
:10D9300093F8A110012939D0032940D039B9236ABD
:10D94000186876F065FF236A186876F0B1F9236AE3
:10D95000DDED010A18689DED000A0368B0EE491A72
:10D96000DB6A9847204695ED028AFCF709F82046C5
:10D97000F0EE400AB0EE480AFFF7D2FE236A626872
:10D980001868D2ED020A036801215B6E984703B064
:10D99000BDEC048B30BD00221A60BFE7194B93F930
:10D9A000E130002BB4BF01210221BDE7236A1868D2
:10D9B00076F02EFF236A186876F090F9C7E7D979D8
:10D9C0000029C4D12046FCF755FBC0E7804C00205D
:10D9D00000000C4400000CC40000FA4400409C45C8
:10D9E00000003442588500200AD7233D00A08C4512
:10D9F00000A08CC58FC2753F000000345C850020FC
:10DA00008FC2F53C805C00200E20704700207047DC
:10DA100000207047002070470020704700207047AA
:10DA20000048704764310D080048704764310D08A4
:10DA300070B52DED028B436A1B6893F8CB3004461A
:10DA4000FBB9052384F848302046FBF799FF636A49
:10DA500002211868B0EE408A7DF0F8FA94F950304F
:10DA6000E2696BB3D2F8F8515D4394F84820052A77
:10DA70004FD8DFE812F02B005F008400B100DF0018
:10DA80001E01836A1B68B3F90830002BB8BF5B42E4
:10DA90009BB2B3F57A6FD4D2C36A1B68B3F908306E
:10DAA000002BB8BF5B429BB2B3F57A6FC9D285F049
:10DAB00049FAE36CC01A40F6C4139842C1D8C3E7D0
:10DAC00094F95150D2F8FC215543CEE7226A94F9DB
:10DAD000511010689FED801A49F64042534351435C
:10DAE00000EE103A00EE901A0268F8EEE00A926B2F
:10DAF000B8EEC00A9047DFED797A41F293139D4268
:10DB000038EE278A05DD94F950308BB1012384F873
:10DB10004830236A62681868D2ED020A0368B0EEE2
:10DB2000480ABDEC028B5B6EBDE8704000211847CF
:10DB30000223ECE7226A9FED681A106849F640421A
:10DB4000534300EE103A0268B8EEC00A926BF0EE52
:10DB5000410A9047DFED627A38EE678A05F50C5589
:10DB6000B5EEC08AF1EE10FA05F1270543F2BA438B
:10DB7000D8BF9FED598A9D42CBD80423C7E7236ABB
:10DB80009FED551A186894F9513049F640425343B5
:10DB900000EE903A0268F8EEE00A926BB0EE410AAD
:10DBA0009047DFED4F7AE36938EE678AD3F8F831B2
:10DBB000B5EEC08AF1EE10FAD8BF9FED478A002B70
:10DBC000B8BF5B4242F228329342A2DD41F2941385
:10DBD0009D429EDD03239AE7236A9FED3F1A186852
:10DBE00094F9513049F64042534300EE903A0268AE
:10DBF000F8EEE00A926BB0EE410A9047DFED387A1A
:10DC0000E36938EE678AD3F8F831B5EEC08A03F5D8
:10DC10000C53F1EE10FA03F1270344F24E62D8BF21
:10DC20009FED2D8A93423FF674AF2E4B9D42FFF637
:10DC300070AFA2E7236A94ED111A1868D4ED100AA8
:10DC4000036894ED0F0A1B6B00219847DFED237AE0
:10DC500094F95020E36938EE278A1AB393ED7E7A5F
:10DC6000D4ED0F7AB8EEC77A77EEC77A9FED1E7AB9
:10DC7000F0EEE77AF4EEC77AF1EE10FA3FF649AF2C
:10DC80000D2294F849101948FBF7DAFE024618B93C
:10DC900001461648FBF7D4FE4AF056F916214AF021
:10DCA0008FF836E793ED7F7AD4ED107AB8EEC77A25
:10DCB000DAE70D2294F849100C48FBF7C1FE024642
:10DCC00018B901460948FBF7BBFE4AF03DF90222AC
:10DCD0000D214AF095F81CE700000000CDCC4C3E29
:10DCE0008FC2753E6DEEFFFF0000FA43802C0020CE
:10DCF00073B5474D0446D5F8EC0003685B6B984755
:10DD000018B90026304602B070BD95F9E130002BFD
:10DD10005FDBA36A1B68B3F90830002BB8BF5B4216
:10DD20009BB2B3F57A6FECD2636A1B6893F8CB6051
:10DD3000002EE6D095F9E030002BE2DBD5F8EC00C0
:10DD400003681B689847002584F8490084F8485008
:10DD500085F0F8F8E36AE064A4F850501B68B3F962
:10DD60000830B3F5967F43DD012384F851304AF043
:10DD7000EBF815214AF024F8264BB3F9A83201EE4E
:10DD8000103AE369B8EEC11A93ED7E0A8DED011ADF
:10DD9000F1EE410A5320B8EEC00ACDED000A20F0A2
:10DDA00033FCE36984ED0F0A93ED7F0A9DED011AC0
:10DDB000DDED000AB8EEC00A542020F025FCE3692E
:10DDC00084ED100AD3ED807AF8EEE77AC4ED117A8B
:10DDD00098E7D5F8EC0003681B689847012890D0B5
:10DDE000D5F8EC0003681B689847002891D188E7B4
:10DDF00013F5967F01DAFF23B7E7A36A1B68B3F92F
:10DE00000830002BACBF0123FF2384F85030AEE76D
:10DE1000805C0020804C0020162070470020704756
:10DE200000207047012070470020704781F00100FA
:10DE3000704700000120704700487047FC310D0812
:10DE400000487047CC120D0803681BB1007900F040
:10DE50000100704718467047F0B5494D95F9356E89
:10DE600085B00446A5F50055002E00F08580454894
:10DE7000FFF7EAFF064600287ED0636920461F6848
:10DE8000FCF702F96368B3F93820B3F9363000EED5
:10DE9000903A434201EE102A00EE103AB8EEC11A51
:10DEA000F8EEE00AB8EEC00A384678F0D9FC6369AB
:10DEB00020461F68FCF7E8F86368B3F93820B3F927
:10DEC000363000EE903A434200EE103A01EE102A4E
:10DED0003846B8EEC11AF8EEE00AB8EEC00A78F09B
:10DEE00039FD05F58043D3F8240D78F0CDFD18B940
:10DEF0006369186879F04CFFB5F9A43004F13C006F
:10DF00001BB9B5F8A230A5F8A430B5F8A43007EED7
:10DF1000903AF8EE677A04F1980203A90027CDED54
:10DF2000037A4BF0D5FC04F15C00C4F8A0700190BA
:10DF30006CF032FF002384F8A530B5F9A4300198C5
:10DF40001BB9B5F8A230A5F8A430B5F8A43007EE97
:10DF5000903AF8EEE77AB7EE000A80EE270A6CF006
:10DF60003FFF09487CF0B6F8C4F8C870DFED077AC7
:10DF700020EE270A84ED310A304605B0F0BD00BF1F
:10DF8000804C0020B05A0020807900200AD7233C22
:10DF900010B50446FBF7BCF92046154B40F83C3B56
:10DFA0004BF022FC134B2365134B9FED142A9FED7E
:10DFB000141ADFED140A9FED140A6365F1EE041ADA
:10DFC00004F15C006CF022FF002320460F49C4F8E6
:10DFD000A830C4F8AC30C4F8B030C4F8B430C4F8D9
:10DFE000B830C4F8BC3042F07FFB204610BD00BF03
:10DFF00004330D08CDCCCC3D000040400AD7233B74
:10E0000000803B459A99993ECDCC4C3E9C320D0800
:10E010002DE9F0432DED028B9BB0914604460D4651
:10E0200084F090FFB8499FEDB98A0646A1F1080037
:10E0300023F09CF994ED161ACDED110A7E20F1EE35
:10E04000410A8DED100A20F0DFFA94ED161A8DEDDD
:10E05000100AF1EE410A7F209DED110A20F0D4FA5A
:10E0600010A904F13C008DED110A4BF04FFCA848BB
:10E07000CDED130A8DED120A7CF02CF8D4ED327A36
:10E08000D4ED140A94ED151AE0EE087A892004F113
:10E090005C074FF00008B0EE670A20F0B5FA12A84E
:10E0A00023F0B0F99B4812A909F028FA14A93846C0
:10E0B0008DED140ACDED150A6CF04EFD3846CDF805
:10E0C0005880CDF85C806CF08BFD8DED160ACDED9F
:10E0D000170AB9F1000F00F001810123C4F8D060E4
:10E0E00084F8CC308C4E04F1A80116A823F066F910
:10E0F000B6F9A83200EE103A16A8B8EEC00A23F01E
:10E1000081F916A9A6F5556009F0E4F918A9284681
:10E110008DED180ACDED190A23F050F9B6F9A832A1
:10E1200095ED007A07EE903AF8EEE77AB0EEC77A0E
:10E13000B4EEE77AF1EE10FA00F3CE8095ED017AB5
:10E14000B0EEC77AF4EEC77AF1EE10FA4CBF0123B5
:10E15000002384F8A530B6F9A83295ED000A5A429A
:10E1600007EE903A00EE902AB8EEE71AF8EEE00AD1
:10E17000CA2020F049FA85ED000AB6F9A83295EDDB
:10E18000010A5A4200EE902A07EE903AF8EEE00AB1
:10E19000B8EEE71ACB2020F037FA85ED010A94F8A3
:10E1A000A4305A1C84F8A4201422B3FBF2F102FB21
:10E1B0001133DBB2002B34D149F0C6FE064684F0A1
:10E1C000C9FE8046D4F8AC000F46F2F79DF9CDE9C0
:10E1D0000E01D4F8A800F2F797F9CDE90C01D4F8B4
:10E1E000A000F2F791F9CDE90A016868F2F78CF91D
:10E1F000CDE908012868F2F787F9CDE906011398FF
:10E20000F2F782F9CDE904011298F2F77DF9CDE930
:10E210000087CDE90201414B414A4249304649F06D
:10E2200009FC1BB0BDEC028BBDE8F08312A823F003
:10E230006BF9DFED3D7AB4EEE70AF1EE10FA57D450
:10E2400094F8CC3063B956E038466CF029FD94F868
:10E25000CC3084ED2A0AC4ED2B0A002B3FF442AFE8
:10E26000DFED325ADFED324A9FED324ADFED323ACE
:10E2700012AA2B4605F10801B2EE0E5AB7EE003A8B
:10E28000B2EC016A94F99D00B0EEC67A67EE256A99
:10E2900007EE900A76EE842AF8EEE77AB0EE647A1A
:10E2A000A7EE857AC3EEA27A27EE087A77EE837A14
:10E2B00027EE267AB5EEC06A67EE877AF1EE10FA9D
:10E2C00048BFF1EE677AE3EC017A9942D8D1CDF8F4
:10E2D0005C80CDF8588005E701233AE794F8CC300C
:10E2E0004BB1D4F8D00040F6B833361A9E429DD9CF
:10E2F000002384F8CC3094F8A530002BA4D1384604
:10E300006CF034FDA3E700BFDC5A00200AD7233CA1
:10E3100080790020303F0020804C0020A0FD0C08B8
:10E3200008320D08CC120D089A99993E0000C84297
:10E330000000BE42000070420000FA432DE9F04F99
:10E340002DED048B0446A5B0BD487BF0C3FEBD4B4C
:10E35000DFEDBD7A1B68DB6A93F89C3060EE278A9C
:10E3600033B9F1EE687AC4ED327AC4ED318A47E010
:10E37000B64D05F54053D3F8103193F8A090B9F19C
:10E38000020FEED184F0DEFD05F58043D3F8343D75
:10E39000C01A40F2DB539842E3D99FEDAD8A95F85D
:10E3A000DB1B8DED218A18AB21AA05F6C8008DED87
:10E3B000228A8DED238A1EF04FFC08B3A54821A9BF
:10E3C00021F0D6F9D4ED2C7A8DED210A37EE800AB2
:10E3D000D4ED2D7ACDED220A77EEA00A9E4884ED89
:10E3E0002C0AC4ED2D0A8DED231AFFF72DFD60B91F
:10E3F00084F0A8FD84ED2D8AC4F8C00084ED2C8A39
:10E4000025B0BDEC048BBDE8F08F05F5005BD4F8BA
:10E41000C020DBF8643E42B9C4F8C03084ED2D8AD8
:10E4200084ED2C8A84ED328AEAE79A42E8D08B4860
:10E4300004F1B00109F04EF889498DED190AF1EEA9
:10E44000607AA1F1080010EE108A17EE907ACDEDF7
:10E450001A0ACDED1B7A8DED1C0A22F087FFDBF83E
:10E46000643ED4F8C0208DED1D0AA3EB020ABAF574
:10E47000FA7FCDED1E0A04F1B8051DAE0CD996E861
:10E480000300C4F8C03084ED2D8A84ED2C8A85E821
:10E490000300C4ED318AC5E72946304622F066FF05
:10E4A00096E8030085E8030094ED329ADBF8643EB9
